:020000040000FA
:04000000ADEF00F070
:100008005582D9CF05F0DACF06F00F0112A91BD01F
:100018008EBC02D0839483928EA802D083A20ED085
:10002800899425EE04F0010EDBBE07D0000EDE5CDD
:10003800020EDE5802E3899201D089828EB883B21B
:1000480001D08984129912A17CD08EB883B289928A
:10005800901C076E8E1C086E04C509F005C50AF0D1
:100068000ABE03D0020E0A5C2FE28EA802D083A239
:100078002BD0094A0A2A09C004F50AC005F502C5A9
:1000880009F003C50AF0060E0924D96E050E0A20E8
:10009800DA6E07C0DFFF060E0924D96E070E0A20A4
:1000A800DA6E08C0DFFF094A0A2A0168010E026EEB
:1000B80009C003F00AC004F00150031602500416E8
:1000C80003C002F504C003F58EB883B2898489841D
:1000D8008EA0FED78EA802D083A202D0899401D028
:1000E800898425EE04F0010EDBBE07D0FB0EDE5C32
:1000F800010EDE5802E3899201D0898208A81FD038
:100108000BD0838202D0838405D0839418D083A235
:1001180016D08394839213D007507F0B016E026A26
:1001280002500DE10150040AF2E0100AF0E0340A2E
:10013800E8E01F0AEFE07F0AE6E01F0AE6E00F01A9
:1001480012910E01CA9906C0DAFF05C0D9FF55926F
:10015800110053EF50F07DC0D9FF7EC0DAFFDE6A90
:10016800DD6A7CC00BF0F8EC45F00BC098F00CC0D1
:1001780099F0000199BF0B0CD8909835D96E993534
:10018800DA6E860ED926010EDA22DECFAFF0DDCF89
:10019800B0F0AF51B01101E10C0C7DC0D9FF7EC0A9
:1001A800DAFFAFC0DEFFB0C0DDFF7F91AFC0D9FF7F
:1001B800B0C0DAFFDF5012E020EE01F0AF51D926CF
:1001C800B051DA22DF5035EC60F00001A46FA4B121
:1001D80005D07F51D8A4A4A5000C0A0CAFC0D9FF44
:1001E800B0C0DAFFDF6A20EE01F0AF51D926B05176
:1001F800DA2298C0DFFF20EE01F0AF51D926B051C6
:10020800DA22DF509AEC42F00001A46FA4B1030C8B
:100218007F5102E0A4B50A0CAFC060F0B0C061F035
:10022800636B626B93EC46F060C0ADF061C0AEF0FA
:10023800040EAD19AE1101E1010CAE5103E1020E3D
:10024800AD5D01E30D0C20EE2BF0AF51D926B05176
:10025800DA22DECFA0F0DECFA1F0DECFA2F0DECF33
:10026800A3F03A0EAF250B6E000EB0210C6E1AECFF
:100278005EF0020E0C180B1001E00D0C450E00018B
:10028800AF250B6E000EB0210C6E1AEC5EF00BC0A1
:10029800A9F00CC0AAF00001AB6BAC6BA951AA1174
:1002A800AB11AC1110E1530EAF250B6E000EB0214F
:1002B8000C6E44EC53F00BC0A9F00CC0AAF00DC0B2
:1002C800ABF00EC0ACF0000120EE17F0AF51D9260C
:1002D800B051DA22A9C0DEFFAAC0DEFFABC0DEFF44
:1002E800ACC0DEFF20EE3FF0AF51D926B051DA2284
:1002F80010EE02F0AF51E126B051E222DFCFE7FF66
:1003080020EE02F0AF51D926B051DA22DE040AE01D
:1003180020EE02F0AF51D926B051DA22020EDE18D3
:1003280001E00D0CA9C00BF0AAC00CF0ABC00DF099
:10033800ACC00EF020EE02F0AF51D926B051DA224F
:10034800DF500F6E106A116A126A07EC57F00BC083
:10035800A9F00CC0AAF00DC0ABF00EC0ACF020EEB6
:100368003CF0AF51D926B051DA22DF50806F816B53
:1003780020EE09F0AF51D926B051DA2280C0DEFF55
:1003880081C0DDFF20EE09F0AF51D926B051DA2245
:10039800DE50DE10D8B40D0C20EE09F0AF51D9268E
:1003A800B051DA22DECF80F0DDCF81F08269836937
:1003B80020EE09F0AF51D926B051DA22DECF84F011
:1003C800DDCF85F08251842783518523805184179E
:1003D800815185178451851101E00D0C400EAF2520
:1003E8000B6E000EB0210C6E1AEC5EF0000120EED0
:1003F80007F0AF51D926B051DA220BC0DEFF0CC08E
:10040800DDFF20EE07F0AF51D926B051DA22DF50D8
:10041800806F0F0E801701E00D0C420EAF250B6E9A
:10042800000EB0210C6E1AEC5EF00BC09CF00CC0F4
:100438009DF000019E6B9F6B9C519D119E119F1119
:1004480010E14F0EAF250B6E000EB0210C6E44EC80
:1004580053F00BC09CF00CC09DF00DC09EF00EC078
:100468009FF03D0E0001AF250B6E000EB0210C6E03
:100478001AEC5EF00BC09AF00CC09BF000019A5188
:100488009B1101E10D0C20EE07F0AF51D926B051B8
:10049800DA22DECF80F0DDCF81F0040E826FD890B3
:1004A80081338033822FFBD79A518025836F9B51EC
:1004B8008121846F856BD8B0852B866BA9518325E4
:1004C800946FAA518421956FAB518521966FAC51D9
:1004D8008621976F94519C5D95519D5996519E59CF
:1004E80097519F5901E20D0C94519C5D0B6E9551EB
:1004F8009D590C6E96519E590D6E97519F590E6ECF
:1005080020EE09F0AF51D926B051DA22DECF80F0C3
:10051800DDCF81F080C00FF081C010F0116A126A3F
:1005280087EC57F00BC0A5F00CC0A6F00DC0A7F0E3
:100538000EC0A8F00001A551A611A711A81101E14C
:100548000D0CAD6BAE6BF60EA55DFF0EA659FF0E3A
:10055800A7590F0EA85903E2AE6B030EAD6FA85151
:10056800A71108E1F60EA55DFF0EA65903E2AE6BD2
:10057800020EAD6FA851A71108E1F60EA55D0F0E8A
:10058800A65903E2AE6B010EAD6FAD51AE1101E19C
:100598000D0C020EA525806F000EA621816F000E9E
:1005A800A721826F000EA821836F20EE13F0AF51B0
:1005B800D926B051DA2280C0DEFF81C0DEFF82C0BA
:1005C800DEFF83C0DEFF20EE1BF0AF51D926B0510D
:1005D800DA22A0C0DEFFA1C0DEFFA2C0DEFFA3C0FA
:1005E800DEFF9A51A025806F9B51A121816F000EDB
:1005F800A221826F000EA321836F20EE1FF0AF515E
:10060800D926B051DA2280C0DEFF81C0DEFF82C069
:10061800DEFF83C0DEFF9451A025806F9551A12194
:10062800816F9651A221826F9751A321836F20EE8B
:1006380027F0AF51D926B051DA2280C0DEFF81C041
:10064800DEFF82C0DEFF83C0DEFF030EAD19AE11F0
:100658004DE1590EAF250B6E000EB0210C6E1AEC51
:100668005EF00B500C1001E00D0C000120EE07F0BD
:10067800AF51D926B051DA22DE50DE1001E00D0C60
:100688005B0EAF250B6E000EB0210C6E44EC53F0E0
:10069800000120EE23F0AF51D926B051DA220BC069
:1006A800DEFF0CC0DEFF0DC0DEFF0EC0DEFF20EE59
:1006B80013F0AF51D926B051DA22DECF80F0DECF69
:1006C80081F0DECF82F0DECF83F0020ED890803743
:1006D800813782378337E82EF9D780C090F081C000
:1006E80091F082C092F083C093F0B8D020EE07F06A
:1006F800AF51D926B051DA22DE50DE1001E10D0CDF
:1007080020EE1FF0AF51D926B051DA22DECF80F0AB
:10071800DECF81F0DECF82F0DECF83F0A9518025D5
:10072800846FAA518121856FAB518221866FAC51AC
:100738008321876F20EE23F0AF51D926B051DA22FA
:1007480084C0DEFF85C0DEFF86C0DEFF87C0DEFF17
:10075800020EAD19AE116BE020EE13F0AF51D926A1
:10076800B051DA22DECF80F0DECF81F0DECF82F02A
:10077800DECF83F0010E8015846F856B866B876BE7
:1007880020EE13F0AF51D926B051DA22DECF88F02F
:10079800DECF89F0DECF8AF0DECF8BF0030E880340
:1007A800F3CF8CF0F4CF8DF08E6B8F6B8903F35001
:1007B8008D27F4508E23000E8F238803F3508D2746
:1007C800F4508E23000E8F23030E8A03F3508E27D6
:1007D800F4508F23000E8903F3508E27F4508F2393
:1007E800000E8803F3508E27F4508F23030E8B03DB
:1007F800F3508F27000E8A03F3508F27000E8903CA
:10080800F3508F27000E8803F3508F27D8908F332B
:100818008E338D338C3384518C25906F85518D2187
:10082800916F86518E21926F87518F2116D020EEBD
:1008380013F0AF51D926B051DA22DECF80F0DECFE7
:1008480081F0DECF82F0DECF83F0D8908035906FD4
:100858008135916F8235926F8335936FFF0E9025A6
:10086800806F010E9121816F000E9221826F000E20
:100878009321836F0A0E05D0D89083338233813356
:100888008033E82EF9D720EE17F0AF51D926B051B2
:10089800DA228051DE5C8151DE588251DE58835164
:1008A800DE5801E20D0C20EE0FF0AF51D926B05101
:1008B800DA22DE68DE68DE68DD68DD52DD5210EEC1
:1008C8000BF0AF51E126B051E222DECFE6FFDECFDA
:1008D800E6FFDECFE6FFDECFE6FF20EE04F0AF5105
:1008E800D926B051DA22800EDF6E030EAD19AE1193
:1008F80001E090D05F0EAF250B6E000EB0210C6E9C
:100908001AEC5EF00B040C1001E084D0AFC037F095
:10091800B0C038F0010E0001A025396E000EA121EB
:100928003A6E000EA2213B6E000EA3213C6E39ECFC
:1009380054F000096FE1000120EE04F0AF51D92610
:10094800B051DA22DF6A2D0EAF250B6E020EB021F0
:100958000C6E1AEC5EF0550E0B185CE1AA0E0C1822
:1009680059E12F0E0001AF250B6E000EB0210C6E61
:1009780044EC53F0520E0B184DE1520E0C184AE19C
:10098800610E0D1847E1410E0E1844E1130E0001E7
:10099800AF250B6E020EB0210C6E44EC53F0720EB4
:1009A8000B1838E1720E0C1835E1410E0D1832E1C2
:1009B800610E0E182FE1170E0001AF250B6E020E07
:1009C800B0210C6E44EC53F0000120EE0FF0AF5153
:1009D800D926B051DA220BC0DEFF0CC0DEFF0DC0F5
:1009E800DEFF0EC0DEFF1B0EAF250B6E020EB02120
:1009F8000C6E44EC53F0000120EE0BF0AF51D926F9
:100A0800B051DA220BC0DEFF0CC0DEFF0DC0DEFFE6
:100A18000EC0DEFFAFC0D9FFB0C0DAFFADC0DFFF48
:100A28000101844B852B000120EE05F0AF51D9263A
:100A3800B051DA2284C1DEFF85C1DDFF000C74C02D
:100A480077F075C078F001017A6B7B6B91D373C036
:100A580048F0770E496E76C04AF04950D96EDA6A86
:100A6800DECFF6FFDDCFF7FFF86A000EF86E08005C
:100A7800F550250AD8A45ED34950D96EDA6ADE2A21
:100A8800000EDD2201017C6B7D6B4B6A4C6A7E692E
:100A98007F694950D96EDA6ADECFF6FFDDCFF7FFFE
:100AA800F86A000EF86E0800F550640AD8B40FD042
:100AB8004950D96EDA6ADECFF6FFDDCFF7FFF86A64
:100AC800000EF86E0800F550690AD8A47ED1495086
:100AD800D96EDA6ADE2A000EDD224A50D96EDA6A49
:100AE800DF50DF2ADF2AD96EDA6ADECF62F0DDCF87
:100AF80063F00001000E63BFFF0E646F656F666FE1
:100B0800676F686F696F48C025F062C026F063C0E0
:100B180027F064C028F065C029F066C02AF067C0D5
:100B28002BF068C02CF069C02DF026C03EF027C01D
:100B38003FF028C040F029C041F02AC042F02BC045
:100B480043F02CC044F02DC045F045AE02D0010E54
:100B580001D0000E3C6E3D6A3C503D10D8B410D018
:100B6800451E441E431E421E411E401E3F1E3E6C33
:100B7800000E3F22402241224222432244224522A3
:100B880001017FBF01D04B927FBF05D07F5107E1A4
:100B98007E05D8B004D0396A010E386E04D07EC103
:100BA80038F07FC139F07CC13AF07DC13BF03C5050
:100BB8003D10D8A402D04BA403D03A06D8A03B06D7
:100BC800476A1F0E466E0201B86B6ED04606D8A063
:100BD8004706990E4624D96E020E4720DA6E3EC0AB
:100BE8000BF03FC00CF040C00DF041C00EF042C009
:100BF8000FF043C010F044C011F045C012F00A0EC7
:100C0800136E146A156A166A176A186A196A1A6AD4
:100C180003EC4AF00BC02EF00CC02FF00DC030F0E2
:100C28000EC031F00FC032F010C033F011C034F0F4
:100C380012C035F02EC01DF030C01EF065EC5EF01D
:100C48001D50300FDF6E3806D8A039063A06D8A0F6
:100C58003B063EC00BF03FC00CF040C00DF041C059
:100C68000EF042C00FF043C010F044C011F045C070
:100C780012F00A0E136E146A156A166A176A186A51
:100C8800196A1A6A56EC45F00BC03EF00CC03FF0EA
:100C98000DC040F00EC041F00FC042F010C043F04C
:100CA80011C044F012C045F047BE1FD0475003E1C1
:100CB8004604D8A01AD03E503F10401041104210B0
:100CC800431044104510D8A481D739BE05D03950F7
:100CD80002E13804D8B07AD73BBE07D03B5003E1D5
:100CE8003A04D8A002D04BB271D73C503D10D8A4DA
:100CF80002D04BA415D04606D8A047063C503D105C
:100D0800D8A403D0376A2B0E02D0376A2D0E366E60
:100D1800990E4624D96E020E4720DA6E36C0DFFFE0
:100D280025C01AF0990E46241B6E020E47201C6E31
:100D38003AC01DF03BC01EF04BA008D01BC014F0F9
:100D48001CC015F01AC016F0ABEC5EF01EBE05D044
:100D58001DC022F01EC023F002D0226A236A206A36
:100D6800216A0AD0000E0D6E200E0C6E1AC00EF00D
:100D780080EC56F0204A212A2250205C2150800A1B
:100D88001F6E2350800A1F58D8A0ECD74BB008D04C
:100D98001BC014F01CC015F01AC016F0ABEC5EF0C6
:100DA8001BC00BF01CC00CF05BEC5CF022500B2459
:100DB8001A6E23500C201B6E1AC025F01BC026F09B
:100DC80025C048F026C049F0CED14950D96EDA6A1C
:100DD800DECFF6FFDDCFF7FFF86A000EF86E0800E9
:100DE800F550780AD8B40FD04950D96EDA6ADECFF8
:100DF800F6FFDDCFF7FFF86A000EF86E0800F55031
:100E0800580AD8A46DD14950D96EDA6ADECFF6FFF8
:100E1800DDCFF7FFF86A000EF86E0800F5CF72F024
:100E28004950D96EDA6ADE2A000EDD224A50D96EA0
:100E3800DA6ADF50DF2ADF2AD96EDA6ADECF60F09D
:100E4800DDCF61F060C06AF061C06BF000016C6BCF
:100E58006D6B6E6B6F6B706B716B48C024F06AC002
:100E680025F06BC026F06CC027F06DC028F06EC06E
:100E780029F06FC02AF070C02BF071C02CF072C03E
:100E88002DF001017FBF01D04B927FBF05D07F516C
:100E980007E17E05D8B004D0376A010E366E04D05B
:100EA8007EC136F07FC137F07CC140F07DC141F092
:100EB8004BA804D0FE0E4026FF0E412225C038F074
:100EC80026C039F027C03AF028C03BF029C03CF0D2
:100ED8002AC03DF02BC03EF02CC03FF0456A1F0EE3
:100EE800446E0201B86B6DD04406D8A045060F0EBB
:100EF8003814426E436A43BE08D0435004E10A0ED8
:100F0800425CD8A002D0570E01D0300E4226000E07
:100F18004322BF0E2E6E2F682D50306E316A2E5030
:100F280030262F503122315005E11A0E305C02E292
:100F3800010E01D0000E326E336A32503310D8B42D
:100F480025D09F0E2E6E2F68200E4210306E000E98
:100F58004310316E2E5030262F503122315005E18A
:100F68001A0E305C02E2010E01D0000E346E356AB2
:100F780034503510D8B40AD042C011F043C012F032
:100F880018EC5CF011C042F012C043F0990E4424F2
:100F9800D96E020E4520DA6E42C0DFFF3606D8A0B1
:100FA80037064006D8A04106040E2E6ED8903F3270
:100FB8003E323D323C323B323A32393238322E2ED2
:100FC800F5D745BE20D0455004E1020E445CD8A0B8
:100FD8001AD0385039103A103B103C103D103E10D2
:100FE8003F10D8A481D737BE05D0375002E1360468
:100FF800D8B07AD741BE07D0415003E14004D8A009
:1010080002D04BB271D74BA816D04406D8A04506DB
:10101800990E4424D96E020E4520DA6E2DC0DFFFEA
:101028004406D8A04506990E4424D96E020E4520E0
:10103800DA6E300EDF6E24C01AF0990E44241B6E4F
:10104800020E45201C6E40C01DF041C01EF04BA092
:1010580008D01BC014F01CC015F01AC016F0ABEC79
:101068005EF01EBE05D01DC022F01EC023F002D0C7
:10107800226A236A206A216A0AD0000E0D6E200EA9
:101088000C6E1AC00EF080EC56F0204A212A22502D
:10109800205C2150800A1F6E2350800A1F58D8A058
:1010A800ECD74BB008D01BC014F01CC015F01AC008
:1010B80016F0ABEC5EF01BC00BF01CC00CF05BEC48
:1010C8005CF022500B241A6E23500C201B6E1AC0A1
:1010D80024F01BC025F024C048F025C049F043D0B7
:1010E8004950D96EDA6ADECFF6FFDDCFF7FFF86A2E
:1010F800000EF86E0800F550250AD8A412D0495001
:10110800D96EDA6ADE2A000EDD22000E0D6E250E7B
:101118000C6E48C00EF080EC56F0496A010E486E1D
:1011280022D04950D96EDA6ADE2A000EDD22486ADA
:10113800496A19D04950D96EDA6ADECFF6FFDDCF99
:10114800F7FFF86A000EF86E0800F5500C6E0D6A8D
:1011580048C00EF080EC56F04950D96EDA6ADE2AA3
:10116800000EDD22DAD7485001017A2749507B2347
:1011780077C0F6FF78C0F7FF0800F55001E067D4A4
:101188007AC173F07BC174F0120097C0ADF098C0BB
:10119800AEF09B51D96EDA6ADE6ADD6A95C00CF052
:1011A80096C00DF0BD0E0E6E9AEC52F00001AC6FB9
:1011B800AC510AE120EE0FF09551D9269651DA226A
:1011C800DF50AC6FAC5102E0AC51120020EE0EF0D3
:1011D8009551D9269651DA22DFA2070C20EE10F09D
:1011E8009551D9269651DA2210EE10F09551E12644
:1011F8009651E222E6CFA0F0E6CFA1F0E6CFA2F02A
:10120800E6CFA3F09951A025A46F9A51A121A56F0B
:10121800000EA221A66F000EA321A76FDE50A45DC9
:10122800DE50A559DE50A659DE50A75901E3DFD29A
:1012380020EE10F09551D9269651DA22DECF9CF097
:10124800DDCF9DF09C1D996F9D1D9A6FD0D220EE29
:1012580010F09551D9269651DA22FF0EDE149C6FB4
:10126800010EDE149D6F000EDE149E6F000EDE145C
:101278009F6F9C519D119E119F1101E0FDD120EEA1
:1012880010F09551D9269651DA22DECF9CF0DECFA8
:101298009DF0DECF9EF0DECF9FF00A0E05D0D890ED
:1012A8009F339E339D339C33E82EF9D7A069A169FB
:1012B80020EE09F0BD51D926BE51DA22DECFA2F0C8
:1012C800DDCFA3F0A051A227A151A3239C51A215C1
:1012D800AF6F9D51A315B06FAF1101E091D020EE13
:1012E80010F09551D9269651DA22DE50DE10DE1024
:1012F800DE101EE120EE06F09551D9269651DA222D
:10130800DECFB7F0DECFB8F0DECFB9F0DECFBAF07F
:10131800B751B811B911BA1127E195C078F096C044
:1013280079F07A6B7B6B7C6B7D6BEBEC22F014D0E5
:1013380095C078F096C079F020EE14F09551D92632
:101348009651DA22DECF7AF0DECF7BF0DECF7CF06A
:10135800DECF7DF0EBEC22F078C0B7F079C0B8F0C2
:101368007AC0B9F07BC0BAF0B751B811B911BA1147
:1013780001E141D2B705B811B911BA1109E120EE5E
:101388000FF09551D9269651DA22020EDF6E020C23
:10139800B7290FE1B8290DE1B9290BE1BA2909E10B
:1013A80020EE0FF09551D9269651DA22010EDF6E04
:1013B800010C20EE14F09551D9269651DA22B7C0C7
:1013C800DEFFB8C0DEFFB9C0DEFFBAC0DEFF20EE28
:1013D80006F09551D9269651DA22DE50DE10DE103D
:1013E800DE100EE120EE06F09551D9269651DA224C
:1013F800B7C0DEFFB8C0DEFFB9C0DEFFBAC0DEFF8F
:1014080020EE18F09551D9269651DA2210EE2BF0DD
:10141800BD51E126BE51E222DE50E61812E1DE504F
:10142800E6180FE1DE50E6180CE1DE50E61809E197
:10143800BDC024F0BEC025F058EC43F0000901E01F
:1014480053D1BDC00BF0BEC00CF0000120EE14F06B
:101458009551D9269651DA22DECF0DF0DECF0EF067
:10146800DECF0FF0DECF10F091EC4AF00BC0B3F0F6
:101478000CC0B4F00DC0B5F00EC0B6F00001B35109
:10148800B411B511B61101E17AD7AF51B327B051F4
:10149800B423000EB523B62399C09CF09AC09DF0E2
:1014A800090E9E6FD8909D339C339E2FFBD79CC00E
:1014B800B1F09DC0B2F0B151B21101E1A2D0B15169
:1014C800AF259C6FB251B0219D6F20EE09F0BD5140
:1014D800D926BE51DA229C51DE5C9D51DE5810E2BD
:1014E80020EE09F0BD51D926BE51DA22DECF9CF09C
:1014F800DDCF9DF0AF519C5DB16FB0519D59B26F7A
:10150800ADC01AF0AEC01BF0B3C01CF0B4C01DF0E3
:10151800B5C01EF0B6C01FF0B1C020F0B2C021F0B7
:1015280020EE01F0BD51D926BE51DA22DF5004EC7D
:101538004FF0000901E0D8D00001B1519C6FB251C1
:101548009D6F9E6B9F6B20EE2BF0BD51D926BE512F
:10155800DA22DECFA0F0DECFA1F0DECFA2F0DECF20
:10156800A3F0B351A05DA46FB451A159A56FB551B3
:10157800A259A66FB651A359A76F9C51A45D9D515E
:10158800A5599E51A6599F51A7592CE22F0EBD254A
:101598000B6E000EBE210C6E20EE2BF0BD51D9262D
:1015A800BE51DA22DECF9CF0DDCF9DF0B3519C5FB7
:1015B800B4519D5B090ED8909C379D37E82EFBD718
:1015C8009C51AD250D6E9D51AE210E6E020E106E12
:1015D8000F6A7CEC5CF020EE03F0BD51D926BE51B9
:1015E800DA22DF6AB1C09CF0B2C09DF0090ED89033
:1015F8009C379D37E82EFBD79CC0BBF09DC0BCF044
:10160800A7D020EE0AF09551D9269651DA2210EE8D
:1016180010F09551E1269651E222DE50E65CDE504C
:10162800E658DE50E658DE50E65818E3BDC024F010
:10163800BEC025F058EC43F0000901E055D0000188
:1016480020EE2BF0BD51D926BE51DA22B3C0DEFF01
:10165800B4C0DEFFB5C0DEFFB6C0DEFF20EE18F076
:101668009551D9269651DA22B3C0DEFFB4C0DEFF09
:10167800B5C0DEFFB6C0DEFF9C69010E9D6F20EE8F
:1016880010F09551D9269651DA22DECF9EF0DDCFA3
:101698009FF09C519E179D519F179E510008BB6F4C
:1016A8009F51D8A0E82A0208BC6FBB51995DBC5174
:1016B8009A5904E299C0BBF09AC0BCF0BDC037F09B
:1016C800BEC038F020EE18F09551D9269651DA228E
:1016D800DECF39F0DECF3AF0DECF3BF0DECF3CF0A4
:1016E80039EC54F0000902E000015AD600019C6967
:1016F800010E9D6F20EE10F09551D9269651DA22F1
:10170800DECF9EF0DDCF9FF09C519E179D519F1715
:10171800BDC0A0F0BEC0A1F09E51A0279F51A1233B
:101728002F0EA0250B6E000EA1210C6EADC00DF082
:10173800AEC00EF0BBC00FF0BCC010F07CEC5CF08B
:1017480020EE03F0BD51D926BE51DA22010EDF6E1C
:10175800BB51995FBC519A5B9B51D96EDA6ABB51F8
:10176800DE26BC51DD22BB51AD27BC51AE2320EE95
:1017780010F09551D9269651DA22BB51DE26BC517C
:10178800DE22000EDE22DE2220EE10F09551D92650
:101798009651DA2210EE0AF09551E1269651E2228E
:1017A800DE50E65CDE50E658DE50E658DE50E6587D
:1017B80020EE0AF0D8A020EE10F09551D9269651C7
:1017C800DA22DECFA8F0DECFA9F0DECFAAF0DECF96
:1017D800ABF020EE0AF09551D9269651DA22A8C02E
:1017E800DEFFA9C0DEFFAAC0DEFFABC0DEFF995155
:1017F8009A1101E02CD520EE0EF09551D92696517C
:10180800DA22000EDB8C000C0C6E0B6A9DD20C5099
:1018180009E14F5007E00B6A0101836B0A0E8FD074
:10182800839004D3020E0C1807E14F5005E00B6AB1
:101838000101836B140E83D01F0E0C6437D0300E59
:101848000C6034D04F5032E00C50E00F506E0B6AF1
:101858000F0E501805E191C14EF00101916B56D25F
:101868005050220D0A0EF324D96E030EF420DA6EBE
:10187800DE50DE10DE10DE1003E0030E506446D2A8
:10188800010E4E6E50501C0D1B0EF324D96E010E26
:10189800F420DA6E50501C0D1B0EF324E16E010E7D
:1018A800F420E26EE7500409DF6E30D23F0E0C647C
:1018B80012D0500E0C600FD04F500DE050501C0D40
:1018C800000EF324D96E010EF420DA6E0C50C00F0E
:1018D800DF6E0B6A1BD2310E0C1807E14F5005E082
:1018E8000C0E0101836F1D0E26D2340E0C1807E171
:1018F8004F5005E00101826B836B0B6A91D7350E5F
:101908000C1808E14F5006E00B6A0D0E0101836FB9
:10191800AC0E15D0370E0C1808E14F5006E0838046
:101928000E0E0101836F750E06D20D0E0C1809E11B
:101938004F5007E00B6A020E0101836FBC0E826FE5
:101948006FD7100E0C1807E14F5005E0030E010188
:10195800836FE90EF0D1180E0C1807E14F5005E01F
:10196800070E0101836F090EE6D13B0E0C1807E143
:101978004F5005E00E0E0101836F7E0EDCD13E0E46
:101988000C1801E053D24F5001E150D20F0E010163
:10199800836F3D0ED0D150501C0D010EF324D96E2B
:1019A800010EF420DA6E0CC0DFFF030E0101836F15
:1019B800EA0EC1D150501C0D020EF324D96E010E4F
:1019C800F420DA6E0CC0DFFF030E0101836FEB0E0B
:1019D800B2D150501C0D030EF324D96E010EF42021
:1019E800DA6E0CC0DFFF030E0101836FEC0EA3D18A
:1019F80050501C0D040EF324D96E010EF420DA6E3B
:101A08000CC0DFFF030E0101836FED0E94D150501F
:101A18001C0D050EF324D96E010EF420DA6E0CC0ED
:101A2800DFFF030E0101836FEE0E85D150501C0DB0
:101A3800060EF324D96E010EF420DA6E0CC0DFFF17
:101A480050501C0D060EF324D96E010EF420DA6EE8
:101A5800DF50606F60C061F0626B636B646B63C082
:101A680064F062C063F061C062F0616B61C065F0F0
:101A780062C066F063C067F064C068F0696B68BFF5
:101A8800696969C06AF069C06BF069C06CF0505050
:101A98001C0D050EF324D96E010EF420DA6EDF500A
:101AA8006D6F6DC06EF06F6B706B716B6FC071F0A6
:101AB8006EC070F06F6B6E6B6EC072F06FC073F0BB
:101AC80070C074F071C075F0766B75BF766976C0BA
:101AD80077F076C078F076C079F050501C0D040E7F
:101AE800F324D96E010EF420DA6EDF507A6F7AC0D3
:101AF8007BF07C6B7D6B7E6B7BC07EF07D6B7C6B43
:101B08007B6B7BC07FF07CC080F07DC081F07EC0A5
:101B180082F0836B82BF836983C084F083C085F0C1
:101B280083C086F050501C0D030EF324D96E010EAD
:101B3800F420DA6EDF50876F87C088F0896B8A6B74
:101B48008B6B8C6B8D6B8E6B8F6B200ED890883760
:101B580089378A378B378C378D378E378F37E82E12
:101B6800F5D77F518825906F80518921916F8151D8
:101B78008A21926F82518B21936F83518C21946FAC
:101B880084518D21956F85518E21966F86518F21B5
:101B9800976F72519025986F73519121996F745175
:101BA80092219A6F755193219B6F765194219C6F66
:101BB800775195219D6F785196219E6F7951972184
:101BC8009F6F65519825A06F66519921A16F675144
:101BD8009A21A26F68519B21A36F69519C21A46F20
:101BE8006A519D21A56F6B519E21A66F6C519F2153
:101BF800A76F50501C0D070EF324D96E010EF42068
:101C0800DA6EA0C0DEFFA1C0DEFFA2C0DEFFA3C067
:101C1800DEFFA4C0DEFFA5C0DEFFA6C0DEFFA7C0B2
:101C2800DEFF83900101826B836B00D150501C0D45
:101C38001A0EF324D96E010EF420DA6E0CC0DFFF01
:101C4800070E0101836F0A0E76D050501C0D190E35
:101C5800F324D96E010EF420DA6E0CC0DFFF070EF4
:101C68000101836F0B0E67D050501C0D180EF32422
:101C7800D96E010EF420DA6E0CC0DFFF070E0101E9
:101C8800836F0C0E58D050501C0D170EF324D96ECC
:101C9800010EF420DA6E0CC0DFFF38D00101826B30
:101CA800836B4E6ABDD50CC08FF20F0E0101836F96
:101CB8003E0E41D00CC090F20F0E0101836F3F0E13
:101CC8003AD00CC091F20F0E0101836F400E33D051
:101CD8000CC092F20F0E0101836F410E2CD00CC084
:101CE80093F20F0E0101836F420E25D00CC094F2BF
:101CF8000F0E0101836F430E1ED00CC095F20F0E1C
:101D08000101836F440E17D00CC096F20101826B5B
:101D1800836B86D50C0E0101836F1E0E0CD00C0E42
:101D28000101836F1C0E826F0A0E0B6E79D50E0EA1
:101D38000101836F760E826F79D00101826B836B0C
:101D4800090E0B6E838072D082C160F083C161F08E
:101D58000001615111E0030A13E0040A25E00B0AAF
:101D680031E0010A35E0030A39E0010A40E0130ACC
:101D780058E03B0A59E05AD0605101E148D556D0A5
:101D88006051E90A01E107D6030A01E113D6010A05
:101D980001E11FD6070A01E12BD6010A01E137D676
:101DA800030A01E143D642D06051090A01E13ED756
:101DB800030A01E14AD7010A01E156D7070A01E1FE
:101DC80062D734D060511D0AA5E0030AA8E02ED0DE
:101DD8006051480A01E126D7E40A28D06051750A03
:101DE800A6E0030AAAE0080A01E158D71FD060510B
:101DF8003D0A01E158D7030A01E15CD7010A01E174
:101E080060D77F0A01E164D7010A01E168D7030AB4
:101E180001E16CD7010A01E170D7070A01E174D723
:101E280005D060512A0A02D060510F0A0B501200E7
:101E38000C6A0B6AE8EC5FF00101FB6F956B070E0B
:101E48008C6E010EFD6F9B6B0F0E0F01596F116B9E
:101E5800196B216B266B2E6B886889688A688A8E55
:101E6800889088928382020E0101FC6F04EC5FF077
:101E780088948384889C839C889E838E8B688968D9
:101E88001C0E00019C6FFA0E9D6FA80E9E6FFF0E30
:101E98009F6FF40EA06FFE0EA16F360EA26FFF0E9D
:101EA800A36F0AEC60F08A98858834EC5EF0DE0E49
:101EB80000019C6FFB0E9D6FFBC19EF09F6B0AECAF
:101EC80060F00101FB2901E1FB6B0F0EFB17A0EC91
:101ED8004BF00101FB6FF60E00019C6FFB0E9D6F2E
:101EE800FBC19EF09F6B0AEC60F00400520E0101EA
:101EF800EF6F2B0EEE6F000EE82EFED7EE2FFCD7FD
:101F0800EF2FFAD700F0D250F00B0109D26ED09E15
:101F18000E01C691CF0ECF16CF82CF80C2890F0196
:101F2800138113891489F28E0E01BA89DFEC58F0F7
:101F38008392839491EC4EF091EC4EF0000E0B6E70
:101F4800340ECBEC5BF0510E0F6EFF0E106E4AECA8
:101F580057F0A80E0F6EFF0E106E4AEC57F0000EE9
:101F68000B6E390ECBEC5BF08FA22FD0290E01013E
:101F7800EF6F960EEE6F7F0EE82EFED7EE2FFCD792
:101F8800EF2FFAD7000E0B6E800ECBEC5BF0730EC2
:101F98000F6EFE0E106E4AEC57F017D0B50E00010A
:101FA8009C6FFE0E9D6F8FCF9EF09F6B0AEC60F0CA
:101FB800290E0101EF6F960EEE6F7F0EE82EFED709
:101FC800EE2FFCD7EF2FFAD704008FB2E7D7838024
:101FD800040075EC49F00101F36F22EC33F00101C4
:101FE800F36F945102E070EC3EF0FEC193FF10ECE9
:101FF80030F0BFEC50F0000E0B6E800ECBEC5BF0B7
:1020080019EC5FF0000E0B6E800ECBEC5BF001015B
:10201800FB510F0D350EF3240F6E0D0EF420106ECC
:102028004AEC57F001019BBFB3EC44F00101FD51AC
:102038000CE0AF0E00019C6FFD0E9D6F0AEC60F086
:10204800020E0101996F220E0BD09F0E00019C6FAA
:10205800FD0E9D6F0AEC60F0010E0101996F040EF0
:10206800986FF26BF86B000EF66F010EF56FF6BF06
:1020780005D0F65166E1040EF55D63E20F0EF50337
:10208800F3CFEEF1F4CFEFF1F603F350EF27250E7F
:10209800EE250B6E0E0EEF210C6E5BEC5CF00C5017
:1020A80003E1030E0B5C49E30C0E00019C6FFE0E6E
:1020B8009D6F0F0E0101F503F3CFEEF1F4CFEFF1B1
:1020C800F603F350EF27250EEE2500019E6F0E0E46
:1020D8000101EF2100019F6F0AEC60F0220E01015F
:1020E800F503F3CFEEF1F4CFEFF1F603F350EF275A
:1020F800000EEE250001C96F030E0101EF2100015A
:10210800CA6F0F0E0101F503F3CFF0F1F4CFF1F12F
:10211800F603F350F127250EF0250001CB6F0E0EC4
:102128000101F1210001CC6F030ECD6FF7EC14F023
:102138000101F36FF3517AEC5BF00101F54BF62BDB
:1021480096D7960502E1070E8C6E020E961901E0ED
:1021580030D10F01108B070E2D6F2BD18EA88994CB
:10216800A2EC5FF00B500C1001E1F8D0F8C1F4F1CB
:10217800F70E0B6E010E0C6E3CEC56F00101F86F79
:10218800F7B9F89F9B511BE0350EF81907E14A0E85
:1021980000019C6FFA0E9D6F0AEC60F03F0E000183
:1021A8009C6FFF0E9D6FF8C19EF09F6B0101010EA1
:1021B800F7A9000E0001A06FA16B0AEC60F0680E91
:1021C8000101F81903E1010E26EC60F00101F7A9FD
:1021D80036D0600EF81933E15F0EF41930E1BE0E07
:1021E80000019C6FFC0E9D6FF8C19EF09F6BF4C1BF
:1021F800A0F0A16B010E8EA2000EA26FA36B010EC0
:102208008EA4000EA46FA56B0AEC60F00101FC839C
:102218002BEE35F099C1DFFF2BEE36F098C1DFFFCA
:1022280083841F6A020E1E6EB8EC35F08394010198
:10223800FC93536AC1EC5FF00101F86BBAD0FD5111
:1022480042E0F751100B0001C26F000EC36F01018D
:10225800F85132EC40F0C2C0F9F1C3C0FAF1080EEF
:102268000101F919FA1101E100F0070E0101F9194C
:10227800FA1102E14BEC5AF0F905FA1102E13FECD0
:1022880052F0020EF919FA1102E1F1EC38F0030EDE
:10229800F919FA1103E1E1EC2AF0F26F050EF919C8
:1022A800FA1103E18DEC3DF0F26F090EF919FA11FC
:1022B80002E1E3EC51F00A0E0101F919FA1179E192
:1022C8003BEC60F076D0F751100B1E6E000E1F6EBF
:1022D800F85188EC1CF01EC0F9F11FC0FAF1070E86
:1022E8000101F919FA1102E1B7EC59F0020EF919D6
:1022F800FA1102E182EC59F0F905FA1102E147EC12
:102308001AF0030EF919FA1102E1E6EC4FF0040E87
:10231800F919FA1102E17DEC5EF0050EF919FA11CE
:1023280002E11BEC4BF0060E0101F919FA1102E16A
:1023380043EC60F0080EF919FA1102E1AAEC3CF03E
:10234800090EF919FA1102E11CEC4EF00A0E01010E
:10235800F919FA112EE1FDEC5CF02BD0A0EC4BF052
:102368000101956F965125E0FB51951922E0838E66
:10237800000E0B6EC00ECBEC5BF019EC5FF0000E9C
:102388000B6EC00ECBEC5BF0170E0F6EFF0E106ECF
:102398004AEC57F095C1FBF1000E486E030E496EEA
:1023A8003AEC5DF022EC33F00101945102E070EC5C
:1023B8003EF08FB22ED0050E0101F2192AE0CED6DA
:1023C800B50E00019C6FFE0E9D6F8FCF9EF09F6B28
:1023D8000AEC60F0290E0101EF6F960EEE6F7F0E8A
:1023E800E82EFED7EE2FFCD7EF2FFAD70400000E09
:1023F8000B6EC00ECBEC5BF019EC5FF0000E0B6EB1
:10240800C00ECBEC5BF0590E0F6EFF0E106E4AEC4F
:1024180057F08FB2D5D7090E0101EF6F1E0EEE6F80
:10242800E40EE82EFED7EE2FFCD7EF2FFAD700F0F8
:10243800839483920001B16BB26B4C0EB36FFA0EAA
:10244800B46FB56B66EC55F0C3D595C00CF096C06B
:102458000DF0B30E0E6E9AEC52F00001B56FB55147
:1024680008E120EE0FF09551D9269651DA22DF5077
:10247800B56FB55102E0B551120020EE0AF0955142
:10248800D9269651DA229751DE5C9851DE58995137
:10249800DE589A51DE5816E220EE0EF09551D926F4
:1024A8009651DA22DFB20ED020EE0AF09551D926E5
:1024B8009651DA22DECF97F0DECF98F0DECF99F092
:1024C800DECF9AF020EE10F09551D9269651DA22F7
:1024D800DECFABF0DECFACF0DECFADF0DECFAEF0CE
:1024E800AF6BB06BB16BB26B20EE10F09551D92683
:1024F8009651DA22AFC0DEFFB0C0DEFFB1C0DEFF0A
:10250800B2C0DEFF9751981199119A1101E100D2DA
:1025180020EE09F0B351D926B451DA22DECF9BF070
:10252800DDCF9CF09B519D6F9C519E6F9F6BA06B64
:10253800090ED8909D379E379F37A037E82EF9D7D8
:102548009DC0B6F09EC0B7F09FC0B8F0A0C0B9F06B
:10255800AB51AC11AD11AE1101E196D0FF0E97252C
:102568000B6EFF0E98210C6EFF0E99210D6EFF0E5B
:102578009A210E6EB6C00FF0B7C010F0B8C011F0B7
:10258800B9C012F087EC57F00BC09BF00CC09CF060
:102598000DC09DF00EC09EF0FF0E0001AB250B6E26
:1025A800FF0EAC210C6EFF0EAD210D6EFF0EAE219D
:1025B8000E6EB6C00FF0B7C010F0B8C011F0B9C0B9
:1025C80012F087EC57F00B5000019B5D0C509C59A2
:1025D8000D509D590E509E5957E3FF0EB6259B6F1F
:1025E800FF0EB7219C6FFF0EB8219D6FFF0EB9211A
:1025F8009E6F9B1D9F6F9C1DA06F9D1DA16F9E1DB3
:10260800A26FFF0EAB25A36FFF0EAC21A46FFF0EC8
:10261800AD21A56FFF0EAE21A66F9F51A315A76F21
:10262800A051A415A86FA151A515A96FA251A6156F
:10263800AA6F20EE10F09551D9269651DA22A7C03C
:10264800DEFFA8C0DEFFA9C0DEFFAAC0DEFF20EEC5
:1026580010F09551D9269651DA22DE50975FDE5058
:10266800985BDE50995BDD509A5B20EE14F0955133
:10267800D9269651DA22DECFBAF0DECFBBF0DECF14
:10268800BCF0DECFBDF060D020EE06F09551D92623
:102698009651DA22DECFBAF0DECFBBF0DECFBCF047
:1026A800DECFBDF0BA51BB11BC11BD113FE195C0E1
:1026B80078F096C079F07A6B7B6B7C6B7D6BEBEC7A
:1026C80022F078C0BAF079C0BBF07AC0BCF07BC009
:1026D800BDF0BA05BB11BC11BD1109E120EE0FF028
:1026E8009551D9269651DA22020EDF6E020CBA29CC
:1026F8000FE1BB290DE1BC290BE1BD2909E120EE61
:102708000FF09551D9269651DA22010EDF6E010C91
:1027180020EE06F09551D9269651DA22BAC0DEFF8E
:10272800BBC0DEFFBCC0DEFFBDC0DEFF20EE14F084
:102738009551D9269651DA22BAC0DEFFBBC0DEFF1A
:10274800BCC0DEFFBDC0DEFFBA51BB11BC11BD115C
:1027580001E085D0DDD0B651975FB751985BB8518D
:10276800995BB9519A5B20EE10F09551D926965194
:10277800DA22B651DE26B751DE22B851DE22B9512F
:10278800DE2220EE0EF09551D9269651DA22DFA2EC
:1027980020D095C078F096C079F0BAC07AF0BBC066
:1027A8007BF0BCC07CF0BDC07DF0EBEC22F078C0C3
:1027B800BAF079C0BBF07AC0BCF07BC0BDF0BA51AA
:1027C800BB11BC11BD111BE1976B986B996B9A6B90
:1027D80050D095C042F096C043F0BAC044F0BBC098
:1027E80045F0BCC046F0BDC047F0AFEC2CF042C08D
:1027F800BAF043C0BBF044C0BCF045C0BDF0000116
:10280800BA2907E1BB2905E1BC2903E1BD2901E19A
:1028180076D7BD51BC11BB1104E1020EBA5D01E2CD
:102828005DD720EE13F0B351D926B451DA22DE5029
:10283800BA5DDE50BB59DE50BC59DE50BD5901E3CC
:102848004DD720EE14F09551D9269651DA22BAC008
:10285800DEFFBBC0DEFFBCC0DEFFBDC0DEFF9751A0
:10286800B65D9851B7599951B8599A51B95901E279
:1028780072D720EE10F09551D9269651DA22975149
:10288800DE269851DE229951DE229A51DE22975196
:102898009B6F010E98159C6F9D6B9E6B9B119D11F4
:1028A8009E1136E0B3C00BF0B4C00CF0BAC00DF006
:1028B800BBC00EF0BCC00FF0BDC010F091EC4AF0E8
:1028C8000BC0AFF00CC0B0F00DC0B1F00EC0B2F04C
:1028D8000001AF51B011B111B21101E1FFD697C09B
:1028E8009BF098C09CF099C09DF09AC09EF00A0E8B
:1028F80005D0D8909E339D339C339B33E82EF9D76F
:102908009B51AF279C51B0239D51B1239E51B223B7
:1029180020EE10F09551D9269651DA2210EE0AF0E1
:102928009551E1269651E222DE50E65CDE50E658EB
:10293800DE50E658DE50E6581CE220EE10F09551C5
:10294800D9269651DA2210EE0AF09551E1269651D1
:10295800E222DECFE6FFDECFE6FFDECFE6FFDECF08
:10296800E6FF20EE0EF09551D9269651DA22000E98
:10297800DB8C20EE10F09551D9269651DA22FF0E05
:10298800DE149B6F010EDE149C6F000EDE149D6F2B
:10299800000EDE149E6F9B519C119D119E1101E14A
:1029A8006AD520EE18F09551D9269651DA22AF5102
:1029B800DE180AE1B051DE1807E1B151DE1804E172
:1029C800B251DE1801E157D520EE18F09551D926FD
:1029D8009651DA22AFC0DEFFB0C0DEFFB1C0DEFF25
:1029E800B2C0DEFF48D5C951CA1101E1090C3F0E3A
:1029F800CD17CB0E7C6FB40E7D6F010E7E6FCDC0F0
:102A08007FF0AFEC00F00101B66FB65101E0A8D23B
:102A1800B4C1B7F1B5C1B8F1B70E0001BB6F010E73
:102A2800BC6FCBC0BDF0CCC0BEF002EC41F00101E0
:102A3800B66FB65104E1DEAF02D0060EB66FCDC058
:102A4800CEF01C0E0001CE1701E1D1D00101B65124
:102A58000FE0040EB61909E1B70E0001BF6F010EB1
:102A6800C06F85EC51F00101B66F0001CD870DD024
:102A7800BBC1CEF0110E0001CE1702E0070E03D045
:102A8800CDA503D0080E0101B66F0101B65101E0D2
:102A9800BDD00001CDA7BAD0B4C112F0B5C113F0B2
:102AA800D1C114F0D2C115F0FCEC57F012C0A4F15A
:102AB80013C0A5F114C0A6F115C0A7F10E0E0101AF
:102AC800D1250B6E000ED2210C6E0D6A0E6A210EF6
:102AD8000F6E500E106E4CEC59F0010120EE0BF009
:102AE800D151D926D251DA22200EDF6EB4C10FF0AF
:102AF800B5C110F0D1C111F0D2C112F0136A146A35
:102B0800156A166ADDEC5CF01C0E0101D1250B6E0E
:102B1800000ED2210C6E0D6A0E6A0F6A106A4CEC18
:102B280059F0010120EE03F0B451D926B551DA224B
:102B3800010EDF6EA451A511A611A71167E020EEC2
:102B48002BF0B451D926B551DA22DECFA8F1DECF69
:102B5800A9F1DECFAAF1DECFABF1B70E0001786F95
:102B6800010E796FA4C17AF0A5C17BF0A6C17CF0F3
:102B7800A7C17DF07E6B7F6B806B816BCFEC41F0E2
:102B88000101B66FB65142E1B4C137F0B5C138F0B2
:102B9800A8C139F0A9C13AF0AAC13BF0ABC13CF0D9
:102BA80039EC54F00101B66FFF0EA4250001CE6F79
:102BB800FF0E0101A5210001CF6FFF0E0101A62123
:102BC8000001D06FFF0E0101A7210001D16F0101A3
:102BD80020EE0BF0B451D926B551DA22CEC0DEFF73
:102BE800CFC0DEFFD0C0DEFFD1C0DEFF0FD00101B5
:102BF800B6510CE1BBA902D0040E07D00001CDA349
:102C080005D00101BBA102D0070EB66F0101B65174
:102C180023E10001CDB7CD8D010120EE2BF0B45199
:102C2800D926B551DA22000110EE1CF0C951E1266F
:102C3800CA51E222DECFE6FFDECFE6FFDECFE6FFB7
:102C4800DECFE6FF20EE20F0C951D926CA51DA229C
:102C5800D1C1DEFFD2C1DDFF0101B65101E080D153
:102C6800B4C112F0B5C113F0D1C114F0D2C115F03E
:102C7800FCEC57F0000120EE06F0C951D926CA51E4
:102C8800DA2212C0DEFF13C0DEFF14C0DEFF15C05B
:102C9800DEFF1C0E0101D1250B6E000ED2210C6E39
:102CA80044EC53F0000120EE0AF0C951D926CA516C
:102CB800DA220BC0DEFF0CC0DEFF0DC0DEFF0EC047
:102CC800DEFFC9C0D9FFCAC0DAFFB4C1DEFFB5C193
:102CD800DDFF010120EE05F0B451D926B551DA2205
:102CE800000110EE02F0C951E126CA51E222DECFFE
:102CF800E6FFDDCFE5FF20EE0EF0C951D926CA5117
:102D0800DA22CDC0DFFF20EE0FF0C951D926CA5113
:102D1800DA22DF6A20EE18F0C951D926CA51DA2220
:102D2800DE6ADE6ADE6ADD6A20EE10F0C951D92655
:102D3800CA51DA22DE6ADE6ADE6ADD6ACDAB10D1FC
:102D480020EE0AF0C951D926CA51DA22DE50DE1027
:102D5800DE10DE1001E104D120EE0AF0C951D926B7
:102D6800CA51DA2210EE10F0C951E126CA51E22206
:102D7800DECFE6FFDECFE6FFDECFE6FFDECFE6FF03
:102D8800010120EE09F0B451D926B551DA22DECF7F
:102D9800CEF0DDCFCFF00001CE51D06FCF51D16F43
:102DA800D26BD36B090ED890D037D137D237D337FF
:102DB800E82EF9D7D0C0A0F1D1C0A1F1D2C0A2F1BC
:102DC800D3C0A3F120EE06F0C951D926CA51DA22A0
:102DD800DECFB0F1DECFB1F1DECFB2F1DECFB3F1AD
:102DE80020EE0AF0C951D926CA51DA22DECFACF159
:102DF800DECFADF1DECFAEF1DECFAFF132D0C9C05C
:102E080042F0CAC043F0B0C144F0B1C145F0B2C10C
:102E180046F0B3C147F0AFEC2CF042C0B0F143C06C
:102E2800B1F144C0B2F145C0B3F10101B351B211DF
:102E3800B11105E1020EB05D02E2020EB66FB029D3
:102E480008E1B12906E1B22904E1B32902E1010E42
:102E5800B66FA051AC5FA151AD5BA251AE5BA3515F
:102E6800AF5B0101B65109E1AC51A05DAD51A1596B
:102E7800AE51A259AF51A359C2E3000120EE14F09C
:102E8800C951D926CA51DA22B0C1DEFFB1C1DEFF6D
:102E9800B2C1DEFFB3C1DEFF0101B65161E1AC5141
:102EA8000001CE6F010E0101AD150001CF6FD06B8F
:102EB800D16BCE11D011D11153E0B4C10BF0B5C113
:102EC8000CF0B0C10DF0B1C10EF0B2C10FF0B3C13A
:102ED80010F091EC4AF00BC0A8F10CC0A9F10DC09C
:102EE800AAF10EC0ABF10101A851A911AA11AB11A9
:102EF80003E1020EB66F34D0ACC1CEF0ADC1CFF055
:102F0800AEC1D0F0AFC1D1F00A0E06D00001D89002
:102F1800D133D033CF33CE33E82EF8D70101A851BF
:102F28000001CE25D26F0101A9510001CF21D36F35
:102F38000101AA510001D021D46F0101AB51000158
:102F4800D121D56F20EE18F0C951D926CA51DA22FD
:102F5800D2C0DEFFD3C0DEFFD4C0DEFFD5C0DEFFA7
:102F68000101B65106E0C9C0D9FFCAC0DAFFDE6A5E
:102F7800DD6AB651120076C091F077C092F07AC03F
:102F8800D9FF7BC0DAFFDE6ADD6A74C00CF075C059
:102F98000DF09D0E0E6E9AEC52F000018C6F8C5164
:102FA8000AE120EE0FF07451D9267551DA22DF506C
:102FB8008C6F8C5102E08C51120020EE0EF074518F
:102FC800D9267551DA22DFA0070C20EE10F07451D3
:102FD800D9267551DA22DECF7CF0DECF7DF0DECF48
:102FE8007EF0DECF7FF020EE0AF07451D9267551BD
:102FF800DA22DECF80F0DECF81F0DECF82F0DECFC6
:1030080083F07C51805D886F7D518159896F7E5135
:1030180082598A6F7F5183598B6F78517C6F7951B0
:103028007D6F7E6B7F6B7C51885D7D5189597E51A8
:103038008A597F518B5901E321D288C078F089C021
:1030480079F01CD220EE10F07451D9267551DA228D
:10305800FF0EDE147C6F010EDE147D6F000EDE1491
:103068007E6F000EDE147F6F7C517D117E117F1103
:1030780001E083D120EE10F07451D9267551DA227F
:10308800DECF7CF0DECF7DF0DECF7EF0DECF7FF0CE
:103098000A0E05D0D8907F337E337D337C33E82EFB
:1030A800F9D78069816920EE09F09D51D9269E5192
:1030B800DA22DECF82F0DDCF83F080518227815182
:1030C80083237C518215936F7D518315946F9311DF
:1030D80066E120EE10F07451D9267551DA22DE50DF
:1030E800DE10DE10DE100FE120EE06F07451D92656
:1030F8007551DA22DECF8DF0DECF8EF0DECF8FF085
:10310800DECF90F01CD074C042F075C043F020EEC2
:1031180014F07451D9267551DA22DECF44F0DECF8F
:1031280045F0DECF46F0DECF47F0AFEC2CF042C0E2
:103138008DF043C08EF044C08FF045C090F0000180
:1031480090518F118E110CE1020E8D5D09E220EE77
:103158000FF07451D9267551DA22020EDF6E020C77
:103168008D290FE18E290DE18F290BE1902909E1C5
:1031780020EE0FF07451D9267551DA22010EDF6E58
:10318800010C20EE14F07451D9267551DA228DC045
:10319800DEFF8EC0DEFF8FC0DEFF90C0DEFF9DC069
:1031A8000BF09EC00CF020EE14F07451D926755126
:1031B800DA22DECF0DF0DECF0EF0DECF0FF0DECF5D
:1031C80010F091EC4AF00BC095F00CC096F00DC0D1
:1031D80097F00EC098F0000195519611971198112B
:1031E80001E1B5D79351952794519623000E972363
:1031F800982378C07CF079C07DF0090E7E6FD89056
:103208007D337C337E2FFBD77CC099F07DC09AF04C
:1032180099519A1101E1A3D0995193257C6F9A5144
:1032280094217D6F20EE09F09D51D9269E51DA2216
:103238007C51DE5C7D51DE5810E220EE09F09D5194
:10324800D9269E51DA22DECF7CF0DDCF7DF0935176
:103258007C5D996F94517D599A6F91C01AF092C014
:103268001BF095C01CF096C01DF097C01EF098C0CA
:103278001FF099C020F09AC021F020EE01F09D5176
:10328800D9269E51DA22DF5098EC53F0000901E06C
:10329800ACD0000120EE03F09D51D9269E51DA22D0
:1032A800DF504EE099517C6F9A517D6F7E6B7F6B3A
:1032B80020EE2BF09D51D9269E51DA22DECF80F0E8
:1032C800DECF81F0DECF82F0DECF83F09551805DD6
:1032D800846F96518159856F97518259866F98519D
:1032E8008359876F7C51845D7D5185597E518659FC
:1032F8007F51875925E220EE2BF09D51D9269E510A
:10330800DA22DECF7CF0DDCF7DF095517C5F9651DF
:103318007D5B090ED8907C377D37E82EFBD77C5132
:1033280091250B6E7D5192210C6E2F0E9D250D6EF1
:10333800000E9E210E6E020E106E0F6A7CEC5CF081
:1033480099C07CF09AC07DF0090ED8907C377D3703
:10335800E82EFBD77CC09BF07DC09CF072D020EE9D
:1033680018F07451D9267551DA2295C0DEFF96C03F
:10337800DEFF97C0DEFF98C0DEFF7C69010E7D6F1F
:1033880020EE10F07451D9267551DA22DECF7EF086
:10339800DDCF7FF07C517E177D517F177E5100086D
:1033A8009B6F7F51D8A0E82A02089C6F9B51785DDB
:1033B8009C51795904E278C09BF079C09CF09DC07B
:1033C80037F09EC038F020EE18F07451D9267551A8
:1033D800DA22DECF39F0DECF3AF0DECF3BF0DECFB7
:1033E8003CF039EC54F0000902E00001C1D691C06C
:1033F8000BF092C00CF000017C69010E7D6F20EE8D
:1034080010F07451D9267551DA22DECF7EF0DDCF67
:103418007FF07C517E177D517F179DC080F09EC044
:1034280081F07E5180277F5181232F0E80250D6EDC
:10343800000E81210E6E9BC00FF09CC010F07CEC3A
:103448005CF09B51785F9C51795B7AC0D9FF7BC057
:10345800DAFF9B51DE269C51DD229B5191279C511E
:10346800922320EE10F07451D9267551DA229B511F
:10347800DE269C51DE22000EDE22DE2278517911F2
:1034880001E0E0D5000C50500C0D5F0EF324D96E0E
:10349800020EF420DA6E0001C469C56950500C0DA3
:1034A800670EF324E16E020EF420E26EE6CFC6F05A
:1034B800E5CFC7F0C451C627C551C723DE50C65D46
:1034C800C751800AC86FDE50800AC8594AE3505075
:1034D8000C0D610EF324D96E020EF420DA6EDF5063
:1034E800C26FC36BC469C56950500C0D690EF324D3
:1034F800D96E020EF420DA6EDF50C66FC76BC45166
:10350800C627C551C723C251C65DC751800AC86FB7
:10351800C351800AC85925E350500C0D620EF3249C
:10352800D96E020EF420DA6EDF50C26FC36BC46925
:10353800C56950500C0D6A0EF324D96E020EF420A2
:10354800DA6EDF50C66FC76BC451C627C551C72393
:10355800C251C65DC751800AC86FC351800AC85995
:1035680061E21F0E01018D6F010E8F6F8390730E44
:1035780000019C6FFA0E9D6F50500C0D5F0EF324E6
:10358800D96E020EF420DA6EDECF9EF0DDCF9FF00A
:1035980050500C0D670EF324D96E020EF420DA6E2B
:1035A800DECFC2F0DDCFC3F0FF0EC225A06FFF0E45
:1035B800C321A16F50500C0D610EF324D96E020E79
:1035C800F420DA6EDF50A26FA36B50500C0D690E19
:1035D800F324D96E020EF420DA6EDF50C46FFF0EAA
:1035E800C425A46FA56BFF0EA52350500C0D620EC9
:1035F800F324D96E020EF420DA6EDF50A66FA76BA3
:1036080050500C0D6A0EF324D96E020EF420DA6EB7
:10361800DF50C56FFF0EC525A86FA96BFF0EA92344
:103628000AEC60F050500C0D620EF324D96E020EB5
:10363800F420DA6EDF50C26FC2C0C3F0C46BC56B32
:10364800C66BC5C0C6F0C4C0C5F0C3C0C4F0C36B68
:1036580050500C0D6A0EF324D96E020EF420DA6E67
:10366800DF50C76FC7C0C8F0C96BCA6BCB6B50506F
:103678000C0D610EF324D96E020EF420DA6EDF50C1
:10368800CC6FCCC0CDF0CE6BCF6BD06BCFC0D0F0B1
:10369800CEC0CFF0CDC0CEF0CD6BCD51C803F3CFA7
:1036A800D1F0F4CFD2F0D36BD46BC903F350D22747
:1036B800F450D323000ED423CE51C803F350D2279D
:1036C800F450D323000ED423CD51CA03F350D3278B
:1036D800F450D423CE51C903F350D327F450D42344
:1036E800CF51C803F350D327F450D423CB51CD0383
:1036F800F350D427CE51CA03F350D427CF51C9036E
:10370800F350D427D051C803F350D42750500C0D90
:10371800690EF324D96E020EF420DA6EDF50D56FED
:10372800D5C0D6F0D76BD86BD96B50500C0D6A0E3C
:10373800F324D96E020EF420DA6EDF50DA6FDAC0A5
:10374800DBF0DC6BDD6BDE6B50500C0D5F0EF32491
:10375800D96E020EF420DA6EDECFDFF0DDCFE0F0B6
:10376800DFC0E1F0E0C0E2F0000EE2BFFF0EE36F61
:10377800E46FE151DB03F3CFE5F0F4CFE6F0E76B5C
:10378800E86BDC03F350E627F450E723000EE82348
:10379800E251DB03F350E627F450E723000EE82359
:1037A800E151DD03F350E727F450E823E251DC034D
:1037B800F350E727F450E823E351DB03F350E727FE
:1037C800F450E823DE51E103F350E827E251DD032A
:1037D800F350E827E351DC03F350E827E451DB0317
:1037E800F350E827E7C0E8F0E6C0E7F0E5C0E6F008
:1037F800E56BE551D603F3CFE9F0F4CFEAF0EB6BD4
:10380800EC6BD703F350EA27F450EB23000EEC23BC
:10381800E651D603F350EA27F450EB23000EEC23CD
:10382800E551D803F350EB27F450EC23E651D703C6
:10383800F350EB27F450EC23E751D603F350EB2772
:10384800F450EC23D951E503F350EC27E651D803A3
:10385800F350EC27E751D703F350EC27E851D60390
:10386800F350EC27D151E925ED6FD251EA21EE6FE3
:10387800D351EB21EF6FD451EC21F06FC351ED25FB
:10388800F26FC451EE21F36FC551EF21F46FC651A9
:10389800F021F56F5050220D000EF324956F030EA2
:1038A800F420966FF2C097F0F3C098F0F4C099F046
:1038B800F5C09AF029EC12F0F16FF15111E0C60E43
:1038C8009C6FFB0E9D6FF2C09EF0F3C09FF0F4C09A
:1038D800A0F0F5C0A1F0F1C0A2F0A36B0AEC60F073
:1038E80050500C0D630EF324D96E020EF420DA6EDC
:1038F800F2C0DEFFF3C0DEFFF4C0DEFFF5C0DEFF7E
:1039080001018F6B83901200236E1F5002E0BFEC01
:1039180050F0226A1E5001E1C9D1239E040E2318DB
:1039280002E14D5003E1140E231807E10101806BF9
:10393800816B1F6A070E1E6E070C3F0E231807E1E6
:103948004D6A0101806B816B1E6A1F6A12005F0E4F
:10395800231807E10101906B806B816B1E6A1F6A57
:1039680012003F0E23640BD05F0E236008D0400E78
:10397800231805E00101906B1E6A1F6A1200400EB1
:1039880023180AE1010E0101906F4D6A0101806B55
:10399800816B1E6A1F6A1200200E231801E086D16F
:1039A800010E4D6EF3D7600E231809E10101905105
:1039B80006E08E51080ED8B4030E226E7CD0600E3D
:1039C800231809E14D5007E001018E5102E0090E6C
:1039D80015D0050E13D0680E231809E14D5007E0E5
:1039E8001A0E0101816F900E54D18380BCD1680EEC
:1039F800231806E10101905103E0020E226E5BD00C
:103A08006A0E231807E14D5005E01A0E0101816F77
:103A1800F40E3FD16C0E231807E14D5005E01A0E45
:103A28000101816F2C0E35D1700E231810E10101B0
:103A380090510DE0840E00019C6FFF0E9D6F0AEC03
:103A480060F0040E226E0101806B816BCED7700E80
:103A5800231801E088D14D5001E185D11B0E0101E9
:103A6800816F620E16D18380020E231805E11A0EAB
:103A78000101816F920E806F050E231805E11A0E61
:103A88000101816FAE0E806F070E231805E11A0E33
:103A98000101816FB80E806F080E231805E11A0E18
:103AA8000101816FCC0E806F030E231802E02328DA
:103AB80006E1226A83900101806B816B54D1140E58
:103AC800231805E11A0E0101816F9E0E806F160EF4
:103AD800231801E048D11A0E0101816FA40ECAD043
:103AE800050E231805E11A0E0101816FF50E806F8E
:103AF800080E231801E037D11A0E0101816FCC0E90
:103B0800806F010E8E6F2FD123C050F01A0E010165
:103B1800816F950EAFD02350216E206A50500C0D46
:103B28005F0EF324D96E020EF420DA6E20C0DEFF99
:103B380021C0DDFF1A0E0101816F960E9BD0235024
:103B4800206E216A50500C0D5F0EF324D96E020EC0
:103B5800F420DA6E20C0DEFF21C0DDFF1A0E01015D
:103B6800816F970E87D050500C0D610EF324D96EDB
:103B7800020EF420DA6E23C0DFFF1A0E0101816FF6
:103B8800980E78D050500C0D620EF324D96E020EA8
:103B9800F420DA6E23C0DFFF0101806B816B010E18
:103BA80037D01A0E0101816FB90E73D01A0E0101B8
:103BB800816FBA0E5FD01A0E0101816FBB0E806F44
:103BC800810E00019C6FFE0E9D6F0AEC60F00101F2
:103BD8008F6B806B816B55D00101806B816B810E7F
:103BE80000019C6FFE0E9D6F0AEC60F04AD0220E19
:103BF80000019C6FFF0E9D6F0AEC60F00101806B65
:103C0800816B010E8C6F3DD00101806B816B060EBC
:103C1800226EA9D023C050F00101806B816B226A0B
:103C280030D001018E6B1A0E816FF70E806F29D08C
:103C38001A0E0101816FF70E1DD08390270E010126
:103C4800816F0F0E17D0180E231801E08CD01A0EB2
:103C58000101816F2D0E0ED01A0E0101816F2E0EFB
:103C680009D01A0E0101816F2F0E04D01A0E01011E
:103C7800816F300E806F77D00101806B816B0A0EE7
:103C8800226E839070D0040E226E270E0101816F80
:103C98000F0E806FAAD68380010104D08390010E95
:103CA80001018E6F806B816B226A5DD080C120F02C
:103CB80081C121F0215007E01A0A09E0010A4BE00E
:103CC8003C0A4FE050D0205001E16DD64CD0205036
:103CD8002C0AB9E0010AC0E0030AC3E0010AC6E001
:103CE8001F0ACAE0A00A01E1BED6020A01E10CD708
:103CF800070A01E110D7030A01E121D7010A01E10E
:103D080032D70F0A01E13ED7060A01E170D73A0A15
:103D180001E17AD70A0AC2E0160A01E142D7010A8C
:103D280001E144D7030A01E146D7010A01E154D76A
:103D3800790A01E162D60E0A01E16CD7380A01E17D
:103D4800CFD6010A01E16DD7030A01E171D7010A53
:103D580001E173D708D02050580A95E03A0A9BE051
:103D680002D020500F0A22C01EF01F6A1200020E55
:103D78004A6E65516411631104E1020E625D01E24D
:103D880011D220EE13F06051D9266151DA22DE50AB
:103D9800625DDE506359DE506459DE50655901E2B8
:103DA800EED100D262C048F063C049F0D8904930E3
:103DB8006B6F48306A6F6A5148266B51492260C060
:103DC80037F061C038F020EE1FF06051D9266151FC
:103DD800DA22DECF6AF0DECF6BF0DECF6CF0DECF1A
:103DE8006DF048C06EF049C06FF0090E706FD89042
:103DF8006F336E33702FFBD76E516A25396E6F5152
:103E08006B213A6E000E6C213B6E000E6D213C6EEC
:103E180039EC54F04A6E4A5001E0C4D100016A6995
:103E2800010E6B6F48C06CF049C06DF06A516C1799
:103E38006B516D1760C06EF061C06FF06C516E27EA
:103E48006D516F232F0E6E25466E000E6F21476E43
:103E5800484A492A62B104D066C042F0436A1AD07F
:103E680066516A6F6B6B6A3B6B3BF00E6B176A515E
:103E78000F0B6B13F00E6A1746C0D9FF47C0DAFF65
:103E8800DF500F0B6C6F6D6B6A516C11426E6B518A
:103E98006D11436E46C0D9FF47C0DAFF42C0DFFF4D
:103EA80020EE03F06051D9266151DA22010EDF6E4F
:103EB80060C037F061C038F020EE1FF06051D9269D
:103EC8006151DA22DECF6AF0DECF6BF0DECF6CF024
:103ED800DECF6DF048C06EF049C06FF0090E706F0C
:103EE800D8906F336E33702FFBD76E516A25396EB9
:103EF8006F516B213A6E000E6C213B6E000E6D21E6
:103F08003C6E39EC54F04A6E4A5001E04BD1000146
:103F18006A69010E6B6F48C06CF049C06DF06A5158
:103F28006C176B516D1760C06EF061C06FF06C510B
:103F38006E276D516F232F0E6E25466E000E6F2172
:103F4800476E62B10CD067C06AF00F0E6A1746C0A0
:103F5800D9FF47C0DAFFDF50F00B6A1112D066C0F4
:103F68006AF067C06BF068C06CF069C06DF0050E50
:103F780005D0D8906D336C336B336A33E82EF9D79C
:103F88006A51446E456A46C0D9FF47C0DAFF44C04B
:103F9800DFFF4FD060C037F061C038F020EE1FF06F
:103FA8006051D9266151DA22DECF6AF0DECF6BF09C
:103FB800DECF6CF0DECF6DF063516E6F64516F6FC2
:103FC8006551706F716B6A516E25396E6B516F2137
:103FD8003A6E6C5170213B6E6D5171213C6E39EC1B
:103FE80054F04A6E4A5001E0DDD000016A69010EC2
:103FF8006B6F62C06CF063C06DF0D8906C376D3732
:104008006A516C176B516D1760C06EF061C06FF02C
:104018006C516E276D516F232F0E6E250B6E000E9F
:104028006F210C6E66C00DF067C00EF042EC5FF0B9
:10403800A4D020EE03F06051D9266151DA22010E96
:10404800DF6EB0D060C037F061C038F020EE1FF0EE
:104058006051D9266151DA22DECF6AF0DECF6BF0EB
:10406800DECF6CF0DECF6DF062C06EF063C06FF033
:1040780064C070F065C071F0080E05D0D890713337
:1040880070336F336E33E82EF9D76A516E25396E67
:104098006B516F213A6E6C5170213B6E6D517121DD
:1040A8003C6E39EC54F04A6E4A507CE100016A6972
:1040B800010E6B6F62C06CF063C06DF0D8906C3706
:1040C8006D37D8906C376D376A516C176B516D1717
:1040D80060C06EF061C06FF06C516E276D516F2338
:1040E8002F0E6E250B6E000E6F210C6E44EC53F0F4
:1040F8000001706B716B726BF00E0E14736F66516A
:10410800746F6751756F6851766F0F0E6915776F09
:1041180070517411666F71517511676F7251761114
:10412800686F73517711696F6A69010E6B6F62C0AE
:104138006CF063C06DF0D8906C376D37D8906C37E1
:104148006D376A516C176B516D1760C06EF061C0A6
:104158006FF06C516E276D516F232F0E6E250B6E0D
:10416800000E6F210C6E66C00DF067C00EF068C0BF
:104178000FF069C010F04CEC59F000015AD760C03C
:10418800D9FF61C0DAFFDF506A6F6B6B6B510AE1D0
:104198006A51010A01E106D6030A01E1FBD6010AC8
:1041A80001E150D74A5012002A6E1BC041F01CC0D2
:1041B80042F02A5001E0040C010E3F6E54B0030C8B
:1041C800E9D1DCEC5FF0000901E1FDD13F6AFBD1E8
:1041D800146A156A166A176A090EADEC5DF00009D3
:1041E80001E0F1D12B0E0B6E0C6A0E6A100E0D6EEB
:1041F8007AEC5AF0000901E1E6D12B44E846030BBA
:10420800E8064DE132C01DF03F0E1D161DC01EF020
:104218001F6A206A216A1FC021F01EC020F01F6A91
:104228001E6A3350236E226A3450246E256A225047
:1042380024262350252224501E24266E25501F2074
:10424800276E000E2020286E000E2120296E2628B9
:104258003B6E000E27203C6E000E28203D6E000E9F
:1042680029203E6E3BC01DF03CC01EF03DC01FF033
:104278003EC020F00A0ED8901D361E361F36203656
:10428800E82EF9D71BC0D9FF1CC0DAFF1DC0DEFF1E
:104298001EC0DEFF1FC0DEFF20C0DEFF97D71D6AED
:1042A80035AE01D01D2A010E1D1630C01EF00F0EAE
:1042B8001E163450030B020DF3501E241D24020F4A
:1042C800406E3150030B1D6E1E6A0A0ED8901D36C3
:1042D8001E36E82EFBD732501F6E206AD8901F3644
:1042E8002036D8901F3620363344E846030B216E1B
:1042F800226A1F502126205022221D5021261E509E
:104308002222212A000E222221C03BF022C03CF0AA
:104318003D6A3E6A40C01DF0F70E1D263BC01EF0E8
:104328003CC01FF03DC020F03EC021F01D2A05D042
:10433800D8901E361F36203621361D2EF9D734D098
:1043480051A43FD0146A156A166A176A8D0EADEC2F
:104358005DF0000901E037D12EEC60F02B0E0B6EFA
:104368000C6A0E6A100E0D6E7AEC5AF0000901E123
:104378002AD1300E406E03D02EEC60F0400640503B
:10438800FBE135C01DF01D3A0F0E1D16100E1E6EF6
:104398001F6A206A216A1D2A05D0D8901E361F364A
:1043A800203621361D2EF9D71BC0D9FF1CC0DAFFD5
:1043B8001EC0DEFF1FC0DEFF20C0DEFF21C0DEFF03
:1043C80005D7146A156A166A176A090EADEC5DF00E
:1043D800000901E0F8D02B0E0B6E0C6A0E6A100E65
:1043E8000D6E7AEC5AF0000901E1EDD051A232D0FD
:1043F80038C01DF0060E1E6ED8901D321E2EFCD73A
:10440800FF0E1D2635503F0B1F6E206AD8901F36B1
:1044180020363644010B1F26000E20221F2A202298
:104428001D2A03D0D8901F3620361D2EFBD71F50CB
:10443800216E2050226E236A246A1BC0D9FF1CC03B
:10444800DAFF21C0DEFF22C0DEFF23C0DEFF24C06A
:10445800DEFFBCD63650030B1D6E1E6AD8901D3683
:104468001E36D8901D361E36D8901D361E36363864
:10447800E842070B1D26000E1E221D2A1E2235406B
:10448800E8423F0B1F0B1F6E206A1F2A000E2022D6
:104498001D501F02F3CF21F0F4CF22F02002F35079
:1044A80022261E501F02F35022262150236E22502E
:1044B800246E256A266A1BC0D9FF1CC0DAFF23C0F8
:1044C800DEFF24C0DEFF25C0DEFF26C0DEFF7ED66D
:1044D80041C0D9FF42C0DAFF51C0DFFF77D6146A66
:1044E800156A166A176A090EADEC5DF000096BE1F2
:1044F80041C00BF042C00CF00E6A100E0D6E7AEC43
:104508005AF0000901E062D65ED0146A156A166A8C
:10451800176A0A0EADEC5DF0000955E141C00BF0D9
:1045280042C00CF00E6A100E0D6E7AEC5AF0E9D704
:10453800146A156A166A176A3A0EADEC5DF000093E
:1045480042E1040E406E0AD02EEC60F041C0D9FF63
:1045580042C0DAFFDF6E414A422A4006405001E17C
:1045680035D6F2D7146A156A166A176A8D0EADEC3D
:104578005DF0000928E12EEC60F041C00BF042C06C
:104588000CF00E6A400E0D6E7AEC5AF0BAD7040E93
:104598003F6E19D01A501D6E1E6A1E50F8E11D504C
:1045A80001E10FD6010A01E113D6020A01E1C8D6DA
:1045B800090A8EE0010A93E0070AA7E0010AB8E0B9
:1045C800030AD0E0E4D73FEC60F03F50120078C017
:1045D800D9FF79C0DAFFDECF8FF0DDCF90F07A51C6
:1045E8007B117C117D1128E120EE0BF08F51D9262B
:1045F8009051DA22DECF87F0DECF88F0DECF89F067
:10460800DECF8AF08751881189118A110FE020EED8
:1046180013F08F51D9269051DA22DE50875DDE5093
:104628008859DE508959DE508A5952E3010E876F46
:10463800886B896B8A6B4CD078C042F079C043F0A4
:104648007AC044F07BC045F07CC046F07DC047F09E
:10465800AFEC2CF042C091F043C092F044C093F00C
:1046680045C094F0000194519311921109E1020E92
:10467800915D06E2010E786F796B7A6B7B6B000CAB
:1046880091290FE192290DE193290BE1942909E180
:1046980091C078F092C079F093C07AF094C07BF022
:1046A800120020EE13F08F51D9269051DA22DE50F5
:1046B800915DDE509259DE509359DE509459E8E3EB
:1046C8007AC087F07BC088F07CC089F07DC08AF012
:1046D80020EE0FF08F51D9269051DA22DE50DE10ED
:1046E800DE10DE1005E1786B796B7A6B7B6B12005C
:1046F8008B6B8C6B8D6B8E6B7A51871909E17B51B3
:10470800881906E17C5189197DE17D518A19D8A45F
:1047180079D087298B6F000E88218C6F000E892134
:104728008D6F000E8A218E6F20EE13F08F51D926DF
:104738009051DA22DE508B5DDE508C59DE508D5957
:10474800DE508E5905E3020E8B6F8C6B8D6B8E6B72
:1047580078C042F079C043F08BC044F08CC045F07B
:104768008DC046F08EC047F0AFEC2CF042C091F0FF
:1047780043C092F044C093F045C094F00001910505
:1047880092119311941184E0912907E1922905E18E
:10479800932903E1942901E17BD791519211931157
:1047A800941130E020EE0BF08F51D9269051DA2287
:1047B800DECF91F0DECF92F0DECF93F0DECF94F033
:1047C80094519311921103E1020E915D17E320EECB
:1047D80013F08F51D9269051DA22DE50915DDE50C8
:1047E8009259DE509359DE50945908E291C087F0EF
:1047F80092C088F093C089F094C08AF08B6B8C6B60
:104808008D6B8E6B8B518C118D118E1162E187C06F
:104818008BF088C08CF089C08DF08AC08EF08B2B0D
:10482800000E8C238D238E2320EE13F08F51D92672
:104838009051DA22DE508B5DDE508C59DE508D5956
:10484800DE508E590DE3020E8B6F8C6B8D6B8E6B69
:104858008A518911881104E1020E875D01E243D76C
:1048680078C042F079C043F08BC044F08CC045F06A
:104878008DC046F08EC047F0AFEC2CF042C091F0EE
:1048880043C092F044C093F045C094F000019151A8
:104898009211931194111DE09105921193119411A5
:1048A80001E1F6D6912907E1922905E1932903E16F
:1048B800942901E1EDD687518B19B1E188518C1902
:1048C800AEE189518D19ABE18A518E1901E10BD7FF
:1048D800A6D78FC060F090C061F08BC062F08CC02A
:1048E80063F08DC064F08EC065F0666967696869B9
:1048F8006969BBEC1EF00001866F86511DE17A5193
:104908007B117C117D1118E08FC060F090C061F0C0
:104918007AC062F07BC063F07CC064F07DC065F053
:104928008BC066F08CC067F08DC068F08EC069F0EF
:10493800BBEC1EF00001866F865143E120EE0BF0C0
:104948008F51D9269051DA228BC0DEFF8CC0DEFF52
:104958008DC0DEFF8EC0DEFF20EE0FF08F51D9260E
:104968009051DA2210EE13F08F51E1269051E22295
:10497800FE0EE624826FFF0EE620836FFF0EE62010
:10498800846FFF0EE620856FDE50825DDE5083590E
:10499800DE508459DE5085590BE320EE0FF08F511D
:1049A800D9269051DA22DE06000EDE5ADE5ADE5A89
:1049B80020EE04F08F51D9269051DA22000EDB80C8
:1049C8000DD0860507E0010E8B6F000E8C6B8D6B8A
:1049D8008E6B04D08B698C698D698E698BC078F079
:1049E8008CC079F08DC07AF08EC07BF0120018C0B0
:1049F800F6FF19C0F7FF0800F5CF9BF0184A192AEF
:104A080000019B5101E11200250E9B1904E09B5106
:104A1800FFEC5FF0ECD7946B956B966B976B18C0B7
:104A2800F6FF19C0F7FF0800F5CF9BF0184A192ABE
:104A3800300E9B190DE1976B010E966F18C0F6FFAB
:104A480019C0F7FF0800F5CF9BF0184A192A06D0BD
:104A58002D0E9B1903E1976B020EEFD72A0E9B19B7
:104A680043E11A50D96EDA6A020EDF26DF5CD96E8E
:104A7800DA6ADECF8CF0DECF8DF08DAF0BD08C51A3
:104A880000088C6F8D51D8A0E82A00088D6F976BAD
:104A9800020E966F8CC094F08DC095F018C0F6FF8A
:104AA80019C0F7FF0800F5CF9BF0184A192A22D041
:104AB8000A0E9403F3CF1BF0F4CF1CF09503F350C8
:104AC8001C269B511B26000E1C22D00E1B24946F03
:104AD800FF0E1C20956F18C0F6FF19C0F7FF0800DD
:104AE800F5CF9BF0184A192A2F0E9B6503D0390E73
:104AF8009B65DED76C0E9B1903E04C0E9B190AE1EF
:104B0800968518C0F6FF19C0F7FF0800F5CF9BF08F
:104B1800184A192A9B5101E112009BC09AF0600EB5
:104B28009A6575D0200E9A5F72D01A50D96EDA6ADB
:104B3800020EDF26DF5CD96EDA6ADECF84F0DECFC4
:104B480085F0926B936B03D00001924B932B92519B
:104B580084251B6E935185211C6E1BC0F6FF1CC05B
:104B6800F7FF000EF86E0E0EF76403D00800F5503C
:104B780005D0F6CFE9FFF7CFEAFFEF50000904E0D0
:104B8800E3D7200EFFEC5FF0000196B30BD09251F3
:104B98001B6E93511C6E924B932B94511B5C955139
:104BA8001C58EFE384C00CF085C00DF0FEEC5AF001
:104BB80003D0200EFFEC5FF0000192511B6E935161
:104BC8001C6E924B932B94511B5C95511C5801E31E
:104BD8000ED7EFD71A50D96EDA6ADF50DF2ADF2AEC
:104BE800D96EDA6ADF50FFEC5FF001D7876B020EEF
:104BF80008D0876B080E05D0876B0A0E02D0876B2A
:104C0800100E866F1AD09B51FFEC5FF0F0D69A51C8
:104C18001B6E1C6A1C50F7E11B50420AE7E0010AB0
:104C2800D9E0070AE9E00B0AE4E01C0A01E17DD7B4
:104C3800060AE2E00D0AE3E0E6D796A511D01A507D
:104C4800D96EDA6A040EDF26DF5CD96EDA6ADECF47
:104C58008EF0DECF8FF0DECF90F0DECF91F027D050
:104C6800440E9A1913E01A50D96EDA6ADF50DF2A17
:104C7800DF2AD96EDA6ADECF1BF0DDCF1CF01BC04D
:104C88008EF01CC08FF0906B916B11D01A50D96EBA
:104C9800DA6ADF50DF2ADF2AD96EDA6ADECF8EF0D1
:104CA800DDCF8FF0000E8FBFFF0E906F916F440E17
:104CB8009A190CE191AF0AD08E6D8F1FD8B08F2B47
:104CC800901FD8B0902B000E91579689986B996BCE
:104CD8008EC088F08FC089F090C08AF091C08BF0A8
:104CE80088C00BF089C00CF08AC00DF08BC00EF0A4
:104CF80086C00FF087C010F0116A126AEAEC59F00A
:104D08000B5000019A6F88C00BF089C00CF08AC064
:104D18000DF08BC00EF086C00FF087C010F0116A3E
:104D2800126A87EC57F00BC088F00CC089F00DC0F0
:104D38008AF00EC08BF0090E00019A650BD0780E30
:104D48009B1903E0816B070E02D0816B270E806FE1
:104D580080519A279851600FD96EDA6A9A51300FAC
:104D6800DF6E984B992B885189118A118B1105E0B8
:104D7800995103E1200E985DB3E396A908D09851A4
:104D8800600FD96EDA6A2D0EDF6E984B992B98C09A
:104D980092F099C093F096B103D0836B200E02D0A5
:104DA800836B300E826F82C09AF003D09A51FFEC69
:104DB8005FF0000196B30BD092511B6E93511C6E9D
:104DC800924B932B94511B5C95511C58EFE3980719
:104DD800D8A099079851600FD96EDA6ADF50FFECB6
:104DE8005FF000019851991104E0F1D7200EFFEC13
:104DF8005FF0000192511B6E93511C6E924B932BE6
:104E080094511B5C95511C5801E3F1D5EFD75050D4
:104E18000C0D620EF324D96E020EF420DA6EDF2A2E
:104E280050500C0D620EF324D96E020EF420DA6E87
:104E3800DF500001C26FC36BC469C56950500C0DC7
:104E48006A0EF324D96E020EF420DA6EDF50C66FB4
:104E5800C76BC451C627C551C723C251C65DC751C8
:104E6800800AC86FC351800AC8594BE250500C0DD4
:104E7800620EF324D96E020EF420DA6EDF6A505007
:104E88000C0D610EF324D96E020EF420DA6EDF2ABF
:104E980050500C0D610EF324D96E020EF420DA6E18
:104EA800DF50C26FC36BC469C56950500C0D690EE1
:104EB800F324D96E020EF420DA6EDF50C66FC76B8A
:104EC800C451C627C551C723C251C65DC751800A00
:104ED800C86FC351800AC85914E250500C0D610EB6
:104EE800F324D96E020EF420DA6EDF6A50500C0DEE
:104EF8005F0EF324D96E020EF420DA6EDE2A000E5D
:104F0800DD2250500C0D620EF324D96E020EF420EF
:104F1800DA6EDF50C26FC2C0C3F0C46BC56BC66B1C
:104F2800C5C0C6F0C4C0C5F0C3C0C4F0C36B505000
:104F38000C0D6A0EF324D96E020EF420DA6EDF50DF
:104F4800C76FC7C0C8F0C96BCA6BCB6B50500C0D8C
:104F5800610EF324D96E020EF420DA6EDF50CC6FA6
:104F6800CCC0CDF0CE6BCF6BD06BCFC0D0F0CEC065
:104F7800CFF0CDC0CEF0CD6BCD51C803F3CFD1F07B
:104F8800F4CFD2F0D36BD46BC903F350D227F450CB
:104F9800D323000ED423CE51C803F350D227F450A4
:104FA800D323000ED423CD51CA03F350D327F45092
:104FB800D423CE51C903F350D327F450D423CF516F
:104FC800C803F350D327F450D423CB51CD03F35067
:104FD800D427CE51CA03F350D427CF51C903F35075
:104FE800D427D051C803F350D42750500C0D690E64
:104FF800F324D96E020EF420DA6EDF50D56FD5C0D7
:10500800D6F0D76BD86BD96B50500C0D6A0EF324C1
:10501800D96E020EF420DA6EDF50DA6FDAC0DBF0F8
:10502800DC6BDD6BDE6B50500C0D5F0EF324D96E1C
:10503800020EF420DA6EDECFDFF0DDCFE0F0DFC065
:10504800E1F0E0C0E2F0000EE2BFFF0EE36FE46FB4
:10505800E151DB03F3CFE5F0F4CFE6F0E76BE86B63
:10506800DC03F350E627F450E723000EE823E2516F
:10507800DB03F350E627F450E723000EE823E15161
:10508800DD03F350E727F450E823E251DC03F35043
:10509800E727F450E823E351DB03F350E727F45004
:1050A800E823DE51E103F350E827E251DD03F35032
:1050B800E827E351DC03F350E827E451DB03F3501E
:1050C800E827E7C0E8F0E6C0E7F0E5C0E6F0E56B02
:1050D800E551D603F3CFE9F0F4CFEAF0EB6BEC6BD4
:1050E800D703F350EA27F450EB23000EEC23E651E4
:1050F800D603F350EA27F450EB23000EEC23E551D6
:10510800D803F350EB27F450EC23E651D703F350C0
:10511800EB27F450EC23E751D603F350EB27F45078
:10512800EC23D951E503F350EC27E651D803F350AB
:10513800EC27E751D703F350EC27E851D603F35097
:10514800EC27D151E925ED6FD251EA21EE6FD35109
:10515800EB21EF6FD451EC21F06FC351ED25F16FC6
:10516800C451EE21F26FC551EF21F36FC651F02102
:10517800F46F50500C0D630EF324D96E020EF42018
:10518800DA6EF1C0DEFFF2C0DEFFF3C0DEFFF4C06E
:10519800DEFF5050220D000EF324956F030EF4200D
:1051A800966F50500C0D630EF324D96E020EF42046
:1051B800DA6EDECF97F0DECF98F0DECF99F0DECF53
:1051C8009AF029EC12F0F56FF55119E0C60E9C6FB4
:1051D800FB0E9D6F50500C0D630EF324D96E020E1A
:1051E800F420DA6EDECF9EF0DECF9FF0DECFA0F0A7
:1051F800DECFA1F0F5C0A2F0A36B0AEC60F00101CC
:105208008F6B1200000E0001746F030E756F350E60
:10521800766F0B0E776F020E796F786BF30E7A6FDD
:105228007B6BBFEC17F001019A6FCF0E00019C6FEA
:10523800FD0E9D6FF3C09EF0F4C09FF00AEC60F085
:10524800F56BF66BF16BF26BF76BF86BF751D30FED
:10525800D96EDA6ADF6AF751E20FD96EDA6A000EA0
:10526800DF6EF74BF82BF8BFF1D7F85103E10F0EBB
:10527800F75DECE3F96BFA6B30D1350EF925D96E91
:105288000B0EFA21DA6E0D0EDE1801E0EBD0960E49
:105298000B6EFF0E0C6ED30E0D6E87EC54F00B5098
:1052A8000C1007E1E20E126EA5EC4CF01250010151
:1052B800FD6F900E0B6EFF0E0C6ED30E0D6E87EC0D
:1052C80054F00B500C1007E1E20E126EA5EC4CF0F6
:1052D800125001019B6F6F0E0B6EFF0E0C6ED30EFA
:1052E8000D6E87EC54F00B500C1007E1E20E126EB5
:1052F800A5EC4CF012500101966FD40E0B6EFF0E08
:105308000C6ED30E0D6E87EC54F00B500C1007E1A9
:10531800E20E126EA5EC4CF012500101946FD80EFB
:105328000B6EFF0E0C6ED30E0D6E87EC54F00B5007
:105338000C1007E1E20E126EA5EC4CF012500101C0
:10534800FE6F0001FB6BFC6BC40E796F7A6B760EF7
:105358007B6FFF0E7C6FFBC07DF0FCC07EF057ECCE
:105368005DF0C40E0B6E0C6AD30E0D6E87EC54F014
:105378000B500C1018E10F0E0001FB03F3CFC2F025
:10538800F4CFC3F0FC03F350C327350EC2250B6ED0
:105398000D0EC3210C6EE20E0D6E0E6A106A0F0E12
:1053A8000F6EA9EC5AF00001FB4BFC2BFCBFCCD7CD
:1053B800FC5103E1100EFB5DC7E3FC6B010EFB6FB4
:1053C800C40E796F7A6B7D0E7B6FFF0E7C6FFBC00E
:1053D8007DF0FCC07EF057EC5DF0C40E0B6E0C6ADD
:1053E800D30E0D6E87EC54F00B500C1018E10F0E15
:1053F8000001FB03F3CFC2F0F4CFC3F0FC03F3507A
:10540800C327250EC2250B6E0E0EC3210C6EE20EAD
:105418000D6E0E6A106A0F0E0F6EA9EC5AF000019D
:10542800FB4BFC2BFCBFCCD7FC5103E1040EFB5D0E
:10543800C7E3F76BF86BF751D30FD96EDA6ADF6AF7
:10544800F751E20FD96EDA6A000EDF6EF74BF82BD0
:10545800F8BFF1D7F85103E10F0EF75DECE3F16BFC
:10546800F26B15D0350EF925D96E0B0EFA21DA6ECE
:105478000A0EDE1830E0350EF925D96E0B0EFA212A
:10548800DA6E200EDE1806E1F26B010EF16FF56B95
:10549800F66B21D0F151F21109E0350EF925D96EDC
:1054A8000B0EFA21DA6EF551E20F08D0350EF92508
:1054B800D96E0B0EFA21DA6EF551D30FE16EE26A5E
:1054C800DFCFE7FFF6BF05D0F65105E10F0EF55D1A
:1054D80002E2F54BF62BF94BFA2BF351F95DF45137
:1054E800FA5901E2CAD6BF0E9C6FFD0E9D6F96C198
:1054F8009EF09F6B0AEC60F02A0E9C6FFE0E9D6F6B
:10550800FDC19EF09F6B0AEC60F01B0E9C6FFE0EB7
:105518009D6F9BC19EF09F6B0AEC60F0FB6BFC6B70
:105528003C0E9C6FFD0E9D6FFBC09EF0FCC09FF073
:105538000F0EFB03F3CFC2F0F4CFC3F0FC03F3501C
:10554800C327350EC225A06F0D0EC321A16F0AEC2B
:1055580060F0FB4BFC2BFCBFE3D7FC5103E1100EC2
:10556800FB5DDEE3FA6B010EF96F4D0E9C6FFD0ECD
:105578009D6FF9C09EF0FAC09FF00F0EF903F3CFAC
:10558800C2F0F4CFC3F0FA03F350C327250EC225A7
:10559800A06F0E0EC321A16F0AEC60F0F94BFA2B35
:1055A800FABFE3D7FA5103E1040EF95DDEE34A0ED0
:1055B8009C6FFA0E9D6F0AEF60F0838E8380E3EC98
:1055C80039F00101AA6FAA5117E050501C0D1B0EAB
:1055D800F324D96E010EF420DA6E50501C0D1B0E08
:1055E800F324E16E010EF420E26EE7500409DF6E49
:1055F80094EC5EF0AA511200945154E0705171116C
:10560800721173114FE050504DE150501C0D070EB0
:10561800F324D96E010EF420DA6E70C1F0F071C176
:10562800F1F072C1F2F00001EF6B000EEF25F36F9D
:10563800010EF021F46F000EF121F56F000EF2213A
:10564800F66FF76BF86BF96BFA6BDE50F3192AE11A
:10565800DE50F41927E1DE50F51924E1DE50F61981
:1056680021E1DE50F7191EE1DE50F8191BE1DE508A
:10567800F91918E1DE50FA1915E1350E286E0B0EEE
:10568800296E01019451A3EC4DF00101FC93010E28
:105698001F6E1E6AB8EC35F00101FC934E6A8390C8
:1056A8004E50120050501C0D170EF324D96E010EE7
:1056B800F420DA6EDECFE7F0DECFE8F0DECFE9F0F7
:1056C800DECFEAF0E8C0E7F0E9C0E8F0EAC0E9F0C8
:1056D8000001EA6BE7C09EF1E8C09FF1E9C0A0F1C4
:1056E800EAC0A1F150501C0D170EF324D96E010E1B
:1056F800F420DA6EDECFE7F0DDCFE8F0E751010104
:10570800A46FA56BFC93A66BA76BA86BA96BA26B88
:10571800A36B97D0A2C1E7F0A3C1E8F0000EE8BFE1
:10572800FF0EE96FEA6FFF0E01019E250001EB6F86
:10573800FF0E01019F210001EC6FFF0E0101A02166
:105748000001ED6FFF0E0101A1210001EE6FE7518D
:10575800EB190EE1E851EC190BE1E951ED1908E1FB
:10576800EA51EE1905E10101A451A51101E1FC83FB
:105778005050220D000EF3240001746F030EF42024
:10578800756F350E766F0B0E776F010E796F786B2C
:10579800AB0E7A6F010E7B6FBFEC17F00101AD6F96
:1057A800AD5101E012D7AB51AC1101E10ED7ABC13D
:1057B8001EF0ACC11FF0B8EC35F00101AB51A627C3
:1057C800AC51A723000EA823A92350501C0D070E87
:1057D800F324D96E010EF420DA6E000EDE240001E7
:1057E800E76F010EDE20E86F000EDE20E96F000E85
:1057F800DE20EA6F000EDE20EB6F000EDE20EC6F7D
:10580800000EDE20ED6F000EDE20EE6F50501C0DF6
:10581800070EF324D96E010EF420DA6EE7C0DEFF1E
:10582800E8C0DEFFE9C0DEFFEAC0DEFFEBC0DEFF56
:10583800ECC0DEFFEDC0DEFFEEC0DEFF0101A24BD3
:10584800A32BA2C1E7F0A3C1E8F0000E0001E8BF56
:10585800FF0EE96FEA6F01019E510001E75D01014A
:105868009F510001E8590101A0510001E9590101C6
:10587800A1510001EA5901E24DD70101A451A51136
:1058880064E05050220D000EF3240001746F030EE3
:10589800F420756F350E766F0B0E776FA4C178F014
:1058A800A5C179F0AB0E7A6F010E7B6FBFEC17F0D4
:1058B8000101AD6FAD5101E088D6FC83A4C11EF093
:1058C800A5C11FF0B8EC35F00101AB51A627AC51CA
:1058D800A723000EA823A92350501C0D070EF3245C
:1058E800D96E010EF420DA6E000EDE240001E76F97
:1058F800010EDE20E86F000EDE20E96F000EDE20CC
:10590800EA6F000EDE20EB6F000EDE20EC6F000E5B
:10591800DE20ED6F000EDE20EE6F50501C0D070EDE
:10592800F324D96E010EF420DA6EE7C0DEFFE8C07A
:10593800DEFFE9C0DEFFEAC0DEFFEBC0DEFFECC041
:10594800DEFFEDC0DEFFEEC0DEFF0101FC934E6A14
:105958008390839EA5D642C0D9FF43C0DAFFDECF2D
:1059680072F0DDCF73F047504610451003E1020E88
:10597800445C10E3000120EE13F07251D9267351F4
:10598800DA22DE50445CDE504558DE504658DE5080
:10599800475808E3010E00016C6F000E6D6B6E6BCB
:1059A8006F6B8FD16C696D696E696F6976D144C010
:1059B80070F045C071F0D8907131616F7031606FCF
:1059C800605170276151712372C037F073C038F08D
:1059D80020EE1FF07251D9267351DA22DECF60F023
:1059E800DECF61F0DECF62F0DECF63F070C064F02E
:1059F80071C065F0090E666FD89065336433662F01
:105A0800FBD764516025396E655161213A6E000EED
:105A180062213B6E000E63213C6E39EC54F00009A4
:105A280001E04FD100016069010E616F70C062F042
:105A380071C063F0605162176151631772C064F0FE
:105A480073C065F062516427635165232F0E642586
:105A5800D96E000E6521DA6EDF506A6F6B6B704B82
:105A6800712B72C037F073C038F020EE1FF07251FE
:105A7800D9267351DA22DECF60F0DECF61F0DECFB7
:105A880062F0DECF63F070C064F071C065F0090E9B
:105A9800666FD89065336433662FFBD764516025F1
:105AA800396E655161213A6E000E62213B6E000E1F
:105AB80063213C6E39EC54F0000901E002D1000189
:105AC8006069010E616F70C062F071C063F060516F
:105AD80062176151631772C064F073C065F0625158
:105AE8006427635165232F0E6425D96E000E652146
:105AF800DA6EDF50676F666B66516A1367516B1316
:105B080044B006D06A51686F0F0E6B15696F0FD0DD
:105B18006AC060F06BC061F0040E626FD8906133A8
:105B28006033622FFBD760C068F061C069F068C05D
:105B38006CF069C06DF04ED072C037F073C038F0A9
:105B480020EE1FF07251D9267351DA22DECF60F0B1
:105B5800DECF61F0DECF62F0DECF63F04550646FD8
:105B68004650656F4750666F676B60516425396EA4
:105B7800615165213A6E625166213B6E635167211E
:105B88003C6E39EC54F0000901E09BD000016069DB
:105B9800010E616F44C062F045C063F0D89062376F
:105BA8006337605162176151631772C064F073C044
:105BB80065F062516427635165232F0E64250B6ECF
:105BC800000E65210C6E1AEC5EF00BC06CF00CC078
:105BD8006DF000016E6B6F6B74D072C037F073C0DC
:105BE80038F020EE1FF07251D9267351DA22DECF39
:105BF80060F0DECF61F0DECF62F0DECF63F044C04C
:105C080064F045C065F046C066F047C067F0080E0E
:105C180005D0D8906733663365336433E82EF9D7F7
:105C280060516425396E615165213A6E6251662171
:105C38003B6E635167213C6E39EC54F0000941E139
:105C480000016069010E616F44C062F045C063F0F5
:105C5800D89062376337D8906237633760516217DC
:105C68006151631772C064F073C065F062516427B4
:105C7800635165232F0E64250B6E000E65210C6E93
:105C880044EC53F00B5000016C6F0C506D6F0D50CD
:105C98006E6F0F0E0E146F6F14D072C0D9FF73C0E1
:105CA800DAFFDF50606F616B615101E073D66051BC
:105CB800010A01E17CD6030A01E13ED7010A8DE021
:105CC80069D66CC042F06DC043F06EC044F06FC03E
:105CD80045F0120095C0D9FF96C0DAFFDECFADF0CF
:105CE800DDCFAEF020EE0EF09551D9269651DA228E
:105CF800DECF99F0DECF9AF0DECF9BF0DECF9CF0BE
:105D0800200E9925A96F000E9A21AA6F000E9B21DB
:105D1800AB6F000E9C21AC6FAC5103E1200EAB5D64
:105D28000AE320EE16F09551D9269651DA22DE6A5A
:105D3800DE6ADE6ADD6A20EE16F09551D9269651A4
:105D4800DA22DE50DE10DE10DE1001E1040CA9516B
:105D5800996F010EAA159A6F9B6B9C6B99119B11F9
:105D68009C1101E029D120EE16F09551D9269651C3
:105D7800DA22DE2A000EDE22DE22DE2220EE12F0F9
:105D88009551D9269651DA22DE50DE10DE10DE104B
:105D98002CE120EE07F0AD51D926AE51DA22DECF44
:105DA80099F0DDCF9AF099519B6F9A519C6F9D6B3A
:105DB8009E6BA9C09FF0AAC0A0F0ABC0A1F0ACC078
:105DC800A2F0060E05D0D890A233A133A0339F339A
:105DD800E82EF9D79B519F5D9C51A0599D51A1591F
:105DE8009E51A25901E2E8D06ED099699A6920EED5
:105DF80009F0AD51D926AE51DA22DECF9BF0DDCFC6
:105E08009CF099519B279A519C23A9C09DF0AAC048
:105E18009EF0ABC09FF0ACC0A0F00A0E05D0D890A1
:105E2800A0339F339E339D33E82EF9D79B519D15A0
:105E3800A16F9C519E15A26FA36BA46BA111A31116
:105E4800A41101E0B9D095C042F096C043F020EE0D
:105E580012F09551D9269651DA22DECF44F0DECFE2
:105E680045F0DECF46F0DECF47F0AFEC2CF042C075
:105E7800AFF043C0B0F044C0B1F045C0B2F000018B
:105E8800B251B111B01104E1020EAF5D01E2020C92
:105E9800AF2907E1B02905E1B12903E1B22901E100
:105EA800010C20EE13F0AD51D926AE51DA22DE50A6
:105EB800AF5DDE50B059DE50B159DE50B25950E3F3
:105EC800975198110BE120EE16F09551D92696516D
:105ED800DA22DE6ADE6ADE6ADD6A040C95C078F0D2
:105EE80096C079F020EE12F09551D9269651DA2213
:105EF800DECF7AF0DECF7BF0DECF7CF0DECF7DF038
:105F0800EBEC22F078C0AFF079C0B0F07AC0B1F015
:105F18007BC0B2F0AF51B011B111B21101E1070C61
:105F2800AF05B011B111B21101E1020CAF2907E1BF
:105F3800B02905E1B12903E1B22901E1010CADC0A5
:105F480037F0AEC038F0AFC039F0B0C03AF0B1C0E9
:105F58003BF0B2C03CF023EC4CF0000901E0010C2E
:105F6800000120EE12F09551D9269651DA22AFC0E1
:105F7800DEFFB0C0DEFFB1C0DEFFB2C0DEFFADC0E5
:105F88000BF0AEC00CF0AFC00DF0B0C00EF0B1C059
:105F98000FF0B2C010F091EC4AF0000120EE16F0BC
:105FA8009551D9269651DA220BC0DEFF0CC0DEFFD0
:105FB8000DC0DEFF0EC0DEFF20EE0EF09551D92693
:105FC8009651DA22A9C0DEFFAAC0DEFFABC0DEFF11
:105FD800ACC0DEFF9969010E9A6FA9C09BF0AAC0F8
:105FE8009CF099519B179A519C17ADC09DF0AEC07B
:105FF8009EF09B519D279C519E232F0E9D27000E9E
:106008009E2320EE1AF09551D9269651DA229DC08A
:10601800DEFF9EC0DDFF000C506A506A030E50641C
:1060280001D090D1505003E11E6A1F6A03D01F6A45
:10603800010E1E6E50501C0D1B0EF324D96E010E5E
:10604800F420DA6EDF6A50501C0D000EF324D96E6E
:10605800010EF420DA6EDF6A50501C0D070EF3248F
:10606800D96E010EF420DA6E070EDE6AE806FDE24C
:106078000D0E1E02F3CF9EF1F4CF9FF11F02F350D5
:1060880001019F27310E9E25D96E020E9F21DA6EDF
:10609800DF50A06FA0C1A1F1A26BA36BA46BA3C139
:1060A800A4F1A2C1A3F1A1C1A2F1A16BA1C1A5F163
:1060B800A2C1A6F1A3C1A7F1A4C1A8F1A96BA8BF69
:1060C800A969A9C1AAF1A9C1ABF1A9C1ACF10D0E89
:1060D8001E02F3CFADF1F4CFAEF11F02F350AE279D
:1060E800300EAD25D96E020EAE21DA6EDF50AF6FDD
:1060F800AFC1B0F1B16BB26BB36BB1C1B3F1B0C1A9
:10610800B2F1B16BB06BB0C1B4F1B1C1B5F1B2C10C
:10611800B6F1B3C1B7F1B86BB7BFB869B8C1B9F1D7
:10612800B8C1BAF1B8C1BBF10D0E1E02F3CFBCF174
:10613800F4CFBDF11F02F350BD272F0EBC25D96E39
:10614800020EBD21DA6EDF50BE6FBEC1BFF1C06B5B
:10615800C16BC26BBFC1C2F1C16BC06BBF6BBFC1AA
:10616800C3F1C0C1C4F1C1C1C5F1C2C1C6F1C76B99
:10617800C6BFC769C7C1C8F1C7C1C9F1C7C1CAF19C
:106188000D0E1E02F3CFCBF1F4CFCCF11F02F3506A
:10619800CC272E0ECB25D96E020ECC21DA6EDF501D
:1061A800CD6FCDC1CEF1CF6BD06BD16BD26BD36B32
:1061B800D46BD56B200ED890CE37CF37D037D137A8
:1061C800D237D337D437D537E82EF5D7C351CE25B4
:1061D800D66FC451CF21D76FC551D021D86FC651C2
:1061E800D121D96FC751D221DA6FC851D321DB6FC2
:1061F800C951D421DC6FCA51D521DD6FB451D625E0
:10620800DE6FB551D721DF6FB651D821E06FB75196
:10621800D921E16FB851DA21E26FB951DB21E36F7F
:10622800BA51DC21E46FBB51DD21E56FA551DE25B4
:10623800E66FA651DF21E76FA751E021E86FA8516B
:10624800E121E96FA951E221EA6FAA51E321EB6F3D
:10625800AB51E421EC6FAC51E521ED6F50501C0DB2
:106268000F0EF324D96E010EF420DA6EE6C1DEFFBC
:10627800E7C1DEFFE8C1DEFFE9C1DEFFEAC1DEFFFC
:10628800EBC1DEFFECC1DEFFEDC1DEFF020E000157
:106298009C6FFB0E9D6F50C09EF09F6B50501C0D65
:1062A8000F0EF324D96E010EF420DA6EDECF9EF1C4
:1062B800DECF9FF1DECFA0F1DECFA1F1DECFA2F1DC
:1062C800DECFA3F1DECFA4F1DECFA5F19EC1A0F011
:1062D8009FC1A1F0A0C1A2F0A1C1A3F0A2C1A4F0E6
:1062E800A3C1A5F0A4C1A6F0A5C1A7F050501C0DEC
:1062F8000F0EF324D96E010EF420DA6EDECFA6F16C
:10630800DECFA7F1DECFA8F1DECFA9F1DECFAAF16B
:10631800DECFABF1DECFACF1DECFADF1A6C1A8F098
:10632800A7C1A9F0A8C1AAF0A9C1ABF0AAC1ACF055
:10633800ABC1ADF0ACC1AEF0ADC1AFF00AEC60F0EE
:10634800502A6CD60101936B4F6A926B826B836BF8
:10635800020E4E6E916F8390020C74C0D9FF75C007
:10636800DAFFDECF90F0DDCF91F0795109E1200E10
:10637800785DD8B0020C76C07AF01F0E7A1701E06B
:10638800020C20EE0EF07451D9267551DA2276C02F
:10639800DEFF77C0DEFF78C0DEFF79C0DEFF20EECB
:1063A80006F07451D9267551DA22DECF8CF0DECF93
:1063B8008DF0DECF8EF0DECF8FF08C518D118E11E7
:1063C8008F1115E190C0D9FF91C0DAFF020EDF648A
:1063D8000ED020EE23F09051D9269151DA22DECF4B
:1063E8008CF0DECF8DF0DECF8EF0DECF8FF08C51CB
:1063F8008D118E118F1140E120EE07F09051D926B2
:106408009151DA22DECF7AF0DDCF7BF07A517C6FC2
:106418007B517D6F7E6B7F6B76C080F077C081F09B
:1064280078C082F079C083F0060E05D0D890833307
:10643800823381338033E82EF9D77C51805D7D51DA
:1064480081597E5182597F51835901E3020C20EE14
:1064580023F09051D9269151DA2210EE16F074519A
:10646800E1267551E222DECFE6FFDECFE6FFDECF82
:10647800E6FFDECFE6FF87D020EE09F09051D9265F
:106488009151DA22DECF7AF0DDCF7BF07A517C6F42
:106498007B517D6F7E6B7F6B090ED8907C377D3783
:1064A8007E377F37E82EF9D77CC088F07DC089F029
:1064B8007EC08AF07FC08BF040D074C042F075C0B7
:1064C80043F08CC044F08DC045F08EC046F08FC0BC
:1064D80047F0AFEC2CF042C08CF043C08DF044C0C4
:1064E8008EF045C08FF000018C2907E18D2905E168
:1064F8008E2903E18F2901E1010C8F518E118D1135
:1065080004E1020E8C5DD8A0020C20EE13F090512D
:10651800D9269151DA22DE508C5DDE508D59DE503D
:106528008E59DE508F5901E3020C8851765F8951EC
:10653800775B8A51785B8B51795B8851765D89519D
:1065480077598A5178598B517959B7E290C00BF035
:1065580091C00CF08CC00DF08DC00EF08EC00FF005
:106568008FC010F091EC4AF0000120EE16F0745143
:10657800D9267551DA220BC0DEFF0CC0DEFF0DC034
:10658800DEFF0EC0DEFF20EE12F07451D9267551E1
:10659800DA228CC0DEFF8DC0DEFF8EC0DEFF8FC02A
:1065A800DEFF20EE16F07451D9267551DA22DE503E
:1065B800DE10DE10DE1001E1020C76C07AF077C042
:1065C8007BF078C07CF079C07DF00A0E05D0D890B9
:1065D8007D337C337B337A33E82EF9D720EE16F0FF
:1065E8007451D9267551DA227A51DE267B51DE2282
:1065F8007C51DE227D51DE227A69010E7B6F76C0E6
:106608007CF077C07DF07A517C177B517D1790C064
:106618007EF091C07FF07C517E277D517F232F0E25
:106628007E27000E7F2320EE1AF07451D92675516B
:10663800DA227EC0DEFF7FC0DDFF000C000E000105
:10664800DB6F250EDA6F000ED96F050ED86F0101CA
:10665800FD5105E1000E0001DB6F280EDA6F010124
:1066680096510DE1FB6B350E0001796F0D0E7A6FB7
:10667800CF0E7B6FFE0E7C6F57EC5DF00DD0420E97
:1066880000019C6FFB0E9D6F96C19EF09F6BFBC136
:10669800A0F0A16B0AEC60F0480E9C6FFE0E9D6F97
:1066A8000101FB510F0D350EF32400019E6F0D0EF5
:1066B800F4209F6F0AEC60F0050E0001D76F0F0EF3
:1066C800D66FF10EE82EFED7D62FFCD7D72FFAD7E4
:1066D800D4D02B0E0C6EFD0E0D6EFEEC5AF0000E93
:1066E8000001C96F030ECA6FC20ECB6FFE0ECC6FCE
:1066F800010ECD6FF7EC14F001019A6F9A517AEC04
:106708005BF001019A510AE1E3EC37F0000E486EA4
:10671800030E496E3AEC5DF001019A6F9A517AECDA
:106728005BF0DB6B280EDA6FA4D00101FB510F0D73
:10673800350EF324D96E0D0EF420DA6E200EDE1815
:1067480006E1FB2B0F0EFB6594D0FB6B92D03C0E41
:1067580000019C6FFC0E9D6F0101FB510F0D350E62
:10676800F32400019E6F0D0EF4209F6F0AEC60F079
:10677800000EC96F030ECA6F0101FB510F0D350ED4
:10678800F3240001CB6F0D0EF420CC6F030ECD6FF8
:10679800F7EC14F001019A6F9A517AEC5BF0010161
:1067A8009A5104E10001DB6B3C0EDA6F040E010123
:1067B8009A1904E10001DB6B320EDA6F050E000155
:1067C800D76F0F0ED66FF10EE82EFED7D62FFCD757
:1067D800D72FFAD74ED0F70E9C6FFC0E9D6F010194
:1067E800FB510F0D350EF32400019E6F0D0EF420A2
:1067F8009F6F0AEC60F0000EC96F030ECA6F0101AB
:10680800FB510F0D350EF3240001CB6F0D0EF42054
:10681800CC6F070ECD6FF7EC14F001019A6F9A5107
:10682800CDE10001DB6B3C0EC8D7D20E9C6FFC0E8D
:106838009D6F0101FB510F0D350EF32400019E6F72
:106848000D0EF4209F6F0AEC60F013D0DAC0D6F07A
:10685800DBC0D7F0D7510DE1D651250A01E139D770
:106868000D0A01E162D7050A04E01F0AB4E00E0A26
:10687800DCE00001D807D8A0D9070001D9BF08D0AB
:10688800D95102E1D80504E33C0EDA19DB11DEE147
:10689800030E010196193BE1839E000E0B6EC00E9C
:1068A800CBEC5BF019EC5FF0000E0B6EC00ECBEC7E
:1068B8005BF03C0E0001DA19DB1116E102014B51C5
:1068C8000CE04B0E0F6E020E106E4AEC57F0E60EFF
:1068D8000F6EFE0E106E4AEC57F09C0E0F6EFF0EF8
:1068E800106E4AEC57F0000C350E796F0D0E7A6F6A
:1068F800480E7B6FFF0E7C6F9AC17DF07E6B57EC64
:106908005DF0350E0F6E0D0E106E4AEC57F0000C50
:106918001550D96EDA6ADECF1FF0DDCF20F01C0EDD
:106928001324236E000E1420246E23C00BF024C001
:106938000CF00E6A200E0D6E106A0B0E0F6E7CECBA
:106948005FF0256A266A216A226A1E6A080E1D6E91
:1069580021501F24166E22502020176E16C0F6FFF5
:1069680017C0F7FF000EF86E0E0EF76403D008008C
:10697800F55005D0F6CFE9FFF7CFEAFFEF50276EC5
:10698800214A222A210E276001D0BED02F0E2718B7
:1069980006E05C0E271803E036D0214A222A21504F
:1069A8001F24166E22502020176E16C0F6FF17C03F
:1069B800F7FF000EF86E0E0EF76403D00800F550CE
:1069C80005D0F6CFE9FFF7CFEAFFEF502F0AE5E051
:1069D80021501F24166E22502020176E16C0F6FF75
:1069E80017C0F7FF000EF86E0E0EF76403D008000C
:1069F800F55005D0F6CFE9FFF7CFEAFFEF505C0A74
:106A080001E082D0CAD72E0E271805E01D50255C5C
:106A18001E5026580FE30B0E1D181E10D8B4060C76
:106A28002E0E271801E0060C266A080E256E1E6A2F
:106A38000B0E8DD72750A3EC5BF00B500C1044E0E5
:106A480021501F24166E22502020176E16C0F6FF04
:106A580017C0F7FF000EF86E0E0EF76403D008009B
:106A6800F55005D0F6CFE9FFF7CFEAFFEF501C6EDF
:106A7800214A222A1C50A7EC58F00B500C10D8B40D
:106A8800060C166817681DC018F01EC019F01650BD
:106A98001826175019221850255C1950265801E35A
:106AA800060C25502324D96E26502420DA6E27C0E0
:106AB800DFFF254A262A25502324D96E2650242074
:106AC800DA6E1CC0DFFF1DD0FD0E0B6EFD0E0C6EC6
:106AD80027C00DF00E6A91EC5DF00B500C1001E030
:106AE800060C600E276405D07B0E276002D0200EAE
:106AF800275E25502324D96E26502420DA6E27C01D
:106B0800DFFF254A262A24D721501F24166E22503B
:106B18002020176E1550D96EDA6A16C0DEFF17C02E
:106B2800DDFF2550261001E1060C23C0D9FF24C043
:106B3800DAFFE50EDE1806E123C0D9FF24C0DAFF2C
:106B4800050EDF6E200E276403D01A6A1B6A03D075
:106B58001B6A040E1A6E20EE0BF02350D92624501F
:106B6800DA221AC0DFFF000C01019D6B886B896B6C
:106B7800FF0E1E24226EFF0E1F20236E8986898039
:106B88008982898489888B68849084928494849883
:106B980083500F011391350EE82EFED700F007D071
:106BA800FC0E00019C6FFF0E9D6F0AEC60F08EA832
:106BB800F7D7E1D08EA88EAA14D0FD5112E18851E2
:106BC80089110FE05E0E00019C6FFD0E9D6F88C15C
:106BD8009EF089C19FF00AEC60F0630E01019D6F81
:106BE800D0D0100E746F270E756F766B776BABD0A5
:106BF8008EB28EA410D07407000E755B765B775B3F
:106C0800742906E1752904E1762902E17729D8A4D7
:106C1800B2D0620E84D0010E82D08EA8ACD0020E03
:106C28007ED0350E8825D96E0B0E8921DA6EDF1CD1
:106C3800866E8851221805E18951231802E1FCB3B8
:106C4800899A884B892B8B6A030E9D6F100E746F7F
:106C5800270E756F766B776B06D08EA204D089905D
:106C6800050E9D6F0ED07407000E755B765B775B23
:106C78007429F3E17529F1E17629EFE177297BE0C1
:106C8800ECD7100E746F270E756F766B776B0DD07F
:106C98008EA40BD0898A89808B681E50885D1F500E
:106CA8008959BDE3630E01013AD07407000E755B84
:106CB800765B775B7429ECE17529EAE17629E8E1EE
:106CC800772959E0E5D78EB20DD07407000E755BB1
:106CD800765B775B74294FE175294DE176294BE1A5
:106CE800772949E1040E1BD08990050E9D6F100E7F
:106CF800746F270E756F766B776B3DD089848EB471
:106D08000DD07407000E755B765B775B742933E1F1
:106D1800752931E176292FE177292DE1060E9D6F3E
:106D28002AD0898A89808B681E50885D1F508959AE
:106D380001E271D7B7D7A20E00019C6FFF0E9D6FBD
:106D48000AEC60F0AFD79D51206E216A215013E103
:106D5800205001E14DD7010A01E15FD7030A01E1A3
:106D680060D7010AB0E0070ABFE0010AC7E0030ADA
:106D7800D8E0640AE0E0630E01019D1902E08EBCD0
:106D880019D78980898289848988898A8B680F01C3
:106D9800138188C11EF089C11FF01200350EFE6FE5
:106DA8000B0EFF6FE4C00BF0E5C00CF05BEC5CF081
:106DB8000B500001F26FC20E956F966B976B986B34
:106DC800996B9A6B29EC12F0FB6FFB510BE0940E58
:106DD8009C6FFB0E9D6F0AEC60F0C26BC36BC46BBB
:106DE800C56B1200C20E746F756BFEC076F0FFC0E3
:106DF80077F0010E796F786BF90E7A6F7B6BBFECC9
:106E080017F0FB6FFB5107E0250E9C6FFC0E9D6F82
:106E18000AEC60F0E2D7FEC0D9FFFFC0DAFF800EAF
:106E2800DE1807E01A0E9C6FFD0E9D6F0AEC60F0ED
:106E3800D4D720EE0AF0FE51D926FF51DA22DF50CE
:106E4800E76FE66B20EE0BF0FE51D926FF51DA22F0
:106E5800DF50E625F76F000EE721F86F0E0E9C6FE6
:106E6800FC0E9D6FF7C09EF0F8C09FF00AEC60F032
:106E7800C20E956F966BF751E76FE66BE6C097F019
:106E8800E7C098F0996B9A6B29EC12F0FB6FFB51F5
:106E9800A4E1C20E746F756BFEC076F0FFC077F088
:106EA800010E796F786BF90E7A6F7B6BBFEC17F078
:106EB800FB6FFB5192E1FC6BFD6BE4C00BF0E5C08E
:106EC8000CF0FCC0E6F0FDC0E7F0050ED890E63700
:106ED800E737E82EFBD7E651FE250D6EE751FF2177
:106EE8000E6EF2C00FF0106AAEEC55F00B500C109D
:106EF8005AE1FCC0E6F0FDC0E7F0050ED890E63791
:106F0800E737E82EFBD7FEC0E8F0FFC0E9F0E6510E
:106F1800E827E751E9230E0EE825D96E000EE9218E
:106F2800DA6EDF50EB6FEA6BFCC0ECF0FDC0EDF001
:106F3800050ED890EC37ED37E82EFBD7FEC0EEF003
:106F4800FFC0EFF0EC51EE27ED51EF230F0EEE25C9
:106F5800D96E000EEF21DA6EDF50F06FF16BEA5157
:106F6800F027EB51F123F0C0F3F0F1C0F4F0000E7C
:106F7800F4BFFF0EF56FF66FDF0E9C6FFD0E9D6F71
:106F8800F3C09EF0F4C09FF0F5C0A0F0F6C0A1F0E9
:106F98000AEC60F0F3C0C2F0F4C0C3F0F5C0C4F06E
:106FA800F6C0C5F01200FC4BFD2BFDBF86D7FD5186
:106FB80005E10F0EFC5D01E310D77FD70ED7890ED0
:106FC800F66EF90EF76E0900F5CFB6F00A00F5CFA8
:106FD800B7F00001BC6B02014B6B030E0101FE61AF
:106FE80005D09650FE19F00BFE1905D0FEC193FF8F
:106FF8009650F00B0A09966ECD6ACE6ADBD0BD6B4F
:10700800350E146E0B0E156EB60E166ED2EC54F0CD
:1070180014C0BAF015C0BBF0BAC0D9FFBBC0DAFFC4
:107028003B0EDE1801E0C1D0C5D0BD5109E1BAC0A0
:107038000FF0BBC010F06FEC58F00001BC6FA9D086
:10704800BD0511E10101FB510001BC1903E07F0EF0
:10705800BC1909E1BAC00FF0BBC010F06FEC58F0D2
:107068000101996F96D0020EBD1911E10101FB5182
:107078000001BC1903E07F0EBC1909E1BAC00FF08A
:10708800BBC010F06FEC58F00101986F82D0020E6F
:10709800BD651FD0080EBD611CD00101FB51000168
:1070A800BC1903E07F0EBC1914E1550EB86F020E2F
:1070B800B96FBAC00FF0BBC010F06FEC58F0000108
:1070C800B36FBD51B825B46F000EB921B56FFD0E71
:1070D80040D0070EBD651FD01B0EBD611CD001013D
:1070E800FB510001BC1903E07F0EBC1914E1000E2E
:1070F800B86F020EB96FBAC00FF0BBC010F06FECDA
:1071080058F00001B36FBD51B825B46F000EB92116
:10711800B56FF80E1ED0280EBD6123D00101FB51BA
:107128000001BC1903E07F0EBC191BE1260EB86FE5
:10713800020EB96FBAC00FF0BBC010F06FEC58F078
:107148000001B36FBD51B825B46F000EB921B56FFA
:10715800E50EB425D96EFF0EB521DA6EB3C0DFFF98
:1071680018D0280EBD1915E10101FB510001BC1909
:1071780003E07F0EBC190DE14B0E0B6E020E0C6E78
:10718800BAC00DF0BBC00EF0106A080E0F6EA9EC65
:107198005AF00001BD2B146A156AB60E166ED2ECB1
:1071A80054F014C0BAF015C0BBF00001BA51BB11BD
:1071B80001E03BD7350E00019F6F0B0EA06FA26B4D
:1071C800910EA16F000EA36F030EA46F1CEC55F077
:1071D8009F51A01101E013D71200FC83350E0B6EEE
:1071E8000B0E0C6E0E6A0D6A010E106E0F6AC2EC61
:1071F80047F02BEE35F050C0DFFFFF0EE8CF36FB2F
:1072080050501C0D1B0EF324D96E010EF420DA6EBB
:10721800DFA403D0010EE8CF39FB50501C0D1B0E24
:10722800F324D96E010EF420DA6EDFA003D0020E2B
:10723800E8CF3BFB50501C0D1B0EF324D96E010EFA
:10724800F420DA6EDFA203D0020EE8CF3BFB5050E9
:107258001C0D1B0EF324D96E010EF420DA6EDFA686
:1072680003D0800EE8CF3AFB8FA403D0080EE8CFF6
:107278003BFB266A276A220E00019C6FFB0E9D6F5E
:10728800CECF9EF09F6BCDCFA0F0A16B26C0A2F011
:1072980027C0A3F0370E2624D96E0B0E2720DA6EEE
:1072A800DF50A46FA56B0AEC60F08F0E2624D96E10
:1072B800020E2720DA6EDF1C256E370E2624D96EC3
:1072C8000B0E2720DA6E370E2624E16E0B0E2720D0
:1072D800E26EE7502514DF6E610E9C6FFF0E9D6F06
:1072E800370E2624D96E0B0E2720DA6EDF509E6FDC
:1072F8009F6B0AEC60F0264A272A27BEBCD7275086
:1073080003E1070E265CB7E350501C0D1B0EF32457
:10731800D96E010EF420DA6EDF504E6E50501C0DFF
:10732800010EF324D96E010EF420DA6EDF50246EBC
:1073380024C040FB50501C0D020EF324D96E010EE0
:10734800F420DA6EDF50246E24C041FB50501C0D2F
:10735800030EF324D96E010EF420DA6EDF50246E8A
:1073680024C042FB50501C0D040EF324D96E010EAC
:10737800F420DA6EDF50246E24C043FB50501C0DFD
:10738800050EF324D96E010EF420DA6EDF50246E58
:1073980024C044FB50501C0D060EF324D96E010E78
:1073A800F420DA6EDF50246E24C045FB1F6A140EE9
:1073B8001E6EB8EC35F00101FC938390120050501A
:1073C8001C0D070EF324D96E010EF420DA6EDECF01
:1073D800E2F0DECFE3F0DECFE4F0DECFE5F05050B0
:1073E8001C0D070EF324D96E010EF420DA6E5050EE
:1073F8001C0D0F0EF324E16E010EF420E26EDE5038
:10740800E65CDE50E658DE50E658DE50E658DE50C0
:10741800E658DE50E658DE50E658DE50E65815E2EB
:10742800010E4E6E50501C0D1B0EF324D96E010E2A
:10743800F420DA6E50501C0D1B0EF324E16E010E81
:10744800F420E26EE7500409DF6E50501C0D070E61
:10745800F324D96E010EF420DA6EDECFBEF0DECF53
:10746800BFF0DECFC0F0DECFC1F0DECFC2F0DECF9E
:10747800C3F0DECFC4F0DECFC5F050501C0D170EA0
:10748800F324D96E010EF420DA6EDECFC6F0DECF1B
:10749800C7F0DECFC8F0DECFC9F00001C651CA6F11
:1074A800C751CB6FC851CC6FC951CD6FCE6BCF6B65
:1074B800D06BD16BBE51CA25D26FBF51CB21D36FD0
:1074C800C051CC21D46FC151CD21D56FC251CE212D
:1074D800D66FC351CF21D76FC451D021D86FC551B2
:1074E800D121D96F50501C0D0F0EF324D96E010E07
:1074F800F420DA6ED251DE5CD351DE58D451DE5816
:10750800D551DE58D651DE58D751DE58D851DE58FD
:10751800D951DE5815E2010E4E6E50501C0D1B0E4F
:10752800F324D96E010EF420DA6E50501C0D1B0E98
:10753800F324E16E010EF420E26EE7500409DF6ED9
:107548004E6A5050220D000EF324956F030EF4205E
:10755800966FE2C097F0E3C098F0E4C099F0E5C0F8
:107568009AF029EC12F0E66FE65115E0010E4E6E26
:1075780050501C0D1B0EF324D96E010EF420DA6E48
:1075880050501C0D1B0EF324E16E010EF420E26E28
:10759800E7500409DF6E4E5012008EA604D0E50EA7
:1075A8001E6EFE0E03D0B70E1E6EFF0E1F6E8EAA45
:1075B80004D0E50E206EFE0E03D0B20E206EFF0E34
:1075C800216E8EA804D0E50E226EFE0E03D0120E98
:1075D800226EFF0E236E8EAE04D0E50E246EFE0ED4
:1075E80003D0BC0E246EFF0E256E8EAC04D0E50EC3
:1075F800266EFE0E03D0AD0E266EFF0E276E8EA4ED
:1076080004D0E50E286EFE0E03D0C60E286EFF0EBF
:10761800296E8EA204D0E50E2A6EFE0E03D0CB0E84
:107628002A6EFF0E2B6E8EA004D0E50E2C6EFE0E79
:1076380003D0C10E2C6EFF0E2D6E90AE04D0E50E59
:107648002E6EFE0E03D0F90E2E6EFF0E2F6E90AC2E
:1076580004D0E50E306EFE0E03D0F60E306EFF0E2F
:10766800316E90AA04D0E50E326EFE0E03D0F30EF2
:10767800326EFF0E336E90A804D0E50E346EFE0E07
:1076880003D0F00E346EFF0E356E90A604D0E50ED2
:10769800366EFE0E03D0ED0E366EFF0E376E90A4DA
:1076A80004D0E50E386EFE0E03D0EA0E386EFF0EDB
:1076B800396E90A204D0E50E3A6EFE0E03D0E70EA6
:1076C8003A6EFF0E3B6E90A004D0E50E3C6EFE0EA7
:1076D80003D0E40E3C6EFF0E3D6ED00E00019C6F91
:1076E800F90E9D6F901C9E6F9F6B8ECFA0F0A16BC3
:1076F8003CC0A2F03DC0A3F03AC0A4F03BC0A5F046
:1077080038C0A6F039C0A7F036C0A8F037C0A9F035
:1077180034C0AAF035C0ABF032C0ACF033C0ADF025
:1077280030C0AEF031C0AFF02EC0B0F02FC0B1F015
:107738002CC0B2F02DC0B3F02AC0B4F02BC0B5F005
:1077480028C0B6F029C0B7F026C0B8F027C0B9F0F5
:1077580024C0BAF025C0BBF022C0BCF023C0BDF0E5
:1077680020C0BEF021C0BFF01EC0C0F01FC0C1F0D5
:107778000AEF60F0070E0B241A6E000E0C201B6E29
:107788000BC0D9FF0CC0DAFFDF500F6E0F380F0B9C
:107798000A0DF3CF10F0F4CF11F00BC0D9FF0CC0D5
:1077A800DAFFDF500F0B1026000E11221028186E7A
:1077B800000E1120196E1D6A010E1C6E1E6A1F6ACA
:1077C800206A216AB2D01C501D1054E01EC00FF070
:1077D8001FC010F020C011F021C012F00A0E0F02D5
:1077E800F3CF13F0F4CF14F0156A166A1002F350B1
:1077F8001426F4501522000E16220F02F3501426F8
:10780800F4501522000E16220A0E1102F350152606
:10781800F4501622000E1002F3501526F4501622CA
:10782800000E0F02F3501526F45016220A0E12020B
:10783800F3501626000E1102F3501626000E100201
:10784800F3501626000E0F02F35016261AC0D9FF61
:107858001BC0DAFFDF50176E17380F0B13241E6E8C
:10786800000E14201F6E000E1520206E000E16202C
:10787800216E54D01EC00FF01FC010F020C011F0B0
:1078880021C012F00A0E0F02F3CF13F0F4CF14F058
:10789800156A166A1002F3501426F4501522000EC9
:1078A80016220F02F3501426F4501522000E162249
:1078B8000A0E1102F3501526F4501622000E10027B
:1078C800F3501526F4501622000E0F02F350152619
:1078D800F45016220A0E1202F3501626000E110258
:1078E800F3501626000E1002F3501626000E0F0253
:1078F800F35016261AC0D9FF1BC0DAFFDF500F0B52
:1079080013241E6E000E14201F6E000E1520206E0C
:10791800000E1620216E1A06D8A01B061C501D103A
:10792800010ED8A4000E1C6E1D6A1806D8A01906F0
:10793800182802E11928D8A446D71EC00BF01FC08A
:107948000CF020C00DF021C00EF012000001D16B28
:10795800010ED06F838E8380D26BD36BD46BD56BC3
:10796800CED05050220D000EF324746F030EF42075
:10797800756F350E766F0B0E776F010E796F786B1A
:10798800D80E7A6F7B6BBFEC17F0DA6FDA5118E01C
:10799800180E01018D6F010E8F6F0001D96BD86F22
:1079A800E00E9C6FFA0E9D6F50C09EF09F6BDAC080
:1079B800A0F0A16BD8C0A2F0D9C0A3F00AEC60F087
:1079C8000101945135E0705171117211731130E059
:1079D80050500C0D630EF324D96E020EF420DA6EAB
:1079E80070C1C7F071C1C8F072C1C9F00001C66B9F
:1079F800000EC625CA6F010EC721CB6F000EC82125
:107A0800CC6F000EC921CD6FDE50CA1911E1DE50CE
:107A1800CB190EE1DE50CC190BE1DE50CD1908E18F
:107A2800350E286E0B0E296E01019451A3EC4DF012
:107A38000101FC938D5101E0FC83D8C01EF0D9C030
:107A48001FF0B8EC35F01EC0D6F01FC0D7F000010B
:107A5800D651D227D751D323000ED423D5238EACA9
:107A680053D0D851D61903E1D951D7190CE0D06BAE
:107A7800D16B8E0E9C6FFE0E9D6FD6C09EF0D7C048
:107A88009FF00AEC60F0C1EC5FF0A2EC5FF00B50E5
:107A98000C1004E0010E01018F6F36D00001CF6B8E
:107AA800050ECE6F1CD0D00E0001C26FC90EE82E95
:107AB800FED7C22FFCD700D0A2EC5FF00B500C1001
:107AC8000EE00001D06BD16B6F0E9C6FFD0E9D6FA9
:107AD800CEC09EF0CFC09FF00AEC60F008D0000145
:107AE800CE07D8A0CF07CE29DEE1CF29DCE1A2EC72
:107AF8005FF00B500C1003E00001D06BD16B00015C
:107B0800D051D11101E02DD701018F6B839E839055
:107B18001200838E83804E6AE3EC39F00101BA6F5C
:107B2800BA5102E0BA511200536AB26BB36BB46B2C
:107B3800B56BB96B010EB86FBD6BC3D0BB6BBC6BBB
:107B48001CD0A2EC5FF00B500C1013E0BD0E0B6EB6
:107B5800010E0C6E3CEC56F00101B76F000E532479
:107B6800D96EDA6A040EDA22B7C1DFFF532ABB4B9B
:107B7800BC2B0101BDAB8EAC02D0BC05E2E3BB510E
:107B8800B227BC51B323000EB423B52350501C0DAB
:107B9800170EF324D96E010EF420DA6EDE50B25DB2
:107BA800DE50B359DE50B459DE50B55902E3B86B14
:107BB800B96BBDAB02D0B86BB96B8EBC02D0B86BD9
:107BC800B96BBC0519E2000E53240B6E0C6A040E47
:107BD8000C22FF0E5324D96EDA6A030EDA22DF5024
:107BE8000D6E0E6A535000080F6E000ED8A0E82ADA
:107BF8000108106EC2EC47F00101945145E0705144
:107C080071117211731140E050503EE150501C0D3B
:107C1800070EF324D96E010EF420DA6E70C1A7F1B5
:107C280071C1A8F172C1A9F1A66B000EA625AA6FB1
:107C3800010EA721AB6F000EA821AC6F000EA92181
:107C4800AD6FAE6BAF6BB06BB16BDE50AA191CE1B8
:107C5800DE50AB1919E1DE50AC1916E1DE50AD1952
:107C680013E1DE50AE1910E1DE50AF190DE1DE5020
:107C7800B0190AE1DE50B11907E1000E226E040EB8
:107C8800236E9451F5EC55F0F0EC52F00101B66F0B
:107C9800B65117E0010E4E6E50501C0D1B0EF3240A
:107CA800D96E010EF420DA6E50501C0D1B0EF32411
:107CB800E16E010EF420E26EE7500409DF6E4E50CB
:107CC8001200B851B91101E039D78FA402D0010EC2
:107CD8004E6E8390839E000C9451D8B412008F0E80
:107CE80000019C6FFD0E9D6F0AEC60F0EAEC53F00A
:107CF8001EC0A4F11FC0A5F120C0A6F121C0A7F1A4
:107D08000101A451A511A611A71117E16A0E0001DE
:107D18009C6FFC0E9D6FA4C19EF0A5C19FF0A6C1EB
:107D2800A0F0A7C1A1F00AEC60F00A0E0E6E000EDA
:107D38000F6A106A116A28EC5BF00101A86BA96B45
:107D4800E00E00019C6FFF0E9D6FA40E0101A82597
:107D5800D96E010EA921DA6EDF5000019E6F9F6B6C
:107D68000AEC60F00101A84BA92BA9BFE9D7A951DA
:107D780003E1040EA85DE4E34A0E00019C6FFA0ECD
:107D88009D6F0AEC60F07A0E9C6FFB0E9D6F0AECFB
:107D980060F023EE00F000EEC2F0210EDBCFEBFF27
:107DA800E806FCE2D40EE46FFF0EE56FD2EC36F085
:107DB800C2C070F1C3C071F1C4C072F1C5C073F123
:107DC80001017051711172117311D8B41200600E53
:107DD80000019C6FFB0E9D6F70C19EF071C19FF0FA
:107DE80072C1A0F073C1A1F00AEC60F0000E956FAB
:107DF800030E966F70C19FF171C1A0F172C1A1F11C
:107E080001019E6B000E9E250001976F010E010176
:107E18009F210001986F000E0101A0210001996FB8
:107E2800000E0101A12100019A6F29EC12F0010155
:107E38009A6F000E0001746F030E756F350E766F22
:107E48000B0E776F796B080E786FA20E7A6F010EA2
:107E58007B6FBFEC17F001019A6FAA6BAB6BDC0E5E
:107E680000019C6FFF0E9D6F350E0101AA25D96E8A
:107E78000B0EAB21DA6EDF5000019E6F9F6B0AEC90
:107E880060F00101AA4BAB2BABBFE9D7AB5105E1C1
:107E9800080EAA5DD8B01200E2D7120043C024F041
:107EA80044C025F058EC43F0456E455001E0D4D06D
:107EB80043C0D9FF44C0DAFF030EDE1801E0BCD08E
:107EC80020EE04F04350D9264450DA22DE0401E0C3
:107ED800B3D02F0E43240B6E000E44200C6E0E6A96
:107EE8000D6A020E106E0F6A7CEC5FF02D0E4324B3
:107EF8000B6E020E44200C6EAA0E0E6E550E0D6E01
:107F080042EC5FF02F0E43240B6E000E44200C6EE3
:107F1800520E0D6E0E6E610E0F6E410E106E4CEC11
:107F280059F0130E43240B6E020E44200C6E720E91
:107F38000D6E0E6E410E0F6E610E106E4CEC59F008
:107F4800170E43240B6E020E44200C6E20EE0FF029
:107F58004350D9264450DA22DECF0DF0DECF0EF0A2
:107F6800DECF0FF0DECF10F04CEC59F01B0E43249F
:107F78000B6E020E44200C6E20EE0BF04350D926F7
:107F88004450DA22DECF0DF0DECF0EF0DECF0FF058
:107F9800DECF10F04CEC59F020EE1BF04350D92600
:107FA8004450DA22DECF60F0DECF61F0DECF62F03F
:107FB800DECF63F0010E00016025646F000E6121C1
:107FC800656F000E6221666F000E6321676F20EEF9
:107FD8002BF04350D9264450DA2264C0DEFF65C036
:107FE800DEFF66C0DEFF67C0DEFF2F0E43241A6E79
:107FF800000E44201B6E20EE2BF04350D92644502F
:10800800DA22DECF1CF0DECF1DF0DECF1EF0DECF91
:108018001FF0216A010E206E20EE01F04350D92690
:108028004450DA22DF5004EC4FF020EE04F04350C5
:10803800D9264450DA22DF6A1A6A1B6A1C6A20EEC3
:1080480001F04350D9264450DA22DF50D8EC20F012
:10805800000902E0010E456E45501200276E00012E
:10806800C35102E010EC30F0266A0001C25101E170
:10807800AED0040E271802E14F5003E1140E271862
:1080880009E10101926B826B836B0001C36B070EE0
:10809800C26F070C3F0E271807E14F6A0101926B68
:1080A8000001C26BC36B12005F0E271807E10101C4
:1080B800936B926B0001C26BC36B12003F0E276477
:1080C80006D05F0E276003D0400E2718F0E1400E5F
:1080D800271809E1010E0101936F0101926B00015C
:1080E800C26BC36B1200200E271803E1010E4F6EFE
:1080F800F4D7650E271809E14F5007E00101826B9C
:10810800836B010E926F8380EAD76E0E271803E106
:10811800020E0101926F700E271807E101019351B9
:1081280004E0826B836B030E926F700E271808E1D0
:108138004F5006E083800101826B836B040E0CD0E4
:10814800720E271844E14F5042E083801C0E010153
:10815800836F2A0E826F050E926FC1D7275008ECE5
:108168000CF0266E46D083802750C4EC56F0266E5D
:108178000101926B3ED08380350E0B6E0B0E0C6E98
:108188000E6A0D6A010E106E0F6AC2EC47F001010B
:10819800FC832BEE35F04EC0DFFF1F6A010E1E6E0A
:1081A800B8EC35F00101FC93080EE1D78390266AFC
:1081B80020D0080E271801E103D0090E271819E16D
:1081C8008390266A4E6A926B826B836B12D0010190
:1081D8009251246E256A25500CE124500AE0010AC8
:1081E800BDE0030AC0E0010AC6E0070ADFE0010AB1
:1081F800E0E026C0C2F00001C36B1200BBC0D9FF8B
:10820800BCC0DAFFDECFC5F0DDCFC6F003D0000179
:10821800BD4BBE2BBDC0F6FFBEC0F7FF000EF86E0B
:108228000E0EF76403D00800F55005D0F6CFE9FF2D
:10823800F7CFEAFFEF502F0AEAE0BDC0F6FFBEC055
:10824800F7FF000EF86E0E0EF76403D00800F55025
:1082580005D0F6CFE9FFF7CFEAFFEF505C0AD7E089
:10826800000120EE06F0BB51D926BC51DA22DE6AA5
:10827800DE6ADE6ADD6ABDC0F6FFBEC0F7FF000E2B
:10828800F86E0E0EF76403D00800F55005D0F6CF4F
:10829800E9FFF7CFEAFFEF500001BF6F200EBF6183
:1082A80014D020EE27F0BB51D926BC51DA22800E1B
:1082B800DF6EBBC074F0BCC075F0000E766F776FD0
:1082C800786F796FB1EC31F023D0BBC013F0BCC02C
:1082D80014F0BD0E156E8CEC34F00001C86FC85157
:1082E80058E1BBC0B3F0BCC0B4F058EC48F0C86F5C
:1082F80020EE27F0BB51D926BC51DA22DF50C76FD8
:10830800C85108E0040EC81944E1C7B542D0050EAB
:10831800C86F3FD0C7B53DD020EE04F0BB51D92679
:10832800BC51DA22DFA8F3D7C5C012F0C6C013F0DB
:10833800BF69010EC06F20EE0EF0BB51D926BC51AB
:10834800DA22DECFC1F0DDCFC2F0BF51C117C05174
:10835800C217C5C0C3F0C6C0C4F0C151C327C251BB
:10836800C4232F0EC325146E000EC421156EFCEC19
:1083780057F0000120EE06F0BB51D926BC51DA2295
:1083880012C0DEFF13C0DEFF14C0DEFF15C0DEFF23
:108398009CD7C851120078C0D9FF79C0DAFFDECF68
:1083A8008FF0DDCF90F07D517C117B1104E1020E3E
:1083B8007A5DD8A0020C20EE13F08F51D926905187
:1083C800DA22DE507A5DDE507B59DE507C59DE5071
:1083D8007D5901E3020C7E517F118011811118E053
:1083E8008FC060F090C061F07EC062F07FC063F023
:1083F80080C064F081C065F0666967696869696909
:10840800BBEC1EF000018E6F8E5102E08E511200FF
:1084180078C042F079C043F07AC044F07BC045F0A0
:108428007CC046F07DC047F0AFEC2CF042C08AF02B
:1084380043C08BF044C08CF045C08DF000018A51D8
:108448008B118C118D1171E08A058B118C118D1196
:1084580001E1020C8A2907E18B2905E18C2903E156
:108468008D2901E1010C8FC060F090C061F07AC0E5
:1084780062F07BC063F07CC064F07DC065F0666B21
:10848800676B686B696BBBEC1EF000018E6F8E51D9
:10849800BDE120EE13F08F51D9269051DA22FE0E5D
:1084A800DE24826FFF0EDE20836FFF0EDE20846FD6
:1084B800FF0EDE20856F20EE0FF08F51D9269051E8
:1084C800DA228251DE5C8351DE588451DE588551B0
:1084D800DE5813E220EE0FF08F51D9269051DA22A0
:1084E800DE2A000EDE22DE22DE2220EE04F08F518C
:1084F800D9269051DA22000EDB808AC07AF08BC030
:108508007BF08CC07CF08DC07DF020EE13F08F5195
:10851800D9269051DA22DE507A5DDE507B59DE5042
:108528007C59DE507D5901E273D7000C1B6E1B503D
:1085380001E0010C54A202D054501200000E2EEC9F
:108548005FF00A0E266E03D02EEC60F02606265049
:10855800FBE1236A000E146A156A166A176AADEC05
:108568005DF0E80601E097D0AA0E146E010E156EB4
:10857800166A176A080EADEC5DF0E80651E1266A46
:1085880026501C0FD96EDA6A2EEC60F0DF6E262AB0
:10859800030E2664F5D71E047EE1AA0E1F187BE1A0
:1085A800030E256EE80E246E15D0146A156A166A35
:1085B800400E176EA90EADEC5DF000090EE0150E29
:1085C8001A6EC60EE82EFED71A2EFCD700D0240647
:1085D800D8A0250624502510E8E1245025105BE09A
:1085E800146A156A166A176A3A0EADEC5DF000094E
:1085F80052E1266A26501C0FD96EDA6A2EEC60F01A
:10860800DF6E262A030E2664F5D71CBC03D0216A28
:10861800040E02D0216A0C0E206E20C023F03BD03D
:10862800146A156A166A176AA90EADEC5DF01A6E1F
:10863800020E1A6003D0236EA90E02D0010E236E1B
:10864800226E030E256EE80E246E14D0146A156A85
:10865800166A176A2250ADEC5DF000090EE0150E9F
:108668001A6EC60EE82EFED71A2EFCD700D02406A6
:10867800D8A0250624502510E9E1245025100AE049
:10868800146A020E156E166A176A100EADEC5DF0CC
:10869800000901E0236A23C051F03FEC60F0235049
:1086A80001E14AD7549048D7366A20EE03F02450A7
:1086B800D9262550DA22DF5001E1A7D02F0E242435
:1086C8001A6E000E25201B6E20EE2BF02450D926A2
:1086D8002550DA22DECF1CF0DECF1DF0DECF1EF0F3
:1086E800DECF1FF0216A010E206E20EE01F024502B
:1086F800D9262550DA22DF5004EC4FF0000901E0BA
:1087080082D020EE03F02450D9262550DA22DF6AE1
:1087180020EE17F02450D9262550DA2210EE1FF04B
:108728002450E1262550E222E6CF2AF0E6CF2BF0AE
:10873800E6CF2CF0E6CF2DF010EE2BF02450E126FA
:108748002550E222E6CF2EF0E6CF2FF0E6CF30F02C
:10875800E6CF31F02A502E5C326E2B502F58336EF4
:108768002C503058346E2D503158356EDE50325CF6
:10877800DE503358DE503458DE50355846E220EE8D
:1087880002F02450D9262550DA22020EDE183DE1E7
:108798002F0E24241A6E000E25201B6E20EE17F0D3
:1087A8002450D9262550DA22DECF26F0DECF27F056
:1087B800DECF28F0DECF29F020EE2BF02450D9268A
:1087C8002550DA22DECF2AF0DECF2BF0DECF2CF0D8
:1087D800DECF2DF026502A241C6E27502B201D6E2C
:1087E80028502C201E6E29502D201F6E216A010E44
:1087F800206E20EE01F02450D9262550DA22DF50D1
:1088080004EC4FF002D0010E366E3650120046C00E
:108818000CF047C00DF06D0E0E6E9AEC52F0000190
:108828006C6F6C5101E099D020EE0EF04650D926BD
:108838004750DA22DFAC91D06DC037F06EC038F007
:1088480020EE1CF04650D9264750DA22DECF39F008
:10885800DECF3AF0DECF3BF0DECF3CF039EC54F01F
:1088680000016C6F6C5179E120EE20F04650D9265A
:108878004750DA22DECF6FF0DDCF70F020EE0BF03C
:108888006F51D9267051DA22000EDB8A46C0D9FF13
:1088980047C0DAFFDECF0FF0DDCF10F06FC011F068
:1088A80070C012F020EE06F04650D9264750DA2262
:1088B800DECF13F0DECF14F0DECF15F0DECF16F0EA
:1088C800DDEC5CF01C0E00016F250B6E000E7021B4
:1088D8000C6E20EE0AF04650D9264750DA22DECF39
:1088E8000DF0DECF0EF0DECF0FF0DECF10F04CEC47
:1088F80059F0160E00016F250B6E000E70210C6EDC
:108908000D6A0E6A210E0F6E500E106E4CEC59F067
:10891800120E00016F250B6E000E70210C6E000EFA
:108928000E6A0D6A42EC5FF0000120EE03F06D5113
:10893800D9266E51DA22010EDF6E6DC043F06EC08B
:1089480044F052EC3FF000016C6F20EE0EF0465000
:10895800D9264750DA22BF0EDF166C5112008968FB
:108968008B688E280BE1AD0E00019C6FFB0E9D6F8E
:108978008ECF9EF09F6B0AEC60F00AD0980E000133
:108988009C6FFA0E9D6F8ECF9EF09F6B0AEC60F085
:1089980090280AE1530E9C6FFC0E9D6F8ECF9EF0BF
:1089A8009F6B0AEC60F009D0BD0E9C6FFA0E9D6FAC
:1089B8008ECF9EF09F6B0AEC60F0290E3F6E960EEC
:1089C8003E6E7F0EE82EFED73E2EFCD73F2EFAD7FE
:1089D80000F0A80E00019C6FFE0E9D6F0AEC60F07F
:1089E80089988498090E3F6E1E0E3E6EE40EE82E9E
:1089F800FED73E2EFCD73F2EFAD700D09B0E0001A3
:108A08009C6FFE0E9D6F0AEC60F0899A849A090E9D
:108A18003F6E1E0E3E6EE40EE82EFED73E2EFCD7AD
:108A28003F2EFAD700D0000E00019C6FFF0E9D6FFD
:108A38000AEC60F088908D9090280AE0530E9C6FA5
:108A4800FC0E9D6F90CF9EF09F6B0AEC60F009D0F2
:108A58004D0E9C6FFA0E9D6F90CF9EF09F6B0AECA7
:108A680060F08D80A30E3F6E570E3E6E020EE82E0C
:108A7800FED73E2EFCD73F2EFAD700D089688B68E8
:108A88008A6883928382290E3F6E960E3E6E7F0E11
:108A9800E82EFED73E2EFCD73F2EFAD700F0D1ECB9
:108AA8003AF0EFD71C6A1AAE12D01A1E191E181EF9
:108AB800171E161E151E141E136C000E14221522E6
:108AC80016221722182219221A22010E1C6E12AE23
:108AD80012D0121E111E101E0F1E0E1E0D1E0C1E71
:108AE8000B6C000E0C220D220E220F2210221122D6
:108AF8001222010E1C1A1D6A1E6A1F6A206A216A48
:108B0800226A236A246A13501410151016101710BD
:108B1800181019101A1045E0010E1B6E0AD0D890D3
:108B280013361436153616361736183619361A36D9
:108B38001B2A1AAEF4D7D8901D361E361F3620369B
:108B4800213622362336243613500B5C14500C5829
:108B580015500D5816500E5817500F5818501058D9
:108B6800195011581A50125811E313500B5E145033
:108B78000C5A15500D5A16500E5A17500F5A1850B5
:108B8800105A1950115A1A50125A1D80D8901A3278
:108B980019321832173216321532143213321B2E8C
:108BA800CAD71C5010E0241E231E221E211E201E80
:108BB8001F1E1E1E1D6C000E1E221F222022212297
:108BC8002222232224221DC00BF01EC00CF01FC03D
:108BD8000DF020C00EF021C00FF022C010F023C00D
:108BE80011F024C012F01200166817680B50D96EE5
:108BF800DA6ADECF18F0DDCF19F018C013F019C00B
:108C080014F01850191003E10B680C68120013C017
:108C1800F6FF14C0F7FF000EF86E0E0EF76403D0CF
:108C28000800F55005D0F6CFE9FFF7CFEAFFEF507F
:108C3800156E134A142A200E156403D03A0E15181F
:108C4800E6E13A0E151868E1000E126E010E116E7B
:108C580018C0F6FF19C0F7FF000EF86E0E0EF76485
:108C680003D00800F55005D0F6CFE9FFF7CFEAFFAB
:108C7800EF500D6E2F0E0D6439D018C0F6FF19C0D5
:108C8800F7FF000EF86E0E0EF76403D00800F550DB
:108C980005D0F6CFE9FFF7CFEAFFEF500D6E3A0E99
:108CA8000D6024D0020E18240D6E000E19200E6ED1
:108CB80013500D181BE114500E1818E118C0F6FFD8
:108CC80019C0F7FF000EF86E0E0EF76403D0080007
:108CD800F55005D0F6CFE9FFF7CFEAFFEF500D6E5C
:108CE800D00E0D24116E126AFF0E122212BE04D08D
:108CF80012500DE111040BE211C016F012C017F06A
:108D08000B50D96EDA6A13C0DEFF14C0DDFF16C03F
:108D18000BF017C00CF012000B6A0C6A120060C04E
:108D280042F061C043F0446A456A466A476A26ECE5
:108D38004DF042C078F043C079F0020E0001781976
:108D480079110DE0795106E1030E785D03E2625175
:108D5800631105E178C060F079C061F012007A6BA8
:108D68007B6B7AC064F07BC065F0643B653BF00EBA
:108D7800651764510F0B6513F00E641760C066F039
:108D880061C067F06451662765516723F50E662553
:108D98000B6E010E67210C6E44EC53F000017A5102
:108DA800040DF350680FD96EDA6A0BC0DEFF0CC0F1
:108DB800DEFF0DC0DEFF0EC0DEFF7A4B7B2B7B5142
:108DC80003E1040E7A5DCDE36251631103E17A6B2E
:108DD8007B6B06D0FF0E62257A6FFF0E63217B6FD7
:108DE8007A51040DF350680FD96EDA6ADE50DE103E
:108DF800DE10DE1004E1796B030E786F18D060C0C6
:108E080042F061C043F07A51040DF350680FD96EF7
:108E1800DA6ADECF44F0DECF45F0DECF46F0DECFB3
:108E280047F026EC4DF042C078F043C079F00001DD
:108E3800625163118FE1795103E1020E785D8AE393
:108E48007A4B7B2B7B5186E1040E7A5D83E2C8D78F
:108E58002F6C696664617461302E62696E20002F20
:108E68006C696664617461312E62696E20002F6CD2
:108E7800696664617461322E62696E20002F6C69C4
:108E88006664617461332E62696E20002F6C6966B6
:108E980064617461342E62696E20002F6C696664A7
:108EA800617461352E62696E20002F6C6966646199
:108EB8007461362E62696E20002F6C696664617475
:108EC80061372E62696E20002F6C69666461746177
:108ED800382E62696E20002F6C696664617461398E
:108EE8002E62696E20002F6C696664617461612E60
:108EF80062696E20002F6C696664617461622E621B
:108F0800696E20002F6C696664617461632E626902
:108F18006E20002F6C696664617461642E62696EEC
:108F280020002F6C696664617461652E62696E2029
:108F3800002F6C696664617461662E62696E200038
:108F48000000000000000000000000000000000019
:108F58000000000000000000000000000000000009
:108F680000000000000000000000000000000000F9
:108F78000000000000000000000000000BC015F019
:108F88000CC016F00F50101001E1120015C0D9FFE7
:108F980016C0DAFF0DC0DFFF0F501524116E1050F8
:108FA8001620126EFF0E1124D96EFF0E1220DA6EF3
:108FB8000DC0DFFF105004E1030E0F5C01E2120048
:108FC80020EE01F01550D9261650DA220DC0DFFF29
:108FD80020EE02F01550D9261650DA220DC0DFFF18
:108FE8000F501524116E10501620126EFE0E11240B
:108FF800D96EFF0E1220DA6E0DC0DFFF0F50152458
:10900800116E10501620126EFD0E1124D96EFF0E2F
:109018001220DA6E0DC0DFFF105004E1070E0F5C5E
:1090280001E2120020EE03F01550D9261650DA227C
:109038000DC0DFFF0F501524116E10501620126E50
:10904800FC0E1124D96EFF0E1220DA6E0DC0DFFF60
:10905800105004E1090E0F5C01E2120015C011F076
:1090680016C012F0111E121E114A122A030E1114F4
:10907800136E146A135015261450162213500F5EDF
:109088001450105AFC0E0F160BD015C0D9FF16C07D
:10909800DAFF0DC0DFFF0F06D8A01006154A162A02
:1090A8000F501010F2E11200B3C0D9FFB4C0DAFFBC
:1090B800DECFB7F0DDCFB8F0B3C074F0B4C075F050
:1090C800000E766F776F786F796FB1EC31F0BA6F09
:1090D800BA5103E00001BA511200B7C037F0B8C066
:1090E80038F020EE16F0B351D926B451DA22DECF8B
:1090F80039F0DECF3AF0DECF3BF0DECF3CF039EC92
:1091080054F00001BA6FBA51E5E120EE1AF0B351FC
:10911800D926B451DA22DECFB5F0DDCFB6F0B5C02E
:10912800D9FFB6C0DAFFDF50B96FB95103E1040EB9
:10913800BA6FD0D720EE04F0B351D926B451DA2251
:1091480010EE1AF0B351E126B451E22200EE0BF012
:10915800E650E926E550EA22EF503F0BDF6E20EE9D
:109168001AF0B351D926B451DA2210EE0BF0DE50C2
:10917800E126DD50E222E7B618D020EE1AF0B3510E
:10918800D926B451DA22DECF0BF0DDCF0CF01C0E5D
:10919800B3250D6E000EB4210E6E106A0B0E0F6E05
:1091A80016EC59F00B500C1095E0B3C095F0B4C014
:1091B80096F00001986B976B6EEC2EF00001BA6F79
:1091C800BA5188E18AD718C00BF019C00CF00E6AA2
:1091D8000D6A106A080E0F6EC2EC47F0236A020E81
:1091E800226E22501824D96E23501920DA6E22508C
:1091F80018241E6E235019201F6E1E28E16E000EC3
:109208001F20E26EE750206E203AF00E201620163E
:1092180022501824E16E23501920E26EE750216E87
:1092280021380F0B2010DF6E224A232A23BED9D7FC
:10923800235003E1070E225CD4E322501824D96E90
:1092480023501920DA6E1AC00BF01BC00CF01CC09A
:109258000DF01DC00EF00A0E0F6E106A116A126A28
:10926800EAEC59F00B3AF00E0B1622501824E16E76
:1092780023501920E26EE7501E6E1E380F0B0B109C
:10928800DF6E18C0D9FF19C0DAFFDF2A1AC00BF049
:109298001BC00CF01CC00DF01DC00EF00A0E0F6EA6
:1092A800106A116A126A87EC57F00BC01AF00CC0EA
:1092B8001BF00DC01CF00EC01DF01A501B101C1026
:1092C8001D108CE118C0D9FF19C0DAFFDF06090E9E
:1092D800DF64090C18C0D9FF19C0DAFF100EDF6E61
:1092E800100C000E0101E26F0A0EE16F000EE06F34
:1092F800050EDF6F7DD00101E26B140EE16F70D0B7
:10930800AA0E0C6EFC0E0D6EFEEC5AF08FB204D055
:109318000101E26B1E0EE16F090E0001FE6F1E0EC9
:10932800FD6FE40EE82EFED7FD2FFCD7FE2FFAD7EF
:1093380000F056D0E80E0C6EFE0E0D6EFEEC5AF0E4
:10934800060E0001B16F090EB26F4C0EB36FFA0E24
:10935800B46FB56B66EC55F001019A6F9A517AECCF
:109368005BF001019A51D8E1E26B230ED4D7390E94
:109378000C6EFE0E0D6EFEEC5AF0000E0001C96F69
:10938800030ECA6F400ECB6F020ECC6F010ECD6F6D
:10939800F7EC14F001019A6F9A517AEC5BF0010135
:1093A8009A510AE106EC29F0000E486E030E496E48
:1093B8003AEC5DF001019A6F9A517AEC5BF0010C7E
:1093C800E1C1FDF0E2C1FEF00001FE5109E1FD51ED
:1093D8000A0A91E01E0A94E00A0AACE03D0AC7E0D6
:1093E800140E0101E119E21103E0DF07D8A0E0073C
:1093F800E0BF000CE051E4E1DF05E2E2000C1C6A8A
:1094080012AE12D0121E111E101E0F1E0E1E0D1EA1
:109418000C1E0B6C000E0C220D220E220F221022A5
:1094280011221222010E1C6E1AAE10D01A1E191E1D
:10943800181E171E161E151E141E136C000E14225D
:10944800152216221722182219221A221350141034
:10945800151016101710181019101A103BE0010EED
:109468001B6E0AD0D89013361436153616361736B2
:10947800183619361A361B2A1AAEF4D713500B5C55
:1094880014500C5815500D5816500E5817500F58A8
:1094980018501058195011581A50125810E31350F8
:1094A8000B5E14500C5A15500D5A16500E5A175080
:1094B8000F5A1850105A1950115A1A50125AD89057
:1094C8001A32193218321732163215321432133250
:1094D8001B2ED4D71C5010E0121E111E101E0F1E7A
:1094E8000E1E0D1E0C1E0B6C000E0C220D220E22E1
:1094F8000F221022112212220BC00BF00CC00CF00C
:109508000DC00DF00EC00EF00FC00FF010C010F01F
:1095180011C011F012C012F01200020E0D5E000E02
:109528000E5A0F5A105A20EE13F00B50D9260C5031
:10953800DA22FE0EDE24116EFF0EDE20126EFF0E02
:10954800DE20136EFF0EDE20146E11500D5C1250DB
:109558000E5813500F581450105805E30B6A0C6A34
:109568000D6A0E6A120020EE27F00B50D9260C5017
:10957800DA22DECF11F0DECF12F0DECF13F0DECF2D
:1095880014F020EE09F00B50D9260C50DA22DECF69
:1095980015F0DDCF16F01550176E1650186E196AB3
:1095A8001A6A17500D02F3CF1BF0F4CF1CF01D6A96
:1095B8001E6A0E02F3501C26F4501D22000E1E22B5
:1095C80018500D02F3501C26F4501D22000E1E22C6
:1095D80017500F02F3501D26F4501E2218500E0289
:1095E800F3501D26F4501E2219500D02F3501D266B
:1095F800F4501E2210501702F3501E2618500F0266
:10960800F3501E2619500E02F3501E261A500D0252
:10961800F3501E2611501B240B6E12501C200C6E8A
:1096280013501D200D6E14501E200E6E1200838ED6
:1096380083800001F76BF86BC2EC57F01EC0F9F09D
:109648001FC0FAF0040E0001FA5D07E3000EF925C9
:10965800F76FFC0EFA21F86F04D0F9C0F7F0FAC0E2
:10966800F8F00101945133E07051711172117311C6
:109678002EE050500C0D630EF324D96E020EF42028
:10968800DA6E70C1A3F171C1A4F172C1A5F1A26B28
:10969800000EA225A66F010EA321A76F000EA4211C
:1096A800A86F000EA521A96FDE50A61910E1DE50A3
:1096B800A7190DE1DE50A8190AE1DE50A91907E142
:1096C800000E226E040E236E9451F5EC55F08FB403
:1096D80015D05050220D000EF3240001956F030E93
:1096E800F420966F000E976F040E986F010E9A6F14
:1096F800996BF70E9B6FC9EC08F0F66F0001F651F5
:1097080009E07F0E9C6FFD0E9D6FF6C09EF09F6B6B
:109718000AEC60F00BEC27F08F6B8390839E090EA8
:1097280000019C6FFD0E9D6FCECF9EF09F6BCDCF3D
:10973800A0F0A16B0AEF60F0FBC120F071D08FECB4
:109748005FF0206EFB1979E0290E1F6E960E1E6ED3
:109758007F0EE82EFED71E2EFCD71F2EFAD700F05C
:109768006CD0F3EC5BF0216E215067E021B0522AF7
:1097780021B252060F0E5216000E0B6EC00ECBEC25
:109788005BF019EC5FF0000E0B6EC00ECBEC5BF0DB
:1097980052500F0D350EF3240F6E0D0EF420106E7F
:1097A8004AEC57F0110E1F6E3C0E1E6ECB0EE82EC3
:1097B800FED71E2EFCD71F2EFAD700F021A43DD0CD
:1097C8000C6A0B6A52C00DF074EC5DF0960E000145
:1097D8009C6FFC0E9D6F52C09EF09F6B0AEC60F070
:1097E80052C020F0000E0B6E800ECBEC5BF019EC33
:1097F8005FF0000E0B6E800ECBEC5BF052500F0D3D
:10980800350EF3240F6E0D0EF420106E4AEC57F04F
:10981800000E0B6EC00ECBEC5BF019EC5FF00DD0B8
:10982800010196511E6E1F6A1F5007E11E50010A62
:1098380086E0030A84E0010A94E02050120037C051
:1098480024F038C025F058EC43F0000901E0010C81
:1098580037C00BF038C00CF039C00DF03AC00EF02C
:109868003BC00FF03CC010F091EC4AF00BC041F047
:109878000CC042F00DC043F00EC044F020EE2BF0B7
:109888003750D9263850DA2241C0DEFF42C0DEFF09
:1098980043C0DEFF44C0DEFF2F0E37240B6E000EE0
:1098A80038200C6E0E6A0D6A020E106E0F6A7CEC80
:1098B8005FF02F0E37243F6E000E3820406E466A48
:1098C800010E456E476A486A04D0455047264650FF
:1098D800482220EE09F03750D9263850DA22DE50D7
:1098E800475CDE5048581FE23FC01AF040C01BF0EA
:1098F800475041241C6E485042201D6E000E4320E4
:109908001E6E000E44201F6E45C020F046C021F098
:1099180020EE01F03750D9263850DA22DF5004EC17
:109928004FF00009D2E020EE09F03750D926385020
:10993800DA224750DE1803E14850DE18D8A4010C9B
:10994800000C1F6A206A186A196A01D0122A010ECF
:109958001E6E1250D96EDA6A200EDE1813E0F70E6A
:10996800146E15681250D96EDA6ADF50166E176ACF
:109978001450162615501722175003E1050E165CD1
:1099880001E31E6A1EC01AF01B6A1A501B1006E07B
:10999800DDD7196A010E186E122A25D01250D96E19
:1099A800DA6ADF50146E156A15501DE114502B0A3F
:1099B800F3E0060AEEE017D00A0E1F02F3CF14F008
:1099C800F4CF15F02002F35015261250D96EDA6A3A
:1099D800DF50145E000E155A300E14241F6E000E50
:1099E8001520206ED9D7D00E146E15681250D96E76
:1099F800DA6ADF50166E176A1450162615501722A9
:109A0800175005E10A0E165C02E2010E01D0000EA5
:109A18001C6E1D6A1C501D10CFE1185019100DE165
:109A28001FC014F020C015F0141E151E144A152A64
:109A380014C012F015C013F012001FC012F020C09D
:109A480013F0120020EE03F04250D9264350DA22D8
:109A5800DF6A20EE2BF04250D9264350DA22DE6826
:109A6800DE68DE68DD6842C037F043C038F044C0C5
:109A780039F045C03AF046C03BF047C03CF039ECFD
:109A880054F0000904E0436A040E426E040C2D0EE3
:109A980042240B6E020E43200C6E1AEC5EF0550E3B
:109AA8000B1803E1AA0E0C1804E0436A030E426E79
:109AB800030C20EE2FF04250D9264350DA22E90E4B
:109AC800DE1812E020EE2FF04250D9264350DA2259
:109AD800EB0EDE1809E020EE2FF04250D926435055
:109AE800DA22E80EDE1827E1650E42240B6E000E1E
:109AF80043200C6ED00E0D6EFF0E0E6E106A030E14
:109B08000F6E16EC59F00B500C1003E1426A436AD1
:109B18001200810E42240B6E000E43200C6E8A0E3A
:109B28000D6EFF0E0E6E106A050E0F6E16EC59F0D4
:109B38000B500C10EBE0436A020E426E020C2C6EC6
:109B4800E50E00019C6FFC0E9D6F2CC09EF09F6B74
:109B580028C0A0F029C0A1F00AEC60F05DD0EAECC2
:109B680053F01EC02DF01FC02EF020C02FF021C0D2
:109B780030F028C0D9FF29C0DAFFDF6A20EE01F0F3
:109B88002850D9262950DA2230C0DFFF20EE02F013
:109B98002850D9262950DA22DF6A20EE03F028500F
:109BA800D9262950DA222FC0DFFF20EE04F02850F2
:109BB800D9262950DA22DF6A20EE05F02850D92666
:109BC8002950DA222EC0DFFF20EE06F02850D926D1
:109BD8002950DA22DF6A20EE07F02850D9262950CA
:109BE800DA222DC0DFFF1200EAEC53F01EC02DF080
:109BF8001FC02EF020C02FF021C030F028C018F070
:109C080029C019F02DC01AF02EC01BF02FC01CF06F
:109C180030C01DF0E7EF48F02C502A6E2B6A2B500D
:109C2800D8A412002A50010A9AE0030ADDE01200C3
:109C38000001F86B8380838E6AD0C2EC57F01EC097
:109C4800F6F01FC0F7F0040E0001F75D03E3010E04
:109C5800F86F03D0FBC0F9F0FA6B8FB414D05050F2
:109C6800220D000EF324956F030EF420966F000E5C
:109C7800976F040E986F010E9A6F996BF90E9B6F90
:109C8800C9EC08F0FB6FFB5109E07F0E9C6FFD0EDD
:109C98009D6FFBC09EF09F6B0AEC60F00101945130
:109CA80033E070517111721173112EE050500C0D88
:109CB800630EF324D96E020EF420DA6E70C1A3F19C
:109CC80071C1A4F172C1A5F1A26B000EA225A66F05
:109CD800010EA321A76F000EA421A86F000EA521D5
:109CE800A96FDE50A61910E1DE50A7190DE1DE506C
:109CF800A8190AE1DE50A91907E1000E226E040E28
:109D0800236E9451F5EC55F00BEC27F08F6B0001A6
:109D1800F85193E0839E839012000F015969116BEB
:109D2800196B216B8C948C928C90889A110E106E02
:109D38003C0E0F6ECB0EE82EFED70F2EFCD7102E42
:109D4800FAD700F0110E106E3C0E0F6ECB0EE82EF7
:109D5800FED70F2EFCD7102EFAD700F0020E106E89
:109D6800A00E0F6E920EE82EFED70F2EFCD7102EE7
:109D7800FAD700D0000E0B6E300ECBEC5BF02A0E3B
:109D88000F6E8E0EE82EFED70F2EFCD7000E0B6E30
:109D9800300ECBEC5BF0000E0B6E300ECBEC5BF0B4
:109DA800000E0B6E390ECBEC5BF0000E0B6E140E32
:109DB800CBEC5BF0000E0B6E560ECBEC5BF0000E9E
:109DC8000B6E6D0ECBEC5BF0000E0B6E700ECBECD9
:109DD8005BF0000E0B6E0C0ECBEC5BF0000E0B6E06
:109DE800060ECBEC5BF0000E0B6E010ECBEC5BF0BD
:109DF800D00E0F6ECA0EE82EFED70F2EFCD712001B
:109E0800236E2350D8A4040C2050211001E1040C27
:109E180054B0030C54B4020C51B608D0090ED890B3
:109E28001C361D361E361F36E82EF9D720042110A1
:109E38001AE11CC014F01DC015F01EC016F01FC09A
:109E480017F0180EADEC5DF0000945E11AC00DF0F1
:109E58001BC00EF0FE0E0F6ED4EC5AF000093BE06A
:109E6800206A216A38D051C022F0060E221609E075
:109E780020C014F021C015F0166A176A970EADECD1
:109E88005DF01CC014F01DC015F01EC016F01FC0F8
:109E980017F0190EADEC5DF000091DE11AC00DF0C8
:109EA8001BC00EF0FC0E0F6ED4EC5AF0000908E04F
:109EB800020E1B262006D8A0210620502110EEE114
:109EC8000D6A0E6AFD0E0F6ED4EC5AF0000903E11C
:109ED800216A010E206E3FEC60F020502110D8A4BA
:109EE800010C000CB3C0D9FFB4C0DAFFDECFBAF062
:109EF800DDCFBBF0B3C074F0B4C075F0000E766F60
:109F0800776F786F796FB1EC31F0BE6FBE5153E166
:109F1800BC6BBD6BBAC037F0BBC038F020EE16F092
:109F2800B351D926B451DA22DECF39F0DECF3AF078
:109F3800DECF3BF0DECF3CF039EC54F00001BE6FD1
:109F4800BE5139E120EE1AF0B351D926B451DA22C4
:109F5800DECFB7F0DDCFB8F0B7C0D9FFB8C0DAFFB1
:109F6800E50EDE1810E020EE1AF0B351D926B451F0
:109F7800DA22DECFB7F0DDCFB8F0B7C0D9FFB8C06E
:109F8800DAFFDF5009E1BC4BBD2BB551BC1906E126
:109F9800B651BD1910E002D0BC6BBD6BB3C095F0D3
:109FA800B4C096F0986B010E976F6EEC2EF000011E
:109FB800BE6FBE51AFE0040EBE1902E1070EBE6FC0
:109FC800BE511200838E83800001D16BD26BD36B9C
:109FD800D46B5050220D000EF324746F030EF4203E
:109FE800756F350E766F0B0E776F010E796F786B84
:109FF800D50E7A6F7B6BBFEC17F0D06F01019451CF
:10A0080035E0705171117211731130E050500C0D20
:10A01800630EF324D96E020EF420DA6E70C1C7F015
:10A0280071C1C8F072C1C9F00001C66B000EC62527
:10A03800CA6F010EC721CB6F000EC821CC6F000E6E
:10A04800C921CD6FDE50CA1911E1DE50CB190EE1DE
:10A05800DE50CC190BE1DE50CD1908E1350E286E23
:10A068000B0E296E01019451A3EC4DF00101FC93F4
:10A07800D5C01EF0D6C01FF0B8EC35F01EC0CEF02B
:10A088001FC0CFF00001CE51D127CF51D223000EEF
:10A09800D323D42301018F6B839E83901200818E7A
:10A0A800819C580EF66E8E0EF76E000EF86E0DEE51
:10A0B80035F011EE2CF00900F5CFEEFFE550E15038
:10A0C800FAE1E250F8E1360EF66EB40EF76E000EC5
:10A0D800F86E02EE00F010EE5FF00900F5CFEEFF2B
:10A0E800E550E150FAE1A00EF66EC00EF76E000ED4
:10A0F800F86E0900F5CFFEF10900F5CFFFF1A40EC7
:10A10800F66EC00EF76E000EF86E0900F5CF54F02B
:10A1180005EE00F018EE35F0EE6AE550E150FCE18E
:10A12800E250FAE104EE00F011EE00F0EE6AE550BC
:10A13800E150FCE1E250FAE103EE00F0AA0EEE6A0B
:10A14800E806FDE102EE5FF05A0EEE6AE806FDE170
:10A1580001EE00F09E0EEE6AE806FDE100EE4BF01F
:10A16800090EEE6AE806FDE155905592000EF86E6C
:10A1780000011CEF0FF00101906B4D6A806B816B41
:10A18800020E8F6F83908E6B8D6B506A030E506436
:10A1980001D049D050500C0D620EF324D96E020E36
:10A1A800F420DA6EDF6A50500C0D610EF324D96E7C
:10A1B800020EF420DA6EDF6A50500C0D5F0EF324A5
:10A1C800D96E020EF420DA6EDE6ADD6A50500C0D8C
:10A1D800630EF324D96E020EF420DA6EDE6ADE6AAC
:10A1E800DE6ADD6A50500C0D6A0EF324D96E020E39
:10A1F800F420DA6E100EDF6E50500C0D690EF32449
:10A20800D96E020EF420DA6E020EDF6E50500C0D7D
:10A21800670EF324D96E020EF420DA6E240EDE6E79
:10A22800DD6A502AB3D7100E02016A6F020E696FF9
:10A23800686B240E676F506A01018C6B12005050D6
:10A248001C0D070EF324D96E010EF420DA6E000EF1
:10A25800DE24BE6F010EDE20BF6F000EDE20C06F51
:10A26800000EDE20C16F000EDE20C26F000EDE2061
:10A27800C36F000EDE20C46F000EDE20C56F505085
:10A288001C0D070EF324D96E010EF420DA6EBEC041
:10A29800DEFFBFC0DEFFC0C0DEFFC1C0DEFFC2C040
:10A2A800DEFFC3C0DEFFC4C0DEFFC5C0DEFF505006
:10A2B8001C0D070EF324D96E010EF420DA6EDECFE2
:10A2C800C6F0DECFC7F0DECFC8F0DECFC9F0505001
:10A2D800220D000EF324956F030EF420966FC6C06E
:10A2E80097F0C7C098F0C8C099F0C9C09AF029EC97
:10A2F80012F0CA6FCA5103E0010E4E6E010C4E6A8D
:10A308001200BFC0D9FFC0C0DAFFDECFC1F0DDCF79
:10A31800C2F0BFC0B3F0C0C0B4F0000EB66F010EFB
:10A32800B56F76EC4FF0C36FC35147E1C1C037F04A
:10A33800C2C038F020EE16F0BF51D926C051DA223B
:10A34800DECF39F0DECF3AF0DECF3BF0DECF3CF0A7
:10A3580039EC54F00001C36FC3512FE120EE1AF01D
:10A36800BF51D926C051DA22DECF0BF0DDCF0CF079
:10A378000E6A0D6A106A200E0F6E7CEC5FF0000109
:10A3880020EE1AF0BF51D926C051DA22DECF0BF0E9
:10A39800DDCF0CF01C0EBF250D6E000EC0210E6E19
:10A3A800106A0B0E0F6E7CEC5CF020EE03F0C151CE
:10A3B800D926C251DA22010EDF6EC3511200838002
:10A3C800838E000E0B6E040E0C6E0E6AF60E0D6E6A
:10A3D800010E106E0F6AC2EC47F0570E00019C6F19
:10A3E800FE0E9D6F0AEC60F0C66BC76BC6C0C2F06C
:10A3F800010EC217C233C2338350C2197F0BC21970
:10A40800836E2E0EFFEC5FF08FB415D05050220DE6
:10A41800000EF3240001956F030EF420966F000ED2
:10A42800976F040E986F010E9A6F996BC30E9B6F0E
:10A43800C9EC08F0C56F0001C55109E0680E9C6FB2
:10A44800FF0E9D6FC5C09EF09F6B0AEF60F0C64B74
:10A45800C72BC7BFCBD7C75103E1640EC65DC6E3A0
:10A468002C0E9C6FFF0E9D6F0AEC60F0839E83900C
:10A4780083904E6A1200FC83505028E1350E0B6E13
:10A488000B0E0C6E550E0D6E020E0E6E106A050E3A
:10A498000F6E3AEC5CF03A0E0B6E0B0E0C6E000E63
:10A4A8000D6E020E0E6E106A130E0F6E3AEC5CF013
:10A4B8004D0E0B6E0B0E0C6E260E0D6E020E0E6EF2
:10A4C800106A0D0E0F6E3AEC5CF027D0350E0B6E4D
:10A4D8000B0E0C6E5A0E0D6E020E0E6E106A050EE5
:10A4E8000F6E3AEC5CF03A0E0B6E0B0E0C6E130E00
:10A4F8000D6E020E0E6E106A130E0F6E3AEC5CF0C3
:10A508004D0E0B6E0B0E0C6E330E0D6E020E0E6E94
:10A51800106A0D0E0F6E3AEC5CF01F6A250E1E6E67
:10A52800B8EC35F00101FC9383901200090E156E0A
:10A538000C500D103BE00CC0D9FF0DC0DAFFDE5007
:10A54800DE1034E00CC0D9FF0DC0DAFFDECF0FF00B
:10A55800DDCF10F00FC0D9FF10C0DAFFDF5026E0C2
:10A568000CC0D9FF0DC0DAFF10EE05F0DE50E12671
:10A57800DD50E22220EE02F00C50D9260D50DA22EE
:10A58800E650DE1813E1E650DE1810E10CC0D9FFE2
:10A598000DC0DAFF10EE01F0DE50E126DD50E222B8
:10A5A800E75035EC60F00F6E0FA0156A155003E008
:10A5B800136A146A08D00CC0D9FF0DC0DAFFDECFC9
:10A5C80013F0DDCF14F00E50D96EDA6A13C0DEFF37
:10A5D80014C0DDFF1550120050501C0D070EF32457
:10A5E800D96E010EF420DA6EDECFE7F0DECFE8F0A8
:10A5F800DECFE9F0DECFEAF0DECFEBF0DECFECF035
:10A60800DECFEDF0DECFEEF0E8C0E7F0E9C0E8F02D
:10A61800EAC0E9F0EBC0EAF0ECC0EBF0EDC0ECF01A
:10A62800EEC0EDF00001EE6BE7C0EFF0E8C0F0F02F
:10A63800E9C0F1F0EAC0F2F0E3EC39F0F56FF5515A
:10A6480002E0F55112008FB414D05050220D000EC4
:10A65800F324956F030EF420966F000E976F040E87
:10A66800986F010E9A6F996BF30E9B6FC9EC08F007
:10A67800F66FF65102E0F651120023EC51F0000C8F
:10A6880020EE03F00B50D9260C50DA22DF50136E5F
:10A69800146A156A166A20EE02F00B50D9260C507F
:10A6A800DA22DF5013C010F014C011F015C012F0F8
:10A6B8000F6A0F10136E1050146E1150156E125051
:10A6C800166E20EE01F00B50D9260C50DA22DF501E
:10A6D80013C010F014C011F015C012F00F6A0F105B
:10A6E800136E1050146E1150156E1250166E0BC06A
:10A6F800D9FF0CC0DAFFDF5013C010F014C011F0FE
:10A7080015C012F00F6A0F10136E1050146E11500E
:10A71800156E1250166E13C00BF014C00CF015C055
:10A728000DF016C00EF01200226E2250D8A4040CB0
:10A738002050211001E1040C54B0030C51B608D08C
:10A74800090ED8901C361D361E361F36E82EF9D74E
:10A75800215006E1020E205C03E2246A110E02D0A9
:10A76800246A120E236E23C025F01CC014F01DC0ED
:10A7780015F01EC016F01FC017F02550ADEC5DF0A7
:10A7880000091DE11AC00BF01BC00CF0020E0E6E82
:10A798000D6A7AEC5AF0000908E0020E1B26200622
:10A7A800D8A0210620502110EDE1120E251807E14E
:10A7B800146A156A166A176A0C0EADEC5DF03FEC68
:10A7C80060F020502110D8A4010C000CC9EC5DF0F9
:10A7D800CC0ECFEC5FF0660ECFEC5FF0B2EC5FF022
:10A7E800246E245005E11E6A1F6A206A216A12003D
:10A7F800226A236A2250240FD96EDA6AB2EC5FF01B
:10A80800DF6E224A232A23BEF5D7235003E1040E24
:10A81800225CF0E3810E00019C6FFC0E9D6F24C04A
:10A828009EF09F6B25C0A0F0A16B26C0A2F0A36B81
:10A8380027C0A4F0A56B24C0A6F025C0A7F026C0A9
:10A84800A8F027C0A9F00AEC60F0275026102510C0
:10A8580003E1060E245CC7E324C01EF025C01FF0E8
:10A8680026C020F027C021F01200416A20EE2BF00C
:10A878003750D9263850DA223950DE1809E13A50D3
:10A88800DE1806E13B50DE1803E13C50DE1839E0E3
:10A8980037C024F038C025F058EC43F0416E4150E1
:10A8A80030E12F0E37241A6E000E38201B6E39C087
:10A8B8001CF03AC01DF03BC01EF03CC01FF0216ADE
:10A8C800010E206E20EE01F03750D9263850DA22DA
:10A8D800DF5098EC53F0000906E039683A683B68A5
:10A8E8003C68010E416E20EE2BF03750D9263850C7
:10A8F800DA2239C0DEFF3AC0DEFF3BC0DEFF3CC0D3
:10A90800DEFF4150120003D00B4A0C2A0D2A0D50CD
:10A91800D96EDA6ADF500E6E0BC0F6FF0CC0F7FF77
:10A92800000EF86E0E0EF76403D00800F55005D03F
:10A93800F6CFE9FFF7CFEAFFEF500E1813E10BC08F
:10A94800F6FF0CC0F7FF000EF86E0E0EF76403D08A
:10A958000800F55005D0F6CFE9FFF7CFEAFFEF5032
:10A968000009D2E10BC0F6FF0CC0F7FF000EF86E2D
:10A978000E0EF76403D00800F55005D0F6CFE9FFB6
:10A98800F7CFEAFFEF500E6E0D50D96EDA6ADF503E
:10A998000E5C0B6E0C6AD8A00C0612001450151031
:10A9A8000AE178C114F079C115F01450151003E1CB
:10A9B800146A156A120014C00FF015C010F016C002
:10A9C80011F09DEC5CF00F5014261050152214C0A5
:10A9D800D9FF15C0DAFFDF5006E10101786B796B0A
:10A9E800146A156A120014C00FF015C010F016C0D2
:10A9F80011F0BDEC5CF00F5014240101786F105079
:10AA08001520796F78C1D9FF79C1DAFFDF5009E0E5
:10AA180078C1D9FF79C1DAFF000EDF6A784B792B4C
:10AA280002D0786B796B14C014F015C015F01200C1
:10AA3800A96BAA6B9FC0ABF0A0C0ACF0A107D8A0CF
:10AA4800A20727D0A3C074F0A4C075F0A50E766F36
:10AA5800776B796B010E786FB10E7A6F7B6BBFECF9
:10AA680017F0B105B2111EE1A551AD6FAE6BAF6B1A
:10AA7800B06BABC0D9FFACC0DAFFADC0DFFFAB4BEA
:10AA8800AC2BA94BAA2B0A0EAD19AE11AF11B01100
:10AA980009E0A151A95DAA51800A486EA251800A15
:10AAA8004858D0E3ABC0D9FFACC0DAFFDF6AA95180
:10AAB800AA1103E19F6BA06B12009FC09FF0A0C07A
:10AAC800A0F01200B3C0B7F0B4C0B8F0B70E0B6E68
:10AAD800F8EC45F00BC0BBF00CC0BCF00001BCBFEB
:10AAE8000B0CD890BB35D96EBC35DA6E860ED926DC
:10AAF800010EDA22DECFB9F0DDCFBAF0B951BA11C2
:10AB080005E0B9C0D9FFBAC0DAFFDF6AB151B211A6
:10AB180005E0B1C0D9FFB2C0DAFFDF6AD890BB3513
:10AB2800D96EBC35DA6E860ED926010EDA22B1C08E
:10AB3800DEFFB2C0DDFFB55101E1000CB30E7C6F42
:10AB4800B10E7D6F7E6B7F6BAFEC00F00001B66FCE
:10AB5800B65112000BC012F00CC013F00DC014F067
:10AB68000EC015F00F06D8A010060F280CE110280B
:10AB78000AE10B6A0C6A1200124A132A144A152AAF
:10AB88000F06D8A0100612C0F6FF13C0F7FF080082
:10AB9800F55015E014C0D9FF15C0DAFFDF500FE0FB
:10ABA8000F5010100CE014C0D9FF15C0DAFF12C006
:10ABB800F6FF13C0F7FFDE500900F518DDE012C0FC
:10ABC800F6FF13C0F7FF0800F5CF11F014C0D9FF46
:10ABD80015C0DAFFDF50115C0B6E0C6AD8A00C06AA
:10ABE8001200266E39D020EE01F02250D9262350CB
:10ABF800DA22DF502A6E20EE03F02250D9262350A5
:10AC0800DA22DF50296E20EE05F02250D926235093
:10AC1800DA22DF50286E20EE07F02250D926235082
:10AC2800DA22DF50276E27C00EF028C00FF029C0A7
:10AC380010F02AC011F028EF5BF022C00BF023C0FF
:10AC48000CF0BEEC3BF00BC027F00CC028F00DC098
:10AC580029F00EC02AF0E7D72650246E256A255021
:10AC6800D8A412002450010ABEE0030AE6E012004C
:10AC780025EE04F0DE50DE10FBE000C513F001C540
:10AC880014F0060E1324D96E050E1420DA6EDF5068
:10AC9800116E060E1324D96E070E1420DA6EDF50DB
:10ACA800126E134A142A0D68010E0E6E13C00FF0AF
:10ACB80014C010F00D500F160E5010160FC000F5EE
:10ACC80010C001F5F29E25EE04F0DE06000EDD5AF6
:10ACD800F28E0BC0D9FF0CC0DAFF12C0DFFF25EEE1
:10ACE80004F0010EDBBE05D0000EDE5C020EDE585D
:10ACF80001E28982115012000E5002E00E5003E169
:10AD08000C50F4EF5FF00E50D96EDA6A040ED926B3
:10AD1800DE50DE1014E00E50D96EDA6A040ED92621
:10AD28000E50E16EE26A020EE126DE50E65CE65065
:10AD3800800A136EDE50800A1358D8B012000E50E5
:10AD4800D96EDA6A020ED926DECF0FF0DDCF10F009
:10AD58000E50D96EDA6ADECF11F0DDCF12F00F5047
:10AD68001124D96E10501220DA6E0CC0DFFF0E507D
:10AD7800D96EDA6A020ED926DE2A000EDD22000C10
:10AD8800EE0E00019C6FFD0E9D6F82C19EF083C187
:10AD98009FF00AEC60F011D0030E0BD0050E206E68
:10ADA8000101826B836B2DD00A0E03D0010E01D0F6
:10ADB800020E206E26D0206A24D082C11EF083C1E4
:10ADC8001FF01F5009E0020A0DE00E0A0FE0010A09
:10ADD80011E02A0A13E0EFD71E500A0ADDE01E0A26
:10ADE800DDE0E9D71E50BC0AE3E0E5D71E501C0A97
:10ADF800DBE0E1D71E50AC0AD9E0DDD71E500F0AC0
:10AE0800DAE1205012000B500F02F3CF13F0F4CF09
:10AE180014F0156A166A0B501002F3501426F450F9
:10AE28001522000E16220C500F02F3501426F4506F
:10AE38001522000E16220B501102F3501526F4505D
:10AE480016220C501002F3501526F45016220D50FD
:10AE58000F02F3501526F450162212500B02F3502D
:10AE680016260C501102F35016260D501002F350FE
:10AE780016260E500F02F350162613C00BF014C0FE
:10AE88000CF015C00DF016C00EF01200150E116E64
:10AE9800C60EE82EFED7112EFCD700D020D0150EF6
:10AEA800116EC60EE82EFED7112EFCD700D0010E6B
:10AEB8000B6E0FC0F6FF10C0F7FF000EF86E0E0EF7
:10AEC800F76403D00800F55005D0F6CFE9FFF7CFB7
:10AED800EAFFEF50CBEC5BF00F4A102AD7D70FC030
:10AEE800F6FF10C0F7FF000EF86E0E0EF76403D0E1
:10AEF8000800F55005D0F6CFE9FFF7CFEAFFEF508D
:10AF08000009CDE11200136A146A156A166A0F5017
:10AF180010101110121029E0010E176E06D0D890EB
:10AF28000F36103611361236172A12AEF8D7D890C7
:10AF380013361436153616360F500B5C10500C5855
:10AF480011500D5812500E5809E30F500B5E105057
:10AF58000C5A11500D5A12500E5A1380D8901232B2
:10AF6800113210320F32172EE2D713C00BF014C073
:10AF78000CF015C00DF016C00EF01200216A226AFE
:10AF8800536A236A2ED0A2EC5FF00B500C101EE01F
:10AF9800230E0B6E0C6A3CEC56F0206E23A80BD0E7
:10AFA8000C0E00019C6FFF0E9D6F20C09EF09F6BE2
:10AFB8000AEC60F00BD0000E5324D96EDA6A040E46
:10AFC800DA2220C0DFFF532A214A222A23AA07D0E7
:10AFD800000E21241E6E040E22201F6E12008EAC5D
:10AFE80002D02204D0E321C01EF022C01FF01200BC
:10AFF8001A0E14240B6E000E15200C6E1AEC5EF05F
:10B008000BC01AF00CC01BF01C6A1D6A12C0D9FFD5
:10B0180013C0DAFF030EDE181CE1140E14240B6EA5
:10B02800000E15200C6E1AEC5EF00B50166E0C50CC
:10B03800176E186A196A17C019F016C018F0176A3F
:10B04800166A16501A1217501B1218501C12195053
:10B058001D121AC012F01BC013F01CC014F01DC042
:10B0680015F01200136E0C0E131807E03FEC60F099
:10B07800DCEC5FF0000901E1FF0C135040091DEC06
:10B0880060F010501DEC60F00F501DEC60F00E5099
:10B098001DEC60F00D501DEC60F0010E126E1350A7
:10B0A80002E1950E126E080E131802E1870E126E59
:10B0B80012501DEC60F00C0E131802E12EEC60F03B
:10B0C8000A0E126E2EEC60F0116E11AE02D0122E26
:10B0D800F9D7115012000F501010D8B4000C0FC03F
:10B0E800D9FF10C0DAFFDF5001E1000C0FC00BF0F0
:10B0F80010C00CF05BEC5CF00BC011F00CC012F04F
:10B10800020E1118121001E0000C130E0B6E0FC086
:10B11800D9FF10C0DAFFDF5051EC5BF00009D8B45A
:10B12800000C140E0B6E20EE01F00F50D9261050B3
:10B13800DA22DF5051EC5BF0000901E1000C133812
:10B14800F00B141012000D6E830EF66EF90EF76EEA
:10B158000900F5500D5C2CE3840EF66EF90EF76EBF
:10B168000D500900F55C04E30C6A010E0B6E010C2E
:10B17800850EF66EF90EF76E0900F5500D5C08E3C2
:10B18800860EF66EF90EF76E0D500900F55CECE2CE
:10B19800870EF66EF90EF76E0900F5500D5C08E3A0
:10B1A800880EF66EF90EF76E0D500900F55CDCE2BC
:10B1B8000B6A0C6A1200866A846A8B688968536A0B
:10B1C8008392839401018A6B8B6B09D0000E8A25C8
:10B1D800D96E040E8B21DA6EDF6A8A4B8B2B8BBFFC
:10B1E800F5D78B05F3E38A6B8B6B09D0350E8A256F
:10B1F800D96E0B0E8B21DA6EDF6A8A4B8B2B8BBFD5
:10B20800F5D78B05F3E30F011769D6501F0B4009DB
:10B21800D66ED6980F0ED612D588D5120E01C29BBF
:10B22800D58E0F0C0BC012F00CC013F00DC014F02B
:10B238000EC015F012C0D9FF13C0DAFFDF50116E2F
:10B2480014C0F6FF15C0F7FF000EF86E0E0EF76477
:10B2580003D00800F55005D0F6CFE9FFF7CFEAFF95
:10B26800EF50115C166E176AD8A01706144A152AF3
:10B27800124A132A0F06D8A010060F50101003E028
:10B2880016501710D7E016C00BF017C00CF01200BC
:10B298000BC0D9FF0CC0DAFF0DC0DFFF0B4A0C2A28
:10B2A8000E500D6E0F500E6E10500F6E106A0BC0C0
:10B2B800D9FF0CC0DAFF0DC0DFFF0B4A0C2A0E5075
:10B2C8000D6E0F500E6E10500F6E106A0BC0D9FF26
:10B2D8000CC0DAFF0DC0DFFF0B4A0C2A0E500D6EB2
:10B2E8000F500E6E10500F6E106A0BC0D9FF0CC0B5
:10B2F800DAFF0DC0DFFF0B4A0C2A12008380FC83A3
:10B308008C050DE1000EE8CF35FB500EE8CF36FB7B
:10B31800000EE8CF37FBE8CF38FB8C6B1AD02BEE4A
:10B3280035F08DC1DFFF000EE8CF36FB0D0EE8CFFC
:10B3380037FB000EE8CF38FB8FA403D0600EE8CFB0
:10B3480038FB8FA406D037CB24F0200E241224C05B
:10B3580037FB1F6A040E1E6EB8EC35F00101FC9332
:10B368008D6B83901200506A030E506401D02AD06E
:10B3780050500C0D620EF324D96E020EF420DA6ED2
:10B38800DF6A50500C0D610EF324D96E020EF420C2
:10B39800DA6EDF6A50500C0D5F0EF324D96E020E80
:10B3A800F420DA6EDE6ADD6A50500C0D630EF32469
:10B3B800D96E020EF420DA6EDE6ADE6ADE6ADD6AB3
:10B3C800502AD2D7506A83908F6B12000F501010FA
:10B3D8001110121023E0010E136E06D0D8900F360C
:10B3E800103611361236132A12AEF8D70F500B5CEE
:10B3F80010500C5811500D5812500E5808E30F50A9
:10B408000B5E10500C5A11500D5A12500E5AD8900B
:10B418001232113210320F32132EE8D70BC00BF054
:10B428000CC00CF00DC00DF00EC00EF0120001099A
:10B438001220010001001700002D119420D00F00E8
:10B448000101091220010001001700002D119420AC
:10B45800D00F000100004F01000F0000000009FF9D
:10B468000000004F01000F0000000009FF00687095
:10B478006469736B2E636667004850393132314412
:0DB48800000000800102E805800102E805D7
:10B496000B6A0C6A50501C0D070EF324D96E010E70
:10B4A600F420DA6E070EDE6AE806FDE250501C0D47
:10B4B6001B0EF324D96E010EF420DA6EDF6A5050AB
:10B4C6001C0D170EF324D96E010EF420DA6EDE6A17
:10B4D600DE6ADE6ADD6A0B4A0C2A0CBEDBD70C502C
:10B4E60003E1040E0B5CD6E383904E6A1200070E4E
:10B4F600106ED00E0F6E0FD02EEC60F0116E11286C
:10B506000DE1E40E00D000D0E82EFCD700D000D02C
:10B516000F06D8A010060F501010EEE1FE0E1118FF
:10B5260001E0000C2EEC60F00BC0D9FF0CC0DAFF76
:10B53600DF6E0B4A0C2A0D06D8A00E060D500E1013
:10B54600F1E12EEC60F02EEC60F0010C0BC011F076
:10B556000CC012F013D00F06D8A010060DC0D9FFEC
:10B566000EC0DAFF0D4A0E2A11C0E1FF12C0E2FF3B
:10B57600114A122ADFCFE7FFE7500BE00F501010F9
:10B5860008E0E9D711C0D9FF12C0DAFFDF6A114A15
:10B59600122A0F06D8A010060F28F4E11028F2E1AF
:10B5A6001200E4EC5DF0000901E1000C0F501DEC07
:10B5B60060F0FD0E0F181EE0020E116E106A0DC02F
:10B5C600D9FF0EC0DAFFDF501DEC60F00D4A0E2ADF
:10B5D6001006D8A0110610501110F1E12EEC60F003
:10B5E6002EEC60F02EEC60F0126E12501F0B050A66
:10B5F60001E0000C010C15D00CC0F6FF0DC0F7FFE2
:10B60600000EF86E0E0EF76403D00800F55005D054
:10B61600F6CFE9FFF7CFEAFFEF50FFEC5FF00C4AF9
:10B626000D2A0CC0F6FF0DC0F7FF000EF86E0E0EC9
:10B63600F76403D00800F55005D0F6CFE9FFF7CF41
:10B64600EAFFEF500009D8E112000EC012F00FC059
:10B6560013F010C014F011C015F0C9EC5DF0CC0E5B
:10B66600CFEC5FF0990ECFEC5FF00C0ECFEC5FF0F5
:10B67600166A176A1650120FD96EDA6ADF50CFECC7
:10B686005FF0164A172A17BEF5D7175002E0C9EF22
:10B696005DF0040E165CEEE3C9EF5DF00C6E0B5028
:10B6A60001E1000C2F0E0C6409D03A0E0C6006D096
:10B6B6000B50D96EDA6A0C50D00F17D0400E0C64BE
:10B6C60009D0470E0C6006D00B50D96EDA6A0C50C2
:10B6D600C90F0BD0600E0C64000C670E0C60000CDA
:10B6E6000B50D96EDA6A0C50A90FDF6E010C1F6E73
:10B6F6008B0E206EF90E216E1E6A0AD020C0F6FF50
:10B7060021C0F7FF204A212A0800F550F7E11E2A3A
:10B716001F501E1807E020C0F6FF21C0F7FF0800E3
:10B72600F550ECE1650E00019C6FFE0E9D6F1FC08B
:10B736009EF09F6B20C0A0F021C0A1F00AEF60F040
:10B746000D6E7F0EF66EF90EF76E0900F5500D5C64
:10B756001CE3800EF66EF90EF76E0D500900F55CCF
:10B7660004E30C6A010E0B6E010C810EF66EF90EE7
:10B77600F76E0900F5500D5C08E3820EF66EF90EC1
:10B78600F76E0D500900F55CECE20B6A0C6A1200CC
:10B796000C6E87920A0EE82EFED700D00BB002D0B0
:10B7A600879401D08784000E0E6E010E0D6E0CAECE
:10B7B60002D0838A01D0839AD8900C36879000F005
:10B7C60000F0878000F000F087900D4A0E2A0EBE2A
:10B7D600EED70E5003E1090E0D5CE9E387821200F5
:10B7E600010E0B6E0C6A88868782878400F000F053
:10B7F600879400F000F00D6A0E6A8DA602D00B50F9
:10B806000C12D8900B36879000F000F0878000F07D
:10B8160000F087900D4A0E2A0EBEEFD70E5003E1B8
:10B82600030E0D5CEAE30C5012009F0E136E1468B3
:10B8360011C015F012C016F013501526145016221A
:10B84600165005E11A0E155C02E2010E01D0000E3B
:10B85600176E186A1750181005E05F0E1114116E56
:10B86600126A120011C011F012C012F012000DC0BF
:10B8760013F00EC014F00BC011F00CC012F010D073
:10B8860013C0D9FF14C0DAFFDF50156E134A142A0D
:10B8960011C0D9FF12C0DAFF15C0DFFF114A122A04
:10B8A6000F06D8A010060F28EBE11028E9E11200D8
:10B8B6000BC00DF00CC00EF002D00B4A0C2A0BC0C8
:10B8C600F6FF0CC0F7FF000EF86E0E0EF76403D0FD
:10B8D6000800F55005D0F6CFE9FFF7CFEAFFEF50A5
:10B8E6000009EBE10D500B5C0B6E0E500C580C6E04
:10B8F60012000BC011F00CC012F00DC013F00EC0F8
:10B9060014F00F501010D8B4120013C0D9FF14C091
:10B91600DAFF11C0E1FF12C0E2FFDFCFE7FF134AF3
:10B92600142A114A122A0F06D8A010060F5010101A
:10B93600ECE11200126A136A04D00F4A102A124A66
:10B94600132A0FC0D9FF10C0DAFFDF500EE011C076
:10B956000BF00FC0D9FF10C0DAFFDF500C6E0D6A76
:10B9660069EC5FF00B500C10E8E112C00FF013C049
:10B9760010F01200126A136A04D00F4A102A124AF3
:10B98600132A0FC0D9FF10C0DAFFDF500EE011C036
:10B996000BF00FC0D9FF10C0DAFFDF500C6E0D6A36
:10B9A60069EC5FF00B500C10E8E012C00FF013C00A
:10B9B60010F012001A0E11240B6E000E12200C6EDF
:10B9C60013C00DF014C00EF042EC5FF00FC0D9FFAB
:10B9D60010C0DAFF030EDE18D8A41200140E1124CC
:10B9E6000B6E000E12200C6E15C00DF016C00EF078
:10B9F60042EF5FF08F6B8380838E000E0B6E040E1A
:10BA06000C6E0E6AF60E0D6E010E106E0F6AC2EC0B
:10BA160047F0570E00019C6FFE0E9D6F0AEC60F01A
:10BA26002C0E9C6FFF0E9D6F0AEC60F0839E839038
:10BA360012000B6E0B500EE046EC60F0200EE82E66
:10BA4600FED749EC60F0CC0E00D0E82EFDD700D032
:10BA560000D0120046EC60F0C00E00D0E82EFDD7F4
:10BA660049EC60F0350EE82EFED700F0120048C013
:10BA760046F049C047F00BEC44F0736F735112E186
:10BA860048C00CF049C00DF0710E0E6E9AEC52F0E3
:10BA96000001736F735106E148C0D9FF49C0DAFF50
:10BAA600DE6ADD6A735112007D0E816F79C082F005
:10BAB6007AC083F0846B856B866B876B820E736F9F
:10BAC6007BC074F07CC075F0810E766F23EC05F0B8
:10BAD600000184517925D96E85517A21DA6EDF6AA3
:10BAE600000C000EF2BE010E0E6E0C50030B7F6EA4
:10BAF6000BC07EFF0DC080FF3F0E81168184F29E33
:10BB0600550E826EAA0E826E818281B2FED7819414
:10BB16000EB002D0F29E01D0F28E120002D00B4A75
:10BB26000C2A0BC0F6FF0CC0F7FF0800F55009E021
:10BB36000BC0F6FF0CC0F7FF0800F5500D180E10ED
:10BB4600EEE10BC0F6FF0CC0F7FF0800F5500B6ED8
:10BB56000C6A1200186E18AE0ED0189E0D6A0E6A88
:10BB66000F6A106A370E36EC58F0196E010E19641A
:10BB760002D01950120014C00DF015C00EF016C0F8
:10BB86000FF017C010F0185036EF58F046EC60F082
:10BB96000A0E0C6EF80EE82EFED70C2EFCD700D03F
:10BBA60049EC60F0E00E00D0E82EFDD714EC60F012
:10BBB600090E0C6E840EE82EFED70C2EFCD749EF2C
:10BBC60060F0130E0C6E880E0B6E0ED02EEC60F02D
:10BBD600FF0A0DE0E40E00D000D0E82EFCD700D01E
:10BBE60000D00B06D8A00C060B500C10EFE10B5042
:10BBF6000C10D8A4010C000C010E116E200E0B18AF
:10BC06000C1011E0F70E0D6E0E680BC00FF00CC095
:10BC160010F00D500F260E501022105003E1050EA5
:10BC26000F5C01E3116A11C00BF00C6A120020EEE2
:10BC360001F00B50D9260C50DA22DF50106E116A33
:10BC46000BC0D9FF0CC0DAFFDF500D6E10500E6E20
:10BC56000D50106E0EC011F010C00BF011C00CF09C
:10BC6600120060900F0E0F01596F070E396F356F76
:10BC76004F0E936E8A6A8A888A828A82010E8F6E36
:10BC8600130E0E01B76F0F0EFA6F100EFC6F140E27
:10BC9600B86F140C9F0E0D6E0E68200E0B100F6EF3
:10BCA600000E0C10106E0D500F260E501022105064
:10BCB60005E11A0E0F5C02E2010E01D0000E0B6EBA
:10BCC6000C6A12001EBE04D01E500FE11D040DE2C8
:10BCD6001DC01FF01EC020F01F1E201E1F4A202A56
:10BCE6001FC01DF020C01EF012001DC01DF01EC09A
:10BCF6001EF01200350E0B6E0B0E0C6E0E6A0D6AE0
:10BD0600010E106E0F6AC2EC47F02BEE35F08FC1B4
:10BD1600DFFF1F6A010E1E6EB8EC35F001018F6B56
:10BD26001200350E0B6E0B0E0C6E0E6A0D6A010EAE
:10BD3600106E0F6AC2EC47F0010EE8CF35FB010129
:10BD4600FC831F6A1E6EB8EC35F00101FC931200ED
:10BD5600186A196A09D017C00CF00D6A16C00EF0E1
:10BD660080EC56F0184A192A18501424D96E195026
:10BD76001520DA6EDF50176E1750EDE112009F0E98
:10BD86000D6E0E680BC00FF00CC010F00D500F2694
:10BD96000E501022105005E11A0E0F5C02E2010E41
:10BDA60001D0000E0B6E0C6A1200BF0E0D6E0E68EF
:10BDB6000BC00FF00CC010F00D500F260E501022C5
:10BDC600105005E11A0E0F5C02E2010E01D0000EC2
:10BDD6000B6E0C6A1200D00E0D6E0E680BC00FF0C3
:10BDE6000CC010F00D500F260E501022105005E119
:10BDF6000A0E0F5C02E2010E01D0000E0B6E0C6AF9
:10BE060012009F869E84090E0E01FD6F9F98890E73
:10BE16009B6E9C6A9E989D8E9D889D9AC599F28A76
:10BE2600F28E9E909D9C9E9A9E8A1200106A110E1A
:10BE36000F6E09D00A0EE82EFED700D0010E0B6E4B
:10BE4600200ECBEC5BF00F06D8A010060F28F2E10F
:10BE56001028F0E112000B6E0B5009E0966A4F0EA7
:10BE6600936E220E966E400E956E968A400C966ADA
:10BE7600100E966E2A0E966E900E936EF4D70BC029
:10BE8600D9FF0CC0DAFF0DC0DFFF0B4A0C2A0EC02B
:10BE96000DF00E6A0BC0D9FF0CC0DAFF0DC0DFFF34
:10BEA6000B4A0C2A120046EC60F0200EE82EFED754
:10BEB60049EC60F0300EE82EFED714EC60F00C6E04
:10BEC600B00E00D0E82EFDD70C5012000B50D96EE4
:10BED600DA6A0C50DE1804E10BC00BF00C6A120093
:10BEE6000B2A0B04D96EDA6ADF50F0E10B6A0C6A92
:10BEF60012000BC011F00CC012F011C0D9FF12C015
:10BF0600DAFF0DC0DFFF114A122A0F06D8A010066D
:10BF16000F501010F2E11200070E8C6E9150070BB5
:10BF26000B6E888A8DAA02D0080E0B26020E01011E
:10BF3600961903E10B1C0F0B0B6E0B50120025EE2E
:10BF460004F0010EDBBE05D0000EDE5C020EDE58EC
:10BF560001E2898204C50BF005C50CF012000D6ADA
:10BF66000E6AD8900D3256EC5FF0000901E00D8E96
:10BF76000E2A070E0E64F5D70D501200000EE8CFFC
:10BF860000F5E8CF01F5E8CF02F5E8CF03F5E8CFF5
:10BF960004F5E8CF05F5000C0C6E0D6A0C50010B8C
:10BFA6001CEC5DF0D8900C320D2A070E0D64F6D706
:10BFB600070C4EEC60F02EEC60F0E4EC5DF000094E
:10BFC60001E0010C3FEC60F0000C0C50030B7F6E9F
:10BFD6000BC07EFF3F0E8116818000F000F080507E
:10BFE60012000B6E03D051EC60F004000E01CDA9D7
:10BFF600FAD70BC09AFF12000B6E03D051EC60F01B
:10C0060004000E01CDA9FAD70BC09AFF12009E0EAE
:10C016001D6E9CC018F09DC019F01D0E1A6EFBEF28
:10C0260024F088888DA803D0010E0B6E01D00B6A10
:10C036000B5012000B6E0BC092FF95B0FED795A069
:10C04600FED7925012000B6E02D0838C839C0B0697
:10C056000B28FBE11200926895B0FED795A0FED79B
:10C06600925012000B6E0B5001E0010C545012005E
:10C0760083804E6A839012004CEC60F02EEF60F0E5
:10C0860083908F6B12008398889812008398888813
:0FC09600120085801200859012001FE712000132
:10F97E0000819FE0FC407E80FC000020004F4B0089
:10F98E004449534B5F455252004E4F545F524541CE
:10F99E004459004E4F5F46494C45004E4F545F4F01
:10F9AE0050454E4544004E4F545F454E41424C45E6
:10F9BE0044004E4F5F46494C455F53595354454D95
:10F9CE0000000D0A2025325820253258202532738A
:10F9DE002025327320253273202532732025327371
:10F9EE00202532732025327320253273202534735F
:10F9FE002025347320253473202534732025347349
:10FA0E0020253473202534732025347320000D0AED
:10FA1E0048504469736B204D6B204949202831387A
:10FA2E004634364B34302920257320257320257318
:10FA3E00205374617274696E672E2E2E0D0A000D9E
:10FA4E000A4461746120706F7274206973202558A6
:10FA5E00202D2053686F756C64206265203C3E201B
:10FA6E0030784646000D0A5365656B20657272202C
:10FA7E002564203E2025642C202564203E2025640C
:10FA8E002C202564203E202564000D0A53746174D9
:10FA9E00757320706F7274206973202558202D2085
:10FAAE0053686F756C642062652030784646000D91
:10FABE000A4461746120706F727420697320255836
:10FACE00202D2053686F756C642062652030784657
:10FADE0046000D0A526420752025642072746E2033
:10FAEE0025642C202564206279746573207265610B
:10FAFE00640D0A000D0A4D617820566563746F72AD
:10FB0E00206469736B20256420256C642028256C85
:10FB1E00582920000D0A25303258253032582053EE
:10FB2E00533830783A5374617475735B25645D2075
:10FB3E00255820000D0A44736B73656C2069732081
:10FB4E0025642C206E756D626572206973202564A4
:10FB5E002000466F756E6420616E205254432066FD
:10FB6E00696C652061742025580D0A004C6F6F6B0F
:10FB7E00696E6720666F7220616E20525443206654
:10FB8E00696C650D0A0046696E6446696C6520668F
:10FB9E0061696C6564207365617263680D0A000D9E
:10FBAE000A53746174757320706F727420697320B8
:10FBBE002558202D204F4B000D0A5365656B207480
:10FBCE006F20256C64206661696C65642025640075
:10FBDE000D0A454550524F4D206469736B206E756A
:10FBEE006D626572202564000D0A4469736B207383
:10FBFE00656C656374206E756D6265722025640098
:10FC0E005365656B696E6720746F20736563746FDF
:10FC1E00722025580D0A0046696E6446696C65208F
:10FC2E006661696C656420726561640D0A000D0A77
:10FC3E004F70656E696E67206578697374696E675B
:10FC4E0020257320000D0A4461746120706F727458
:10FC5E00206973202558202D204F4B000D0A476F29
:10FC6E007420256C7520202D20726573657474695F
:10FC7E006E6700202558202558202558202558200D
:10FC8E00256C752020200A000D0A57726F746520AE
:10FC9E006469736B6E6F3A20256420000D0A5761FC
:10FCAE006974696E6720666F7220636172642000EA
:10FCBE003C6964656E743E202558202558202564C5
:10FCCE00202564000D0A46696C6520257320697332
:10FCDE00206F70656E20000D0A7274635F7265612D
:10FCEE00642825642C255829000D0A4F70656E690D
:10FCFE006E67206E657720257320000D0A25303241
:10FD0E005825303258204578697420004E6F742083
:10FD1E0061204C4946206469736B0D0A000D0A522E
:10FD2E0065616420646573637269626520000D0A03
:10FD3E0046696C6520255820697320257320000DB7
:10FD4E000A4469736B20255820697320257320009F
:10FD5E002041544E2061737365727465642025646E
:10FD6E00000D0A487374206279746573322025641D
:10FD7E00000D0A5772697465206661696C202564EE
:10FD8E00000D0A52656164696E67205254430D0A74
:10FD9E00000D0A416D69676F2039313231440D0A09
:10FDAE00000D0A53532F38302039313232440D0AA8
:10FDBE00000D0A44736B73656C20697320256420F3
:10FDCE00000D0A52656164202564206279746573A2
:10FDDE0000566563746F722069732025580D0A00F2
:10FDEE000D0A535338306578656320256420002250
:10FDFE002A2B2C3A3B3C3D3E3F5B5D7C7F000D0A3F
:10FE0E004F70656E696E672025732020000D0A44C1
:10FE1E006562756720697320256420000D0A507293
:10FE2E006F746F20697320256420000D0A5265617E
:10FE3E006420636F6E66696720000D0A46696C6503
:10FE4E006E616D6520257320000D0A466F726D611F
:10FE5E007474696E67200072633D25752046525F8B
:10FE6E0025730D0A002A2A204E4F204449534B2059
:10FE7E002A2A002A2A20566572696679202A2A00C3
:10FE8E000D0A73627974657331202564000D0A4181
:10FE9E00737365727420454F49000D0A4173736583
:10FEAE0072742041544E000D0A4E6F2063617264CD
:10FEBE002025640064657363726962652E636667EC
:10FECE00002F6C6966646174612E62696E00EB7658
:10FEDE00904558464154202020000D0A4D6F756EF6
:10FEEE0074696E67200041707220323220323032D7
:10FEFE0031000D0A41737365727420505000202535
:10FF0E005820772041544E20004C6F6164696E6713
:10FF1E002E2E2E002A2A20525141202A2A00466DCA
:10FF2E00742065786974200031393A31383A3338A3
:10FF3E00005B2532582025645D004572726F722079
:10FF4E0025640048504469736B20004E6F20636136
:10FF5E007264002D3E202558200072633D256420DA
:10FF6E000044534B53454C004E414D4525580044DB
:10FF7E0049534B2558000D0A44534A004641543309
:10FF8E00320044454255470050524F544F0052657F
:10FF9E00616479007B4552527D00302E3138004924
:10FFAE0046432000454F49200052454E20005352F3
:10FFBE0051200044415620004E444143004E5246CB
:10FFCE0044004641540052544300434C4B002025FC
:10FFDE005800253258004430004431004432004469
:10FFEE0033004434004435004436004437002B00BF
:01FFFE000002
:020000040020DA
:10000000FF0FFF0FFF0FFF0FFF0FFF0FFF0FFF0F80
:020000040030CA
:0C0000008CFFFFFC8EFFFFFFFFFFFFFFE7
:00000001FF
